:020000040800F2
:10800000000001208DE6000871DA000875DA00082A
:1080100079DA00087DDA000881DA00080000000043
:1080200000000000000000000000000085DA0008E9
:1080300089DA0008000000008DDA000891DA0008F3
:10804000D5E60008D5E60008D5E60008D5E6000824
:10805000D5E60008D5E60008D5E60008D5E6000814
:10806000D5E60008D5E60008D5E6000895DA000850
:10807000C5DA0008D1DA0008D5E60008D5E6000820
:10808000DDDA0008E9DA0008F5DA0008D5E60008CC
:1080900025DB0008D5E60008D5E60008D5E600088F
:1080A000D5E60008D5E60008D5E60008D5E60008C4
:1080B000D5E6000855DB0008D5E60008D5E600083F
:1080C000D5E60008D5E60008D5E60008D5E60008A4
:1080D000D5E6000885DB000891DB0008BDDB000861
:1080E000D5E60008D5E60008D5E600080000000047
:1080F0000000000000000000000000000000000080
:108100000000000000000000D5E60008D5E60008E9
:10811000D5E60008E9DB0008D5E60008D5E600084A
:10812000D5E60008D5E60008D5E60008D5E6000843
:10813000D5E60008D5E60008D5E6000815DC0008FD
:10814000D5E6000845DC0008D5E60008D5E60008BD
:10815000000000000000000000000000000000001F
:10816000000000000000000000000000000000000F
:1081700000000000000000000000000000000000FF
:1081800000000000000000000000000000000000EF
:1081900000000000000000000000000000000000DF
:1081A00000000000000000000000000000000000CF
:1081B00000000000000000000000000000000000BF
:1081C00000000000000000000000000000000000AF
:1081D000000000000000000000000000000000009F
:0881E0005FF8E0F166666666D7
:1081E80010B5054C237833B9044B13B10448AFF3E9
:1081F80000800123237010BD5802002000000000F9
:108208003473010808B5034B1BB103490348AFF3A6
:10821800008008BD000000005C02002034730108E3
:10822800034613F8012B002AFBD1181A01387047AE
:1082380081F0004102E000BF83F0004330B54FEA0F
:1082480041044FEA430594EA050F08BF90EA020F7C
:108258001FBF54EA000C55EA020C7FEA645C7FEA0F
:10826800655C00F0E2804FEA5454D4EB5555B8BF32
:108278006D420CDD2C4480EA020281EA030382EAA3
:10828800000083EA010180EA020281EA0303362D35
:1082980088BF30BD11F0004F4FEA01314FF4801C08
:1082A8004CEA113102D0404261EB410113F0004F1A
:1082B8004FEA03334CEA133302D0524263EB4303D1
:1082C80094EA050F00F0A780A4F10104D5F1200E6F
:1082D8000DDB02FA0EFC22FA05F2801841F10001CA
:1082E80003FA0EF2801843FA05F359410EE0A5F19E
:1082F80020050EF1200E012A03FA0EFC28BF4CF0CF
:10830800020C43FA05F3C01851EBE37101F0004584
:1083180007D54FF0000EDCF1000C7EEB00006EEB91
:108328000101B1F5801F1BD3B1F5001F0CD349081B
:108338005FEA30004FEA3C0C04F101044FEA445272
:1083480012F5800F80F09A80BCF1004F08BF5FEAF9
:10835800500C50F1000041EB045141EA050130BDD9
:108368005FEA4C0C404141EB0101013C28BFB1F5EB
:10837800801FE9D291F0000F04BF01460020B1FA36
:1083880081F308BF2033A3F10B03B3F120020CDA09
:108398000C3208DD02F1140CC2F10C0201FA0CF0E7
:1083A80021FA02F10CE002F11402D8BFC2F1200C4C
:1083B80001FA02F120FA0CFCDCBF41EA0C01904002
:1083C800E41AA2BF01EB0451294330BD6FEA04044B
:1083D8001F3C1CDA0C340EDC04F11404C4F1200236
:1083E80020FA04F001FA02F340EA030021FA04F348
:1083F80045EA030130BDC4F10C04C4F1200220FA9F
:1084080002F001FA04F340EA0300294630BD21FADC
:1084180004F0294630BD94F0000F83F4801306BFA2
:1084280081F480110134013D4EE77FEA645C18BF96
:108438007FEA655C29D094EA050F08BF90EA020F2D
:1084480005D054EA000C04BF1946104630BD91EA25
:10845800030F1EBF0021002030BD5FEA545C05D128
:108468004000494128BF41F0004130BD14F5800467
:108478003CBF01F5801130BD01F0004545F0FE41DB
:1084880041F470014FF0000030BD7FEA645C1ABF10
:10849800194610467FEA655C1CBF0B46024650EA47
:1084A800013406BF52EA033591EA030F41F4002173
:1084B80030BD00BF90F0000F04BF0021704730B5F9
:1084C8004FF4806404F132044FF000054FF00001CE
:1084D80050E700BF90F0000F04BF0021704730B58F
:1084E8004FF4806404F1320410F0004548BF404264
:1084F8004FF000013EE700BF42004FEAE2014FEAB9
:1085080031014FEA02701FBF12F07F4393F07F4F93
:1085180081F06051704732F07F4208BF704793F096
:108528007F4F04BF41F40021704730B54FF46074A9
:1085380001F0004521F000411CE700BF50EA0102AC
:1085480008BF704730B54FF000050AE050EA010255
:1085580008BF704730B511F0004502D5404261EBC5
:1085680041014FF4806404F132045FEA915C3FF406
:10857800D8AE4FF003025FEADC0C18BF03325FEAA3
:10858800DC0C18BF033202EBDC02C2F1200300FA54
:1085980003FC20FA02F001FA03FE40EA0E0021FA79
:1085A80002F11444BDE600BF70B54FF0FF0C4CF467
:1085B800E06C1CEA11541DBF1CEA135594EA0C0F19
:1085C80095EA0C0F00F0DEF82C4481EA030621EA54
:1085D8004C5123EA4C5350EA013518BF52EA03358F
:1085E80041F4801143F4801338D0A0FB02CE4FF041
:1085F8000005E1FB02E506F00042E0FB03E54FF071
:108608000006E1FB03569CF0000F18BF4EF0010E68
:10861800A4F1FF04B6F5007F64F5407404D25FEA64
:108628004E0E6D4146EB060642EAC62141EA555117
:108638004FEAC52040EA5E504FEACE2EB4F1FD0C59
:1086480088BFBCF5E06F1ED8BEF1004F08BF5FEAD7
:10865800500E50F1000041EB045170BD06F0004689
:1086680046EA010140EA020081EA0301B4EB5C0436
:10867800C2BFD4EB0C0541EA045170BD41F480112E
:108688004FF0000E013C00F3AB8014F1360FDEBF53
:10869800002001F0004170BDC4F10004203C35DA2F
:1086A8000C341BDC04F11404C4F1200500FA05F3B2
:1086B80020FA04F001FA05F240EA020001F0004253
:1086C80021F0004110EBD37021FA04F642EB0601C9
:1086D8005EEA430E08BF20EAD37070BDC4F10C04F3
:1086E800C4F1200500FA04F320FA05F001FA04F2B7
:1086F80040EA020001F0004110EBD37041F10001A3
:108708005EEA430E08BF20EAD37070BDC4F12005AD
:1087180000FA05F24EEA020E20FA04F301FA05F215
:1087280043EA020321FA04F001F0004121FA04F2BD
:1087380020EA020000EBD3705EEA430E08BF20EA8D
:10874800D37070BD94F0000F0FD101F000464000C7
:1087580041EB010111F4801F08BF013CF7D041EA49
:10876800060195F0000F18BF704703F0004652004D
:1087780043EB030313F4801F08BF013DF7D043EA1E
:108788000603704794EA0C0F0CEA135518BF95EAD4
:108798000C0F0CD050EA410618BF52EA4306D1D15B
:1087A80081EA030101F000414FF0000070BD50EA7A
:1087B800410606BF1046194652EA430619D094EA04
:1087C8000C0F02D150EA013613D195EA0C0F05D1EE
:1087D80052EA03361CBF104619460AD181EA030142
:1087E80001F0004141F0FE4141F470014FF00000FA
:1087F80070BD41F0FE4141F4780170BD70B54FF095
:10880800FF0C4CF4E06C1CEA11541DBF1CEA135514
:1088180094EA0C0F95EA0C0F00F0A7F8A4EB0504F6
:1088280081EA030E52EA03354FEA013100F08880ED
:108838004FEA03334FF0805545EA131343EA1263B6
:108848004FEA022245EA111545EA10654FEA00266B
:108858000EF000419D4208BF964244F1FD0404F524
:10886800407402D25B084FEA3202B61A65EB030580
:108878005B084FEA32024FF480104FF4002CB6EB3D
:10888800020E75EB030E22BFB61A754640EA0C00BD
:108898005B084FEA3202B6EB020E75EB030E22BFFD
:1088A800B61A754640EA5C005B084FEA3202B6EB3E
:1088B800020E75EB030E22BFB61A754640EA9C00FD
:1088C8005B084FEA3202B6EB020E75EB030E22BFCD
:1088D800B61A754640EADC0055EA060E18D04FEA8B
:1088E800051545EA16754FEA06164FEAC30343EA2B
:1088F80052734FEAC2025FEA1C1CC0D111F4801FF8
:108908000BD141EA00014FF000004FF0004CB6E7F0
:1089180011F4801F04BF01430020B4F1FD0C88BF8F
:10892800BCF5E06F3FF6AFAEB5EB030C04BFB6EB9A
:10893800020C5FEA500C50F1000041EB045170BD8D
:108948000EF0004E4EEA113114EB5C04C2BFD4EBBA
:108958000C0541EA045170BD41F480114FF0000E3E
:10896800013C90E645EA060E8DE60CEA135594EABA
:108978000C0F08BF95EA0C0F3FF43BAF94EA0C0FBD
:108988000AD150EA01347FF434AF95EA0C0F7FF432
:1089980025AF104619462CE795EA0C0F06D152EA86
:1089A80003353FF4FDAE1046194622E750EA41066A
:1089B80018BF52EA43067FF4C5AE50EA41047FF47B
:1089C8000DAF52EA43057FF4EBAE12E74FF0FF3CE0
:1089D80006E000BF4FF0010C02E000BF4FF0010CB1
:1089E8004DF804CD4FEA410C7FEA6C5C4FEA430C2A
:1089F80018BF7FEA6C5C1BD001B050EA410C0CBF79
:108A080052EA430C91EA030F02BF90EA020F0020DA
:108A1800704710F1000F91EA030F58BF994208BF41
:108A280090422CBFD8176FEAE37040F001007047FE
:108A38004FEA410C7FEA6C5C02D150EA013C07D155
:108A48004FEA430C7FEA6C5CD6D152EA033CD3D0A0
:108A58005DF8040B704700BF8446104662468C469A
:108A68001946634600E000BF01B5FFF7B7FF0028CD
:108A780048BF10F1000F01BD4DF808EDFFF7F4FFF6
:108A88000CBF012000205DF808FB00BF4DF808ED81
:108A9800FFF7EAFF34BF012000205DF808FB00BFA4
:108AA8004DF808EDFFF7E0FF94BF012000205DF8C6
:108AB80008FB00BF4DF808EDFFF7CEFF94BF01207B
:108AC80000205DF808FB00BF4DF808EDFFF7C4FF74
:108AD80034BF012000205DF808FB00BF4FEA410CBD
:108AE8007FEA6C5C02D150EA013C0AD14FEA430CA0
:108AF8007FEA6C5C02D152EA033C02D14FF00000DD
:108B080070474FF0010070474FEA410212F500121A
:108B180015D211D56FF47873B3EB625212D94FEABC
:108B2800C12343F0004343EA505311F0004F23FAA6
:108B380002F018BF404270474FF00000704750EAFB
:108B4800013005D111F0004008BF6FF000407047B8
:108B58004FF00000704700BF4FEA4102B2F1E04316
:108B680024BFB3F5001CDCF1FE5C0DD901F0004C0C
:108B78004FEAC0024CEA5070B2F1004F40EB83005C
:108B880008BF20F00100704711F0804F21D113F188
:108B98003872BCBF01F00040704741F480114FEAC1
:108BA8005252C2F11802C2F1200C10FA0CF320FA4A
:108BB80002F018BF40F001004FEAC1234FEAD32367
:108BC80003FA0CFC40EA0C0023FA02F34FEA4303D1
:108BD800CCE77FEA625307D150EA01331EBF4FF05A
:108BE800FE4040F44000704701F0004040F0FE4075
:108BF80040F40000704700BF80F0004002E000BF72
:108C080081F0004142001FBF5FEA410392EA030F6F
:108C18007FEA226C7FEA236C6AD04FEA1262D2EBB9
:108C28001363C1BFD218414048404140B8BF5B42BE
:108C3800192B88BF704710F0004F40F4000020F057
:108C48007F4018BF404211F0004F41F4000121F06D
:108C58007F4118BF494292EA030F3FD0A2F10102B7
:108C680041FA03FC10EB0C00C3F1200301FA03F1F5
:108C780000F0004302D5494260EB4000B0F5000F18
:108C880013D3B0F1807F06D340084FEA310102F1D7
:108C98000102FE2A51D2B1F1004F40EBC25008BF89
:108CA80020F0010040EA03007047490040EB000053
:108CB800013A28BFB0F5000FEDD2B0FA80FCACF154
:108CC800080CB2EB0C0200FA0CF0AABF00EBC25081
:108CD80052421843BCBFD0401843704792F0000F6F
:108CE80081F4000106BF80F400000132013BB5E7C2
:108CF8004FEA41037FEA226C18BF7FEA236C21D038
:108D080092EA030F04D092F0000F08BF084670479C
:108D180090EA010F1CBF0020704712F07F4F04D16A
:108D2800400028BF40F00040704712F100723CBF7D
:108D380000F50000704700F0004343F0FE4040F4A7
:108D4800000070477FEA226216BF08467FEA236365
:108D58000146420206BF5FEA412390EA010F40F450
:108D6800800070474FF0000304E000BF10F000439C
:108D780048BF40425FEA000C08BF704743F0964383
:108D880001464FF000001CE050EA010208BF70479E
:108D98004FF000030AE000BF50EA010208BF704725
:108DA80011F0004302D5404261EB41015FEA010C3A
:108DB80002BF84460146002043F0B64308BFA3F132
:108DC8008053A3F50003BCFA8CF2083AA3EBC25314
:108DD80010DB01FA02FC634400FA02FCC2F1200233
:108DE800BCF1004F20FA02F243EB020008BF20F06A
:108DF8000100704702F1200201FA02FCC2F12002D0
:108E080050EA4C0021FA02F243EB020008BF20EAC4
:108E1800DC7070474FF0FF0C1CEAD0521EBF1CEAF2
:108E2800D15392EA0C0F93EA0C0F6FD01A4480EAE0
:108E3800010C400218BF5FEA41211ED04FF00063C9
:108E480043EA501043EA5111A0FB01310CF00040F5
:108E5800B1F5000F3EBF490041EAD3715B0040EA1B
:108E6800010062F17F02FD2A1DD8B3F1004F40EBEB
:108E7800C25008BF20F00100704790F0000F0CF0BE
:108E8800004C08BF49024CEA502040EA51207F3A82
:108E9800C2BFD2F1FF0340EAC250704740F400005D
:108EA8004FF00003013A5DDC12F1190FDCBF00F04E
:108EB80000407047C2F10002410021FA02F1C2F1FC
:108EC800200200FA02FC5FEA310040F1000053EA98
:108ED8004C0308BF20EADC70704792F0000F00F0E6
:108EE800004C02BF400010F4000F013AF9D040EAEC
:108EF8000C0093F0000F01F0004C02BF490011F480
:108F0800000F013BF9D041EA0C018FE70CEAD1537D
:108F180092EA0C0F18BF93EA0C0F0AD030F0004CFD
:108F280018BF31F0004CD8D180EA010000F00040B1
:108F3800704790F0000F17BF90F0004F084691F06F
:108F4800000F91F0004F14D092EA0C0F01D14202A9
:108F58000FD193EA0C0F03D14B0218BF084608D172
:108F680080EA010000F0004040F0FE4040F40000BC
:108F7800704740F0FE4040F4400070474FF0FF0C4F
:108F88001CEAD0521EBF1CEAD15392EA0C0F93EA96
:108F98000C0F69D0A2EB030280EA010C49024FEAE8
:108FA800402037D04FF0805343EA111143EA1013A1
:108FB8000CF000408B4238BF5B0042F17D024FF459
:108FC800000C8B4224BF5B1A40EA0C00B3EB510F34
:108FD80024BFA3EB510340EA5C00B3EB910F24BF1D
:108FE800A3EB910340EA9C00B3EBD10F24BFA3EBA2
:108FF800D10340EADC001B0118BF5FEA1C1CE0D16A
:10900800FD2A3FF650AF8B4240EBC25008BF20F01C
:10901800010070470CF0004C4CEA50207F32C2BF70
:10902800D2F1FF0340EAC250704740F400004FF00D
:109038000003013A37E792F0000F00F0004C02BF3E
:10904800400010F4000F013AF9D040EA0C0093F008
:10905800000F01F0004C02BF490011F4000F013B62
:10906800F9D041EA0C0195E70CEAD15392EA0C0FCA
:1090780008D142027FF47DAF93EA0C0F7FF470AF02
:10908800084676E793EA0C0F04D14B023FF44CAF45
:1090980008466EE730F0004C18BF31F0004CCAD1DA
:1090A80030F000427FF45CAF31F000437FF43CAF16
:1090B8005FE700BF4FF0FF3C06E000BF4FF0010C38
:1090C80002E000BF4FF0010C4DF804CD4FEA40021A
:1090D8004FEA41037FEA226C18BF7FEA236C11D064
:1090E80001B052EA530C18BF90EA010F58BFB2EB17
:1090F800030088BFC81738BF6FEAE17018BF40F097
:10910800010070477FEA226C02D15FEA402C05D14A
:109118007FEA236CE4D15FEA412CE1D05DF8040BCF
:10912800704700BF844608466146FFE70FB5FFF762
:10913800C9FF002848BF10F1000F0FBD4DF808ED1A
:10914800FFF7F4FF0CBF012000205DF808FB00BF0B
:109158004DF808EDFFF7EAFF34BF012000205DF865
:1091680008FB00BF4DF808EDFFF7E0FF94BF0120B2
:1091780000205DF808FB00BF4DF808EDFFF7D2FFAF
:1091880094BF012000205DF808FB00BF4DF808EDF2
:10919800FFF7C8FF34BF012000205DF808FB00BFBF
:1091A8004FEA4002B2F1FE4F0FD34FF09E03B3EBEC
:1091B80012620DD94FEA002343F0004310F0004F2C
:1091C80023FA02F018BF404270474FF00000704782
:1091D80012F1610F01D1420205D110F0004008BF21
:1091E8006FF0004070474FF00000704753B94AB91C
:1091F800002908BF00281CBF4FF0FF314FF0FF3097
:1092080000F08CB9ADF1080C6DE904CE00F006F859
:10921800DDF804E0DDE9022304B070472DE9F047EA
:10922800089D8E4604468846002B4AD18A42174636
:1092380062D9B2FA82F64EB1C6F1200301FA06F8F5
:1092480020FA03F3B74043EA0808B4404FEA174E40
:10925800B8FBFEF11FFA87FC0EFB118801FB0CF22C
:10926800230C43EA08439A4209D9FB1801F1FF305D
:1092780080F0EB809A4240F2E88002393B449A1A27
:10928800B2FBFEF00EFB102200FB0CFCA3B243EA7B
:1092980002439C4509D9FB1800F1FF3280F0D780C2
:1092A8009C4540F2D4803B44023840EA014000210A
:1092B800A3EB0C031DB10022F340C5E90032BDE861
:1092C800F0878B4205D90DB1C5E900010021084698
:1092D800F5E7B3FA83F1002946D1734502D38242F8
:1092E80000F20881841A6EEB030201209046002DDB
:1092F800E5D0C5E90048E2E7002A00F09180B2FA1B
:1093080082F6002E40F0A5808A1A0121030C4FEA4C
:10931800174E80B2BCB2B2FBFEFC0EFB1C2243EA25
:10932800024304FB0CF29A4207D9FB180CF1FF38F0
:1093380002D29A4200F2E380C4469B1AB3FBFEF2C3
:109348000EFB123302FB04F440EA03439C4207D9A4
:10935800FB1802F1FF3002D29C4200F2CD80024697
:109368001B1B42EA0C40A5E7C1F120068B4022FAFC
:1093780006F71F432EFA06FA4FEA1749BAFBF9F81F
:109388000EFA01FE20FA06F309FB18AA1FFA87FC59
:1093980043EA0E0300FA01FE08FB0CF01C0C44EA39
:1093A8000A44A04202FA01F20AD93C1908F1FF3A2C
:1093B80080F09E80A04240F29B80A8F102083C44C5
:1093C800241A98B2B4FBF9F309FB134403FB0CFC11
:1093D80040EA0444A44509D93C1903F1FF3080F060
:1093E8008580A44540F28280023B3C4443EA084021
:1093F800A4EB0C04A0FB028C64454346E14664D30D
:1094080061D05DB1BEEB030264EB090404FA06F611
:1094180022FA01F31E43CC40C5E9006400214EE75F
:10942800B1FBF2FC010C41EA0E4180B240EA014274
:109438003B46B1FBF7F138463C46B846BE462026C7
:10944800A2EB080241EA0C4165E7014617E710461E
:109458002BE7C6F120012EFA01FCB7400EFA06FEF2
:1094680020FA01F141EA0E014FEA174EBCFBFEF863
:10947800BCB20EFB18CC08FB04F90A0C42EA0C42F9
:10948800B04091454FEA104380B23ED9BA1808F16E
:10949800FF3C01D291451FD8A2EB0902B2FBFEF9AD
:1094A80009FB04F80EFB192A8AB242EA0A4242452D
:1094B80029D2BA1809F1FF31C2D24245C0D2A9F166
:1094C80002013A44BCE7C6459BD2B8EB02036CEBF9
:1094D800070C0138E14694E7A7EB09094A44B2FBB7
:1094E800FEF9A8F1020C09FB04F8DBE703467DE767
:1094F800D04665E70846FAE63B44023A30E7ACF165
:10950800020C3B4419E749469AE7A2EB0902B2FB71
:10951800FEF9C44609FB04F8C4E700BF704700BF62
:1095280080B500AF06220549054805F02FFA034625
:10953800002B01D001F0CAFB00BF80BD74020020DF
:10954800900200200E4B02689A4218D14FF0010C8D
:109558000C4A0D4B11880D4889B21980518889B27F
:109568005980918889B29980D18889B2D980118926
:1095780089B21981528992B25A8180F800C0704725
:109588000024014074020020800200208C02002088
:1095980080B584B000AF3B1D00221A605A609A6003
:1095A8003C4B3D4A1A603B4B4FF480729A60394BF2
:1095B80000221A73374B00221A75364B4FF40022DB
:1095C800DA61344B00225A60324B06221A61314864
:1095D80005F004F90346002B01D001F077FB0323C3
:1095E8007B600123BB600423FB603B1D19462948AF
:1095F80005F084FB0346002B01D001F067FB042330
:109608007B600223BB603B1D1946224805F076FBB0
:109618000346002B01D001F059FB08237B6003238C
:10962800BB603B1D19461B4805F068FB0346002B31
:1096380001D001F04BFB09237B600423BB603B1D79
:109648001946144805F05AFB0346002B01D001F0D7
:109658003DFB10237B600523BB603B1D19460D486D
:1096680005F04CFB0346002B01D001F02FFB112322
:109678007B600623BB603B1D1946064805F03EFB90
:109688000346002B01D001F021FB00BF1037BD4677
:1096980080BD00BF900200200024014080B58AB040
:1096A80000AF786007F1180300221A605A609A60C8
:1096B800DA607B681B68384A934268D1374B9B69EC
:1096C800364A43F400739361344B9B6903F4007387
:1096D8007B617B69314B9B69304A43F0040393619A
:1096E8002E4B9B6903F004033B613B692B4B9B6941
:1096F8002A4A43F008039361284B9B6903F0080347
:10970800FB60FB681823BB610323FB6107F11803A7
:109718001946234807F030FA0323BB610323FB6192
:1097280007F1180319461F4807F026FA1E4B1F4A6F
:109738001A601D4B00225A601B4B00229A601A4B7C
:109748008022DA60184B4FF480721A61164B4FF47E
:1097580080625A61144B20229A61134B4FF4805255
:10976800DA61114806F07AFD0346002B01D001F0BA
:10977800ADFA7B680C4A1A620B4A7B685362002276
:109788000721122006F017FD122006F030FD00BF59
:109798002837BD4680BD00BF0024014000100240AC
:1097A80000080140000C0140C002002008000240EF
:1097B80080B582B000AF03460A46FB711346BB7101
:1097C800FB79072B50D801A252F823F0F59700082F
:1097D800059800081598000825980008359800088D
:1097E800459800085398000863980008BB791A4602
:1097F8004FF48071214807F05AFB36E0BB791A46CE
:109808004FF400711D4807F052FB2EE0BB791A4651
:109818004FF48061194807F04AFB26E0BB791A46E5
:109828004FF40061154807F042FB1EE0BB791A4669
:109838004FF48051114807F03AFB16E0BB791A46FD
:1098480008210F4807F033FB0FE0BB791A464FF4A5
:1098580000410C4807F02BFB07E0BB791A460821AA
:10986800094807F024FB00E000BFFB790749BA79F3
:10987800CA5400BF0837BD4680BD00BF001801406C
:1098880000100140000801400014014004030020BA
:1098980080B483B000AF0346FB71FB79034AD35C05
:1098A80018460C37BD4680BC704700BF0403002033
:1098B80080B582B000AF0346FB71FB79062B3BD81D
:1098C80001A252F823F000BFED980008F9980008AB
:1098D80005990008119900081D99000829990008A0
:1098E800359900080221174807F0CAFA034624E010
:1098F8000421144807F0C4FA03461EE080211248E8
:1099080007F0BEFA034618E08021104807F0B8FABD
:10991800034612E010210E4807F0B2FA03460CE0A5
:1099280008210B4807F0ACFA034606E00221064876
:1099380007F0A6FA034600E0002318460837BD469C
:1099480080BD00BF0008014000180140001401401C
:10995800000C014080B483B000AF02237B600F4B42
:109968009B690E4A43F0100393610C4B9B6903F00B
:1099780010033B603B680A4B5B6823F470227B68EA
:109988001B04074913434B60054B4FF080521A6183
:1099980000BF0C37BD4680BC704700BF00100240B6
:1099A8000010014080B500AFFFF7D4FF00224FF44C
:1099B8008051184807F07BFA174805F099FBFFF724
:1099C800AFFD00210020FFF7F3FE00210120FFF783
:1099D800EFFE00210220FFF7EBFE00210320FFF736
:1099E800E7FE00210420FFF7E3FE00210520FFF732
:1099F800DFFE00210620FFF7DBFE00210720FFF72E
:109A0800D7FE064803F072FF054803F06FFF00BF5A
:109A180080BD00BF00100140900200200C03002010
:109A28003403002090B587B000AF78600C4B7B61A1
:109A38000C4B3B6179697868FFF7E2F803461C46EE
:109A480039697869FFF7E6F9034619462046FFF7B2
:109A580095FA0346FB60FB6818461C37BD4690BD67
:109A680000007A443211803BB0B586B000AFF86090
:109A7800B9607A603B60F868FEF72CFD1CA3D3E957
:109A88000023FEF7BBFE02460B4614461D46B86887
:109A9800FEF732FD02460B4620462946FEF784FDB6
:109AA80002460B4610461946FFF756F803467B61F7
:109AB80079687869FFF760FB0346002B01D00E4BED
:109AC80010E079697868FFF79BF8034619467869CA
:109AD800FFF754FA034619463868FFF79BF903461F
:109AE8003B613B6918461837BD46B0BDAFF30080EF
:109AF8000000000000FEAF40000080BF80B588B0C5
:109B080000AF0346FB710023FB61FB79002B03D0F8
:109B18001C4BDB889BB202E01A4B9B889BB2FB6113
:109B2800FB79002B01D0012200E0002213469B00A4
:109B38001344DB00144A1344FA691146184603F02B
:109B4800FAFEB861BB69B3F57A6F01D9142315E041
:109B58000E4B7B610E4B3B610E4BFB60FB683A6919
:109B68007969B869FFF780FF03461846FFF75AFF7F
:109B7800B860B868FFF714FB03461BB218462037D5
:109B8800BD4680BD800200200C03002033335340C3
:109B98000000A04000007A4480B500AF174B184A77
:109BA8001A60164B08225A60144B00229A60134B15
:109BB8000022DA60114B4FF460221A610F4B4FF408
:109BC80080125A610D4B00221A760C4B01225A76EC
:109BD8000A4B01229A76094B0122DA76074B0022BA
:109BE8001A77064B01225A77044805F038FB0346DA
:109BF800002B01D001F06AF800BF80BD5C03002093
:109C08000064004080B500AF174B184A1A60164B25
:109C180010225A60144B00229A60134B0022DA601B
:109C2800114B4FF460221A610F4B4FF480125A61A6
:109C38000D4B00221A760C4B01225A760A4B012250
:109C48009A76094B0122DA76074B00221A77064BDF
:109C580001225A77044805F002FB0346002B01D085
:109C680001F034F800BF80BD840300200068004084
:109C780080B58EB000AF786007F1200300221A602B
:109C88005A609A60DA607B681B68614A934253D1D4
:109C9800604B1B6801335F4A13605E4B1B68012BE6
:109CA8000BD15D4BDB695C4A43F00073D3615A4BBF
:109CB800DB6903F00073FB61FB69574B9B69564AEC
:109CC80043F020039361544B9B6903F02003BB616D
:109CD800BB6901233B6200237B620023BB6207F15F
:109CE800200319464D4806F047FF02233B62022332
:109CF8007B620323FB6207F120031946474806F0FD
:109D08003BFF474B5B683B633B6B23F4C0433B63C0
:109D18003B6B43F0E0633B633B6B43F4C0433B6303
:109D28003F4A3B6B536000220321142006F043FA9C
:109D3800142006F05CFA67E07B681B68394A934296
:109D480062D1354BDB69344A43F08063D361324BCF
:109D5800DB6903F080637B617B692E4B1B680133F1
:109D68002C4A13602B4B1B68012B0BD12A4BDB6948
:109D7800294A43F00073D361274BDB6903F0007372
:109D88003B613B69244B9B69234A43F00803936179
:109D9800214B9B6903F00803FB60FB6820233B62AF
:109DA80000237B620023BB6207F1200319461E488B
:109DB80006F0E2FE40233B6202237B620323FB6240
:109DC80007F120031946184806F0D6FE144B5B68C5
:109DD8007B637B6B43F0E0637B637B6B43F48003C3
:109DE8007B630F4A7B6B5360002200213F2006F003
:109DF800E2F93F2006F0FBF900220321412006F09A
:109E0800DAF9412006F0F3F900BF3837BD4680BDC6
:109E180000640040AC030020001002400014014020
:109E28000000014000680040000C014080B400AF11
:109E3800084B00221A70074B00225A70054B00226B
:109E480062F06902DA7300221A7400BFBD4680BC52
:109E5800704700BFB003002080B500AF1F4B5A7891
:109E68001F4B1B789A4206D01C4B5A781C4B1A7011
:109E78001A4B00221A7000F0E7FB0346002B03D0B0
:109E8800164B0B225A7716E0164B1B7B002B03D080
:109E9800124B07225A770EE0124B5B7B002B03D044
:109EA8000E4B0A225A7706E00C4B9B7F002B02D1FF
:109EB8000A4B00225A77094B5B7F0021184600F0B5
:109EC80047FD0346002B06D0044B5B7F1A46064924
:109ED800052000F045FB00BF80BD00BFB003002097
:109EE800D0030020040900205073010880B582B017
:109EF80000AF0346FB71414B1B78FA799A4203D1B4
:109F08003F4AFB79537075E03C4AFB7913703B4B31
:109F18001B78002B03D13B49072000F021FB374B6E
:109F28001B78012B03D13849072000F019FB334B6C
:109F38001B78022B03D13549072000F011FB2F4B6A
:109F48001B78032B03D13249072000F009FB2B4B68
:109F58001B78042B03D12F49072000F001FB274B66
:109F68001B78052B03D12C49072000F0F9FA234B65
:109F78001B78062B03D12949072000F0F1FA1F4B63
:109F88001B78072B03D12649072000F0E9FA1B4B61
:109F98001B78082B03D12349072000F0E1FA174B5F
:109FA8001B78092B03D12049072000F0D9FA134B5D
:109FB8001B780A2B03D11D49072000F0D1FA0F4B5B
:109FC8001B780B2B03D11A49072000F0C9FA0B4B59
:109FD8001B780C2B03D11749072000F0C1FA074B57
:109FE8001B780D2B03D11449072000F0B9FA044A55
:109FF800FB7953700837BD4680BD00BFCF030020F2
:10A00800B003002064730108787301089073010895
:10A01800A8730108C0730108DC730108FC73010808
:10A028001C7401083C740108547401086C7401081C
:10A0380084740108A0740108B874010880B487B05A
:10A0480000AF134B5B889BB27B61114B5B899BB262
:10A058003B6140F2BA43FB60FB687A6903FB02F29A
:10A068003B69B2FBF3F3BB60BB68A3F2BB6341F689
:10A07800186202FB03F3074A82FB03129211DB17F3
:10A08800D31A7B607B6818461C37BD4680BC704776
:10A0980080020020D34D621080B500AF0E4B1B68C4
:10A0A8009F229A620C4B1B6840F2C112DA620A4B7B
:10A0B8001B684FF4E1729A63074B1B6840F2C712A2
:10A0C8005A630421044808F029FA0021024808F0DC
:10A0D80023F900BF80BD00BFDC11002080B485B02B
:10A0E80000AF0346FB71FB794FF4E17202FB03F307
:10A0F8000B4A82FB03125211DB17D31AFB60094A81
:10A10800FB791370084B1B68FA689A63064B1B6847
:10A1180001225A6300BF1437BD4680BC704700BF98
:10A128001F85EB51D8030020DC11002080B400AF5C
:10A13800024B1B781846BD4680BC7047D8030020E8
:10A1480080B500AFFFF77AFF0346034A1360024B5E
:10A158001B68184680BD00BFD403002080B582B0BC
:10A1680000AFFFF7EDFF7860214B1B78062B02D07C
:10A178001F4B1B7838E07B6842F6F722934201DDDB
:10A18800002331E07B68B3F5FA5F06DB7B6842F2B7
:10A198001072934201DC012326E07B6841F287328A
:10A1A800934206DD7B6841F65832934201DC022374
:10A1B8001AE07B68B3F5FA6F05DB7B68B3F57A6F55
:10A1C80001DC032310E07B6813F57A7F05DB7B68ED
:10A1D800B3F5FA6F01DC042306E07B68054A934275
:10A1E80001DA052300E0062318460837BD4680BD7E
:10A1F8000400002009D5FFFF80B400AF024B1B7894
:10A208001846BD4680BC70470500002080B582B066
:10A2180000AFFFF7A3FF0346FB71FB79062B06D1BE
:10A22800134B06221A70134B00221A701DE0104BB4
:10A238001B78FA799A4206D00D4AFB7913700D4BB8
:10A2480001221A7011E00B4B1B78632B05D8094BC0
:10A258001B780133DAB2074B1A70064B1B78632B55
:10A2680003D9034B1A78044B1A700837BD4680BDD2
:10A2780006000020D90300200500002080B582B028
:10A2880000AF04F07DFA0246224B1B68D31A002B5C
:10A298003CDD04F075FA03461E4A1360FFF7B6FF6B
:10A2A800FFF7AAFF0346FB711B4B1B78BB711B4BC7
:10A2B8001B78002B09D11A4AFB791370194ABB790C
:10A2C8001370164B01221A7021E0154B1B78FA798E
:10A2D8009A420AD0124B1B781A46FB79124907207A
:10A2E80000F03EF90E4AFB7913700E4B1B78BA79D1
:10A2F8009A420CD00B4B1B781A46BB790B490720A6
:10A3080000F02EF9074ABB79137000E000BF083748
:10A31800BD4680BDDC030020D8030020E0030020F8
:10A3280007000020E1030020D0740108EC74010844
:10A3380080B500AF064B074A1A60054805F071FF63
:10A348000346002B01D000F0C1FC00BF80BD00BF58
:10A35800E40300200030024080B485B000AF78608C
:10A368007B681B68094A93420BD1094B5B69084A11
:10A3780043F040035361064B5B6903F04003FB6005
:10A38800FB6800BF1437BD4680BC704700300240F0
:10A398000010024080B584B000AFF860B9607A6000
:10A3A8007B689BB21946B86800F006F87B681846C7
:10A3B8001037BD4680BD000080B485B000AF78601E
:10A3C8000B467B8072B600BF0023FB8145E0284B1B
:10A3D800B3F804349BB2B3F5806F18D3244BB3F8A9
:10A3E80002349BB201335A42C3F30903C2F3090290
:10A3F80058BF53429AB21E4BA3F802241C4BB3F821
:10A4080004349BB2013B9AB2194BA3F80424FB898C
:10A418007A681344164AB2F8002492B21978144B99
:10A428009954134BB3F800349BB201335A42C3F327
:10A438000903C2F3090258BF53429AB20C4BA3F85E
:10A4480000240B4BB3F804349BB201339AB2084B87
:10A45800A3F80424FB890133FB81FA897B889A429B
:10A46800B5D362B600BF00BF1437BD4680BC704785
:10A47800EC03002080B483B000AF72B600BF064B77
:10A48800B3F80434FB8062B600BFFB8818460C376B
:10A49800BD4680BC704700BFEC03002080B582B089
:10A4A80000AF72B600BF2D4BB3F804349BB2002B3B
:10A4B80002D162B600BF4EE0284BB3F80434FB80EB
:10A4C800FB88802B01D98023FB80244BB3F802340E
:10A4D8009BB2C3F58063BB80FA88BB889A4201D9D6
:10A4E800BB88FB801D4BB3F804349BB2FA889A42B0
:10A4F8000CD11A4BB3F802349BB21A46174B1344CB
:10A50800F9885022184602F053FE0BE0134BB3F8BB
:10A5180002349BB21A46114B1344F988512218464B
:10A5280002F046FE0D4BB3F802349AB2FB8813448E
:10A538009BB2C3F309039AB2084BA3F80224074B52
:10A54800B3F804349AB2FB88D31A9AB2034BA3F82F
:10A55800042462B600BF0837BD4680BDEC03002066
:10A568000EB480B585B000AF0346FB71154AFB7980
:10A57800137007F12003BB60BB68FA697E2112489B
:10A588000AF08CFDF860FB68002B01DAFB6812E02A
:10A59800FB687D2B01DD7E23FB60FB680133094AE4
:10A5A8000021D154FB689BB202339BB2194605487F
:10A5B800FFF702FFFB6818461437BD46BDE8804028
:10A5C80003B07047F4070020F507002080B582B07B
:10A5D80000AF1C4B5B691B4A43F001035361194BE5
:10A5E8005B6903F001037B607B68002201210B207B
:10A5F80005F0E1FD0B2005F0FAFD002204210C20F6
:10A6080005F0D9FD0C2005F0F2FD002201210D20F6
:10A6180005F0D1FD0D2005F0EAFD002201211020F2
:10A6280005F0C9FD102005F0E2FD002204211120EB
:10A6380005F0C1FD112005F0DAFD00BF0837BD4661
:10A6480080BD00BF0010024080B400AF024B1B78F1
:10A658001846BD4680BC70477408002080B500AF1E
:10A66800064B1B78002B07D1044B01221A700449B2
:10A678000420FFF775FF00E000BF80BD74080020CC
:10A688000875010880B58AB000AF07F114030022ED
:10A698001A605A609A60DA60944B9B69934A43F057
:10A6A80010039361914B9B6903F010033B613B6975
:10A6B8008E4B9B698D4A43F0040393618B4B9B69D6
:10A6C80003F00403FB60FB68884B9B69874A43F0EF
:10A6D80008039361854B9B6903F00803BB60BB6863
:10A6E800824B9B69814A43F0400393617F4B9B698E
:10A6F80003F040037B607B687C4B9B697B4A43F09B
:10A7080020039361794B9B6903F020033B603B680E
:10A7180000224FF40F71764806F0C9FB002248F278
:10A728006001744806F0C3FB00224FF4F8517248E8
:10A7380006F0BDFB00224FF44861704806F0B7FBF5
:10A74800002218216E4806F0B2FB4FF401737B61BA
:10A758000123BB610023FB6103233B6207F1140360
:10A768001946634806F008FA38237B610123BB6168
:10A778000023FB6102233B6207F1140319465C487E
:10A7880006F0FAF902237B610023BB610023FB6119
:10A7980007F114031946574806F0EEF904237B61C4
:10A7A8000023BB610223FB6107F1140319465148DA
:10A7B80006F0E2F960237B610123BB610023FB61A2
:10A7C80003233B6207F1140319464A4806F0D4F9FB
:10A7D80044F282037B610023BB610023FB6107F124
:10A7E80014031946444806F0C7F94FF4F8537B613F
:10A7F8000123BB610023FB6102233B6207F11403C1
:10A8080019463D4806F0B8F94FF440637B610123CF
:10A81800BB610023FB6103233B6207F11403194664
:10A82800364806F0A9F94FF400437B610123BB6168
:10A838000023FB6102233B6207F1140319462D48EC
:10A8480006F09AF918237B610123BB610023FB61A1
:10A8580002233B6207F114031946294806F08CF9D4
:10A8680080237B610023BB610023FB6107F1140394
:10A878001946234806F080F918237B610023BB6141
:10A888000023FB6107F1140319461C4806F074F90C
:10A8980080237B610123BB610023FB6102233B62B0
:10A8A80007F114031946154806F066F94FF440738A
:10A8B8007B611223BB6103233B6207F11403194632
:10A8C8000E4806F059F90F4B5B687B627B6A43F0D0
:10A8D800E0637B627B6A43F002037B62094A7B6A1E
:10A8E800536000BF2837BD4680BD00BF001002403E
:10A8F800001001400008014000180140000C014010
:10A90800001401400000014080B400AFBFF34F8F36
:10A9180000BF064BDB6803F4E0620449044B1343B1
:10A92800CB60BFF34F8F00BF00BFFDE700ED00E035
:10A938000400FA0580B400AF034B044A9A6000BFD4
:10A94800BD4680BC704700BF00ED00E000800008F5
:10A9580080B485B000AF03460A46FB711346BB714D
:10A96800BB791F2B01D900230EE00023FB73BB79B1
:10A97800084AD35CFA799A4201D00123FB73BB7968
:10A988000449FA79CA54FB7B18461437BD4680BC83
:10A99800704700BF7808002080B584B000AF7860A9
:10A9A80003F0EEFEB8607B68FB60FB68B3F1FF3F25
:10A9B80010D00F4B1B781A46FB681344FB6009E064
:10A9C80001F044FC00F016F8FFF758FC01F000FA1B
:10A9D80002F094FA03F0D4FE0246BB68D31AFA6870
:10A9E8009A42EDD800BF00BF1037BD4680BD00BFFA
:10A9F8008C00002080B582B000AF03F0C1FE786003
:10AA08002A4B1B687A68D31A092B49D9274A7B68CD
:10AA180013600320FEF74CFF0346002B0CBF0123F5
:10AA28000023DBB2FB70FB78002B02D1204B002205
:10AA38001A701F4B1B78002B34D1FB78002B2BD0BE
:10AA48001C4B1B68002B02D11B4B01221A70194B9F
:10AA58001B680A33174A1360164B1B6841F2883289
:10AA6800934202D1144B03221A70124B1B6849F609
:10AA78004042934217D912220021002002F098FB8D
:10AA880000BF0E4B93F84130DBB2212BF9D00A20DE
:10AA980003F080FEFFF738FF064B00221A6002E041
:10AAA80000BF00E000BF0837BD4680BD9808002001
:10AAB800080000209C080020B0030020FC120020A1
:10AAC80080B500AF0B4804F0E9FDFFF765F80948C9
:10AAD80004F0A0FD0346002B01D000F0F7F8022196
:10AAE800044805F048F80346002B01D000F0EEF8C2
:10AAF80000BF80BD5C03002080B582B002AFFFF7C5
:10AB080019FF03F0E5FD06F0F7F900F06FF8FFF71D
:10AB1800B9FDFFF75BFDFEF73BFDFFF73DF8FFF7DB
:10AB280071F801F0F9F903F0DBF903F059FBFFF7CD
:10AB3800FFFB03F001FB03F029FB03F07BFB03F0B1
:10AB480041F9FEF72FFF01F01FF94FF4967003F05B
:10AB580021FE01F013FE02F0A7F91F490720FFF7B5
:10AB6800FFFC02F07DF91D4B1B889BB21A461C495D
:10AB78000720FFF7F5FC194B9B781A46194907205F
:10AB8800FFF7EEFC154B9B889BB21A46134BDB88EC
:10AB98009BB21946114B1B899BB200930B46124975
:10ABA8000720FFF7DDFCFFF78BFF00F0E5F9FFF763
:10ABB8003DF900F0F3FA00F0B7FB0A20FFF7ECFECE
:10ABC80000F08AF8FFF748F900F09EFD0A20FFF729
:10ABD800E3FE00BFEDE700BF20750108C4110020A7
:10ABE80034750108487501085C75010880B59CB08A
:10ABF80000AF07F138033822002118460AF07AFA24
:10AC080007F1240300221A605A609A60DA601A6118
:10AC18003B1D2022002118460AF06CFA0523BB636D
:10AC28004FF480333B6404237B640123BB6401231A
:10AC3800FB644FF48033FB630223BB654FF480331E
:10AC4800FB654FF4E0133B6602237B664FF4C06359
:10AC5800BB664023FB6607F13803184606F01CFA6A
:10AC68000346002B01D000F031F80F237B6202234A
:10AC7800BB620023FB624FF480633B6300237B636A
:10AC880007F124030221184606F01CFD0346002B99
:10AC980001D000F01BF803237B604FF48073BB6086
:10ACA8004FF40043FB603B1D184606F001FF0346C6
:10ACB800002B01D000F00AF8034B01221A6000BFF4
:10ACC8007037BD4680BD00BF7000424280B400AFFF
:10ACD80072B600BF00BFFDE72DE9B04384B000AFF6
:10ACE8002C4B00221A702C4B5B78082B03D1294B74
:10ACF80001221A7602E0274B00221A7603F040FD63
:10AD0800F860244B5B68FA68D31ABB60214AFB6879
:10AD18005360214BD3F80330BA6802FB03F31F4A90
:10AD2800A2FB03239B097B601A4BD3E902237968B2
:10AD380000200C46054612EB040843EB0509154BA9
:10AD4800C3E90289134BD3E90223154BA3FB022362
:10AD5800DB0A104A13610F4B1B7E002B08D00D4BEA
:10AD68001A690C4B5B69D31A0B4AC2F807300CE01E
:10AD7800094B0022DA7100221A7200225A7200224C
:10AD88009A72044B1B69034A536100BF1037BD46D2
:10AD9800BDE8B083A0080020B0030020D34D6210A6
:10ADA800C5B3A29180B582B000AF0346FB71064AD5
:10ADB800FB79D37103F0E4FC0346034A136100BF37
:10ADC8000837BD4680BD00BF0409002080B500AF2C
:10ADD80003F0D6FC0246024B1B69D31A184680BD05
:10ADE8000409002038B5424C424D23462A46012129
:10ADF80004F0A0FD10B96D68EBB203B138BD03F0E3
:10AE0800BFFCC5F305453C4B022D186013D0042D3B
:10AE180017D194E80300394B394A83E80300187ABC
:10AE28001C79D9799B79146282F8240082F825105C
:10AE380082F8263038BD334B94E8030083E80300DA
:10AE480038BD062D11D194E803002F4B83E8030089
:10AE5800188859889A8840BA49BA52BA80B289B2D1
:10AE680092B2C3E902011A6138BD082D3AD0092D02
:10AE7800C4D194E80300214B244D214C93F804C01D
:10AE8800234A85E8030000BA84F806C0A2FB00C282
:10AE980009BAC5E90201C2F38F1013284FF0010E59
:10AEA80094BF002501251B4B84F808E0A3FB01C3D0
:10AEB800E1795B0971456080A3804FEA9212A5721F
:10AEC8009CD999B292B201FB02F2134C1349A4FB2C
:10AED8000242A1F815300D76D308A1F81300C1F885
:10AEE800033038BD0E4B94E8030083E8030038BDF7
:10AEF8004C090020300900202C090020CC08002033
:10AF080004090020C0080020D8080020F408002008
:10AF1800D34D62101F85EB51CDCCCCCCB0030020B3
:10AF2800EC08002080B58AB000AF0E237B610023B7
:10AF3800BB610123FB6100233B6000237B6000238E
:10AF4800BB600023FB6000233B6101233B620123BC
:10AF58003B610E237B623B461946064804F07AFAA9
:10AF68000346002B01D0FFF7B1FE00BF2837BD46CE
:10AF780080BD00BF8403002080B500AF154804F0F1
:10AF88008DFBFEF73FFEFFF7CDFF124804F042FBB2
:10AF98001021104804F0EFFD282200210E480AF085
:10AFA800A9F80D4B0022DA7103F0EAFB03460A4ABE
:10AFB8001361094B49F640425A61074B00221A7641
:10AFC800054B0022DA610021002000F007F800BFDD
:10AFD80080BD00BF840300200409002080B584B030
:10AFE80000AF03460A46FB711346BB7107F108031D
:10AFF8000822002118460AF07DF8FB79002B15D1AC
:10B008000D4B1B7A002B13D0BB79002B0CBF0123EF
:10B018000023DBB23B7207F10803F9791A22F0200A
:10B0280000F066F81420FFF7B7FC02E000BF00E06C
:10B0380000BF1037BD4680BD0409002080B586B02A
:10B0480000AF0346FB710B46BB8013467B8007F1BC
:10B0580008030822002118460AF04CF8FB79002B57
:10B0680040D1BB88952B01D89623BB801F4B1B7EF4
:10B07800002B06D1BB88B3F5FA7F02D340F2F31355
:10B08800BB807B88642202FB03F37B61BB884FF49F
:10B098007A7202FB03F33B617B691B0EDBB23B73E5
:10B0A8007B691B0CDBB27B737B691B0ADBB2BB734E
:10B0B8007B69DBB2FB733B691B0EDBB23B723B69FE
:10B0C8001B0CDBB27B723B691B0ADBB2BB723B69B0
:10B0D800DBB2FB7207F10803F9791C22F02000F0BB
:10B0E80007F800E000BF1837BD4680BD04090020FE
:10B0F80080B58CB000AF3B600346FB710B46BB715B
:10B1080013467B71FB7987F82830BB7987F829309B
:10B118007B7903F03F03DAB297F82A3062F305032C
:10B1280087F82A307B8D0A2262F389137B850A23EC
:10B1380087F82F30BB6A7B610023FB610423BB6166
:10B1480008233B621EE0144804F0C0FB0346002BB2
:10B158000ED007F10C0307F110013A680E4804F00D
:10B16800E6FA034687F82E3097F82E30002B0ED0DB
:10B178000120FFF711FC97F92F30DBB2013BDBB25E
:10B1880087F82F3097F92F30002BDCDC00E000BF68
:10B198003037BD4680BD00BF8403002080B582B033
:10B1A80000AF3B4600221A605A603B460422002149
:10B1B800F020FFF79DFF1420FFF7EEFB3B46062229
:10B1C8000021F020FFF794FF1420FFF7E5FB3B4632
:10B1D80009220021F020FFF78BFF1420FFF7DCFB8A
:10B1E8004D4BB3F81B309BB24C4AA2FB0323DB0840
:10B1F8009BB21A46484BB3F813309BB202FB03F3D9
:10B208001A46474B5B699A4211D9454B5A6913460E
:10B218009B0013445B001A463F4BB3F813309BB2B4
:10B22800B2FBF3F39AB23C4BA3F8112006E03A4B79
:10B23800B3F81B309AB2384BA3F81120364BB3F849
:10B2480011309BB240F23252934208D9324B00225D
:10B2580042F032025A74002242F005029A742E4BD0
:10B26800B3F811309BB21A462B4BB3F80F309BB290
:10B2780002FB03F32B4A82FB03129210DB17D31A4B
:10B288001A46254BC3F80B20254B5B7A002B3ED082
:10B29800214BB3F80F309BB2B3F5FA7F06D10A22DF
:10B2A8004FF496710020FFF7C9FE0BE01A4BB3F874
:10B2B8000F309BB2184AB2F8112092B219460020FA
:10B2C800FFF7BCFE1420FFF767FB134BB3F81330EE
:10B2D8009BB2B3F5F57F17D9114BDB69002B05D16C
:10B2E80003F04EFA03460E4AD36110E003F048FA21
:10B2F80002460B4BDB69D31A42F20F72934206D90E
:10B30800074B01221A7602E0054B0022DA6100BFE2
:10B318000837BD4680BD00BFB0030020CDCCCCCCE3
:10B32800040900206766666698B500AF03F028FA3E
:10B338000246B34B1B68D31AB3F5FA7F20D9B14B39
:10B3480000221A72AF4B00229A72AF4B00221A7178
:10B35800AD4B00221A72AC4B0022DA71AA4B0022C4
:10B368009A71AA4B00229A60A84B0022DA60A74B78
:10B3780000221A61A64B0022DA60A54B00229A60CF
:10B38800A04B1B7A002B03D09E4B1B78002B0CD1B3
:10B39800A04B0022DA7400221A759E4B00225A75BF
:10B3A80000229A759B4B00221A769A4B9B7F002BA2
:10B3B8000CD001210420FEF7FBF903F0E1F9034664
:10B3C800954A13608F4B01221A7010E003F0D8F9E8
:10B3D8000246914B1B68D31A4EF66022934206D957
:10B3E80000210420FEF7E4F9864B00221A7005209C
:10B3F800FEF75EFA03461A46824BDA72814B1B7AD5
:10B40800002B07D07F4B1B7B002B03D17D4B1B7878
:10B41800002B02D17B4B00225A727A4BDB79092B25
:10B4280000F2518101A252F823F000BF5DB4000878
:10B4380091B40008ADB40008EBB400082FB50008BB
:10B4480071B50008DBB5000881B6000831B6000800
:10B45800BBB600086B4B00225A7000210320FEF790
:10B46800A7F9684B1B7A002B00F03181654B1B78DC
:10B47800002B00F02C81634B1B7B002B40F02781B5
:10B488000120FFF78FFC22E1FFF7A0FC0346B3F58C
:10B498007A6F40F21E815B4B01225A720220FFF73D
:10B4A80081FC16E1574B00221A76564B0022DA61CE
:10B4B80000210320FEF77CF9524B5B7A002B03D165
:10B4C8000020FFF76FFC15E1524BDB7D002B00F0ED
:10B4D800028101210020FFF781FD0320FFF762FCB4
:10B4E800F9E0484B9B7A002B07D0464B5B7A002B40
:10B4F80003D00420FFF756FCEFE0FFF767FC034694
:10B5080042F21072934240F2E8803E4B01225A7395
:10B51800404B0A225A770020FFF744FC3F49042099
:10B52800FFF71EF8D9E001210320FEF741F9354B5A
:10B53800DB7A002B03D00520FFF734FCCFE0FFF7C0
:10B5480045FC0346B3F57A7F40F2C9802D4B0122B2
:10B558001A73304B07225A770620FFF723FC30492D
:10B568000420FEF7FDFFBAE02A4BDB7D002B03D059
:10B57800244B5B7A002B03D10620FFF713FCB9E0BC
:10B588000520FEF795F903461C460320FEF780F9CF
:10B5980003469C4217D003F0F3F80246214B1B6880
:10B5A800D31AB3F57A7F40F29C801A4B07225A7758
:10B5B800144B01221A730620FFF7F4FB18490420E4
:10B5C800FEF7CEFF8DE003F0DBF80346154A136063
:10B5D80087E0104B00225A7400229A740D4BB3F87E
:10B5E80015309BB21D2B06D9FFF7F0FB034641F23D
:10B5F8008832934277D90820FFF7D4FB73E000BF65
:10B608002C09002004090020CC080020D8080020BC
:10B61800F4080020B00300205409002074750108C4
:10B62800847501085809002000210320FEF7C0F89E
:10B63800314BDB7A002B07D100210020FFF7CEFC2D
:10B648000720FFF7AFFB50E0FFF7C0FB0346B3F559
:10B658007A7F4AD9284B01221A73284B07225A7736
:10B6680000210020FFF7BAFC0720FFF79BFB2449C5
:10B678000420FEF775FF38E01F4B9B7A002B03D19F
:10B688000920FFF78FFB32E0FFF7A0FB034642F2E9
:10B69800107293422BD9184B01225A73174B0A2266
:10B6A8005A770020FFF77EFB16490420FEF758FF63
:10B6B8001DE0FFF78BFB0346B3F57A6F19D902201B
:10B6C800FFF770FB15E00020FFF76CFB12E000BFEE
:10B6D80010E000BF0EE000BF0CE000BF0AE000BFB2
:10B6E80008E000BF06E000BF04E000BF02E000BFC2
:10B6F80000E000BF00BF98BD04090020B00300208F
:10B7080084750108A475010880B500AF3C4B5B7FC8
:10B71800002B03D03B4800F025FB6FE0384B1B782B
:10B72800032B03D1384800F01DFB67E0344B1B782E
:10B73800012B03D1354800F015FB5FE0304B5B78F7
:10B748000D2B57D801A252F823F000BF8DB700087F
:10B7580095B700089DB70008A5B70008ADB7000861
:10B76800B5B70008BDB70008C5B70008CDB70008D1
:10B77800D5B70008DDB70008E5B70008EDB7000841
:10B78800F5B70008224800F0EDFA37E0214800F04C
:10B79800E9FA33E01B4800F0E5FA2FE01E4800F014
:10B7A800E1FA2BE01C4800F0DDFA27E01B4800F026
:10B7B800D9FA23E0194800F0D5FA1FE0174800F03D
:10B7C800D1FA1BE0154800F0CDFA17E0144800F054
:10B7D800C9FA13E0124800F0C5FA0FE0104800F06B
:10B7E800C1FA0BE00E4800F0BDFA07E00A4800F085
:10B7F800B9FA03E0064800F0B5FA00BF80BD00BF03
:10B80800B003002060000020180000200C00002079
:10B8180024000020300000203C00002048000020C8
:10B828005400002080B487B000AFF860B9601146BA
:10B838001A460B46FB801346BB80FA88BB889A429F
:10B8480001D9BB88FB80BB88002B01D10123BB80B9
:10B85800FA8813461B029A1ABB8892FBF3F3FB8201
:10B86800FB681B781A46FB8AC3F1FF0303FB02F24D
:10B87800BB681B781946FB8A01FB03F31344204A73
:10B8880082FB03121A44D211DB17D31ADAB23B6ACD
:10B898001A70FB685B781A46FB8AC3F1FF0303FB47
:10B8A80002F2BB685B781946FB8A01FB03F3134479
:10B8B800134A82FB03121A44D211DB17D31ADAB2E5
:10B8C8003B6A5A70FB689B781A46FB8AC3F1FF03F0
:10B8D80003FB02F2BB689B781946FB8A01FB03F362
:10B8E8001344074A82FB03121A44D211DB17D31AF6
:10B8F800DAB23B6A9A7000BF1C37BD4680BC7047FD
:10B908008180808042EA002242EA014230B44FF04E
:10B91800180C4FF40075D343564C52E000BF00BFDB
:10B9280000BF00BF00BF00BF00BF00BF00BF00BF17
:10B9380000BF00BF00BF00BF00BF00BF00BF00BF07
:10B9480000BF00BF00BF00BF00BF00BF00BF6561F0
:10B9580000BF00BF00BF00BF00BF00BF00BF00BFE7
:10B9680000BF00BF00BF00BF00BF00BF00BF00BFD7
:10B9780000BF00BF00BF00BF00BF00BF00BF00BFC7
:10B9880000BF00BF00BF00BF00BF00BF00BF00BFB7
:10B9980000BF00BF00BF00BF00BF00BF00BF00BFA7
:10B9A80000BF00BF00BF00BF00BF00BF00BF00BF97
:10B9B80000BF00BF00BF00BFBCF1010C4FEA43034A
:10B9C80055D01A022561A9D400BF00BF00BF00BF2F
:10B9D80000BF00BF00BF00BF00BF00BF00BF00BF67
:10B9E80000BF00BF00BF00BF00BF00BF00BF00BF57
:10B9F80000BF00BF00BF00BF00BF00BF00BF00BF47
:10BA080000BF00BF00BF00BF00BF00BF00BF00BF36
:10BA180000BF00BF00BF00BF00BF00BF00BF00BF26
:10BA280000BF00BF00BF00BF00BF00BF00BF00BF16
:10BA3800656100BF00BF00BF00BF00BF00BF00BFFF
:10BA480000BF00BF00BF00BF00BF00BF00BF00BFF6
:10BA580000BF00BF00BF00BF00BF00BF00BF00BFE6
:10BA680000BF00BFBCF1010C4FEA4303A9D130BCB1
:10BA7800704700BF0010014038B50C46EFF3108541
:10BA880072B6827841780078FFF73CFFA278617837
:10BA98002078FFF737FF85F3108838BD80B485B06C
:10BAA80000AF78607B681B781A4613461B019B1A07
:10BAB8009B00214A82FB03121A44D211DB17D31AC6
:10BAC800DBB23B727B685B781A4613461B019B1AF4
:10BAD8009B00194A82FB03121A44D211DB17D31AAE
:10BAE800DBB27B727B689B781A4613461B019B1A54
:10BAF8009B00114A82FB03121A44D211DB17D31A96
:10BB0800DBB2BB7207F10C0307F108021268114699
:10BB180019800233120C1A7000233A7B62F3070370
:10BB28007A7B62F30F23BA7B62F317431846143704
:10BB3800BD4680BC704700BF8180808080B582B0E0
:10BB480000AF4C4B5B7FBB7102F01AFE3860BB79CB
:10BB5800002B18D1484B00221A70484B00221A704B
:10BB6800474B00221A70474B00221A60464B0022AE
:10BB78001A70464B00221A70444B00225A70434BED
:10BB880000229A7072E0404B1B78BA799A420ED024
:10BB9800394B00221A70394B00221A70384B002298
:10BBA8001A70384B00221A60374ABB791370354B2C
:10BBB8001B683A689A4209D2344BFF221A70334BF9
:10BBC80000225A70314B00229A704FE02F4B00220E
:10BBD8001A702E4B00225A702C4B00229A702C4B54
:10BBE8001B683A68D31A632B3FD9294A3B6813600C
:10BBF8000023FB71224B1B78002B06D0204B1B78AF
:10BC0800013BDAB21E4B1A701EE01B4B1B78BA7947
:10BC18009A4213D9194B1B78002B03D1174B0122D9
:10BC28001A7011E00123FB71144B00221A70124B99
:10BC38001B780133DAB2104B1A7005E00E4B002264
:10BC48001A700F4B1E221A70FB79002B0ED03B681E
:10BC580064330C4A13600D4BFF221A700B4B002201
:10BC68005A700A4B00229A7000E000BF0837BD46A0
:10BC780080BD00BFB00300207209002073090020B6
:10BC880074090020780900207C0900205C09002044
:10BC98008009002080B483B000AF78607B681B788F
:10BCA8001A46642302FB03F3174A82FB03121A4461
:10BCB800D211DB17D21A154B1B689A637B685B7825
:10BCC8001A46642302FB03F30F4A82FB03121A4449
:10BCD800D211DB17D21A0D4B1B68DA637B689B788D
:10BCE8001A46642302FB03F3074A82FB03121A4431
:10BCF800D211DB17D21A054B1B681A6400BF0C3728
:10BD0800BD4680BC704700BF81808080241200201F
:10BD180080B584B000AF78607868FFF7BFFE03464F
:10BD28001A463A73C3F307227A73C3F30743BB7304
:10BD38000B48FFF7B3FE03461A463A72C3F30722CD
:10BD48007A72C3F30743BB7207F1080207F10C03C9
:10BD580011461846FFF790FE00BF1037BD4680BD5C
:10BD68005C09002080B483B000AF7860054B7A6826
:10BD78001068516803C312891A8000BF0C37BD468A
:10BD880080BC70476809002080B582B000AF0023EE
:10BD98003B7100237B710023BB7104210B4806F023
:10BDA800BDFB0821094806F0B9FB0C21074806F03D
:10BDB800B5FB3B1D1846FFF76DFF3B1D1846FFF707
:10BDC800A7FF00BF0837BD4680BD00BF2412002072
:10BDD80080B582B002AF02F0D3FC0246494B1B6823
:10BDE800D31A142B40F28A8002F0CAFC0346454A53
:10BDF8001360454B5B8801339AB2434B5A80424BE0
:10BE08001B78032B67D801A252F823F025BE00083F
:10BE180057BE000883BE0008B5BE00083A4B5A88D2
:10BE28003A4BDB7819463A4B00930B463749394869
:10BE3800FFF7F8FC344B5B88344AD27893424ED9EA
:10BE4800314B01221A70304B00225A8047E02E4BAA
:10BE58002E4A04331268114619800233120C1A70E4
:10BE6800294B5B88294A127993423AD9264B0222F8
:10BE78001A70254B00225A8033E0234B5A88234BF3
:10BE88005B791946224B00930B4622491F48FFF75E
:10BE9800C9FC1D4B5B881D4A5279934223D91A4B22
:10BEA80003221A70184B00225A801CE0164B174ABE
:10BEB800043307321188927819809A70124B5B8884
:10BEC800124A9279934210D90F4B00221A700E4BE6
:10BED80000225A8009E00C4B00221A7006E000BFCD
:10BEE80004E000BF02E000BF00E000BFFFF726FE4D
:10BEF8000748FFF7CFFE0648FFF70AFF00BFBD4619
:10BF080080BD00BF84090020600900206809002066
:10BF1800640900206F09002080B500AF0A4B0B4A66
:10BF28001A60094B4FF0FF325A60074B4FF480728A
:10BF38009A60054806F040F80346002B01D0FEF74A
:10BF4800C5FE00BF80BD00BF880900200028004052
:10BF580080B584B000AF78607B681B680B4A934259
:10BF680010D104F0BDFF0A4BDB69094A43F00063B6
:10BF7800D361074BDB6903F00063FB60FB68054B8B
:10BF880001221A6000BF1037BD4680BD002800405E
:10BF9800001002403C044242024659B370B50C46B8
:10BFA800CB0758BF1549154D48BF144986B054BF33
:10BFB8000B46134B14F0020F0491124908BF29468F
:10BFC80014F0040F104808BF284614F0080F019019
:10BFD8000E480F4E08BF2E4614F0100F18BF054626
:10BFE8000091CDE902650B4905940420FEF7B8FAE3
:10BFF80006B070BD04200849FEF7B2BAB07901084E
:10C00800B8750108BC750108C0750108CC75010830
:10C01800C4750108F4750108D475010830B54FF4EA
:10C028008072054683B01149114807F072FA08B9C1
:10C0380003B030BD04460E4807F07DFE0246234695
:10C0480014460C492A4604200094FEF789FA032076
:10C058002146FFF7A1FF084800F0DCFE002CE7D0DE
:10C06800034803B0BDE8304007F014BBC009002006
:10C0780044130020287601086476010838B51A4B65
:10C088000C46834213D129B3B1F5807F16D802F04C
:10C0980077FB0346154D164A214616482B60136058
:10C0A80000F010FEBDE838401348FFF7B7BF0A4656
:10C0B800BDE8384005201149FEF752BA4FF48073A5
:10C0C8000A4604200E49FEF74BFABDE838400A48F4
:10C0D800FFF7A4BF05200B49FEF742FABDE8384038
:10C0E8000548FFF79BBF00BF44130020D00C002079
:10C0F800D40C0020C0090020F076010880760108E1
:10C1080000770108BC760108F8B5044607F013FE6D
:10C11800294B05469C4232D0284EB44217D0284BB2
:10C128009C4245D00346002226490420FEF718FA0F
:10C1380029460020FFF730FF204607F0ABFA2046DB
:10C1480007F040FA2046BDE8F84001F01FB9034661
:10C1580003221C490420FEF703FA29460320FFF7AF
:10C168001BFF204607F096FA204607F02BFA00221C
:10C17800154B16481A70BDE8F840FFF74FBF02226A
:10C1880017460E4E2B460F490420FEF7E9F92946BB
:10C198003846FFF701FF204607F07CFA204607F0F3
:10C1A80011FAB442E3D02046BDE8F84001F0EEB8F9
:10C1B80005221746E6E700BFFC12002044130020C2
:10C1C8006C12002040770108C20C00208C7701080F
:10C1D80080B582B000AF78607B68164A934224D15C
:10C1E800154B00221A70154B1B88002B1ED0134BC1
:10C1F8001B881A461249134808F0C4FF0E4B012247
:10C208001A700E4B1B881A460E490A4807F0B4F8F4
:10C218000346002B05D0084B00221A700A4800F08C
:10C22800F9FD064B00221A8000E000BF0837BD4622
:10C2380080BD00BF44130020C20C0020C00C0020A9
:10C24800C00B0020C00A00209C77010880B582B08E
:10C2580000AF02F095FA0246A54B1B68D31A002BD3
:10C2680040F36B8202F08CFA0346A14A136000F097
:10C2780097FDA04B1B78002B03D09E4B1A789E4B42
:10C288001A709C4B1B78032B1BD19C4B1B68002BF3
:10C2980005D102F075FA0346984A136014E002F0DB
:10C2A8006FFA0246954B1B68D31A1A4642F20F736F
:10C2B8009A4209DD8F4B00221A70904B00221A60B7
:10C2C80002E08E4B00221A608A4B1B78012B19D191
:10C2D8008B4B1B68002B05D102F052FA0346884AA3
:10C2E800136012E002F04CFA0246854B1B68D31A21
:10C2F800B3F57A7F09DB7F4B00221A70804B00224E
:10C308001A6002E07E4B00221A6002F039FA0246F7
:10C318007C4B1B68D31A0A2B5EDD02F031FA024609
:10C32800794B1B68D31AC72B06DD00F09BFB02F084
:10C3380027FA0346744A1360744B1B78002B08D005
:10C3480073490420FEF70CF900F02CFB6F4B002218
:10C358001A70684B1B78012B07D0664B1B78032B90
:10C3680003D0644B5B7F002B1AD002F009FA024617
:10C37800684B1B68D31AB3F57A7F11DD02F000FA17
:10C388000346644A136064490520FEF7E9F8594BEF
:10C398001B78032B02D16420FDF7A0FE00F002FBFE
:10C3A8005E4B1B780C2B03D05C4B1B780B2B13D1EB
:10C3B80002F0E6F90246574B1B68D31AB3F57A7FA9
:10C3C8000ADD02F0DDF90346524A1360544905209C
:10C3D800FEF7C6F800F0E6FA524B1B68002B0CD0AB
:10C3E80002F0CEF902464F4B1B68D31A1A4641F2A7
:10C3F80088339A4201DD012300E00023FB71494B99
:10C408001B68002B0CD002F0BBF90246454B1B6899
:10C41800D31A1A4642F210739A4201DD012300E052
:10C428000023BB71BB797B71FB79002B0AD03E4B93
:10C438001B78002B06D13D490420FEF791F83A4BB2
:10C4480001221A70BB79002B0AD0394B1B78002BBC
:10C4580006D138490420FEF783F8354B01221A70BB
:10C46800FB79002B05D1304B00221A70304B00228B
:10C478001A70314ABB791370304B1B78052B00F2C8
:10C48800138101A252F823F0A9C40008D1C40008FE
:10C498004DC5000891C50008CDC5000825C600088F
:10C4A80000210520FDF784F90020FDF71FFD244B2E
:10C4B8001B78002B00F0ED807B79002B40F0E980A1
:10C4C8001E4B02221A70E4E000210520FDF770F9E6
:10C4D8000220FDF70BFD074B5B7F002B40F0DB8054
:10C4E8007B79002B40F0D780144B02221A70D2E0DF
:10C4F800280D0020B0030020BC0900202C0D0020CE
:10C50800300D0020B4090020340D0020C30C002099
:10C51800B8770108B8090020CC770108240D00205D
:10C52800E4770108C80C0020CE0C00200078010830
:10C53800CF0C002014780108CD0C0020250D002018
:10C54800D411002001210520FDF732F90120FDF763
:10C55800CDFC7C4B1B78012B03D07A4B1B78022B2C
:10C5680002D1794B03221A70784B5B7F002B00F0C5
:10C578009480764B5B7F1A4675490420FDF7F0FFDF
:10C58800714B01221A7088E001210520FDF710F98E
:10C598000420FDF7ABFC6D4B1B78022B06D16D49CF
:10C5A8000720FDF7DDFF684B04221A70654B1B78E6
:10C5B800002B74D168490720FDF7D2FF624B022295
:10C5C8001A706CE001210520FDF7F2F8634B1B7827
:10C5D800022B03D9614B1B78042B03D10320FDF7F1
:10C5E80085FC04E05D4B1B781846FDF77FFC554B36
:10C5F8001B78002B06D158490720FDF7B1FF524B95
:10C6080002221A70564B1B78002B4AD05549072036
:10C61800FDF7A6FF4C4B05221A7042E000210520C9
:10C62800FDF7C6F80D20FDF761FC02F0A9F80246F7
:10C638004D4B1B68D31AB3F57A7F1ADD02F0A0F8C8
:10C648000346494A1360464B1B78002B0AD0444BDB
:10C658001B78FF2B0DD0424B1B78013BDAB2404BC5
:10C668001A7006E041490720FDF77AFF364B02228F
:10C678001A703B4B1B78002B15D1324B1B78012BC2
:10C6880011D13B490720FDF76BFF2F4B03221A708E
:10C6980009E000BF08E000BF06E000BF04E000BFFB
:10C6A80002E000BF00E000BFBB79002B14D0274B8D
:10C6B8000022DA75294B00221A706420FDF70EFD5E
:10C6C800214B1B78012B24D01F4B1B78002B20D02B
:10C6D8001D4B01221A701CE0264B1B78012B03D13D
:10C6E8001A4B0022DA7514E0234B1B78002B14BF79
:10C6F80001230023DBB21A46144BDA75134BDB7D9A
:10C70800002B06D1114B5B78032B02D10F4B002273
:10C71800DA750C4B1B78012B07D00A4B1B78022BC0
:10C7280003D0084B1B78032B03D1084B01229A77BF
:10C7380004E0064B00229A7700E000BF0837BD46A8
:10C7480080BD00BF05000020250D0020B00300209B
:10C758003C7801086478010888780108240D0020D5
:10C76800C40C002098780108380D0020A87801082A
:10C77800D0780108BC090020BD09002080B500AFB1
:10C78800FDF78AFC6420FDF7A9FC134B4FF47A727D
:10C798001A80114B96225A800F4B40F232529A80DF
:10C7A8000D4B0A22DA800C4B49F640429A6001F0A0
:10C7B800E7FF0346094A1360084B1B68084A1360E1
:10C7C8000848FFF72BFC00F0E3F807490720FDF7BE
:10C7D800C7FE00BF80BD00BF9C090020D00C002010
:10C7E800D40C00200C79010814790108E9B38446B7
:10C7F80000B58E464FF6FF701D49E6441CF8012B24
:10C80800424042F300030B4083EA520343F3000221
:10C818000A40C3F34E035A4042F300030B40C2F3ED
:10C828004E02534043F300020A40C3F34E035A40FA
:10C8380042F300030B40C2F34E02534043F300029D
:10C848000A40C3F34E035A4042F300030B40C2F3BD
:10C858004E02534043F300000840C3F34E035840D0
:10C86800E64580B2CAD15DF804FB4FF6FF70704709
:10C8780001A0FFFF80B586B000AFB9607B600346BA
:10C88800FB731346BB81BB890333FB82FA8A3B8C5B
:10C898009A4201D9002329E07B68FA7B1A70BB8988
:10C8A800002B09D0BB68002B06D07B680133BA89FE
:10C8B800B968184608F066FCBB8901339BB2194673
:10C8C8007868FFF793FF0346BB82BB8901337A6818
:10C8D8001344BA8AD2B21A70BB8A1B0A99B2BB89AE
:10C8E80002337A681344CAB21A70FB8A184618379A
:10C8F800BD4680BD80B586B002AF03463960FB7186
:10C908001346BB80BA88F8794FF480730093194BAB
:10C918003968FFF7AFFF0346FB81FB89002B1FD067
:10C92800154B1B78002B09D0FB891A46114913486F
:10C9380008F028FC124AFB89138011E00E4B0122F3
:10C948001A70FB891A460B490E4806F015FD034676
:10C95800002B05D0084B00221A700B4800F05AFA39
:10C9680001F00EFF0346094A136000BF1037BD46A9
:10C9780080BD00BFC00A0020C20C0020C00B0020F0
:10C98800C00C00204413002020790108B4090020BD
:10C9980080B500AF002200215220FFF7ABFF00BF97
:10C9A80080BD00BF80B500AF002200215320FFF7F3
:10C9B800A1FF00BF80BD00BF80B582B000AF01F00D
:10C9C800DFFE78601E4B1B687A68D31A3B601C4AEE
:10C9D8007B6813601B4BB3F813309BB21A46194B94
:10C9E800B3F815309BB202FB03F3174A82FB03121C
:10C9F8009210DB17D31A1A46144B1A60134B1B6894
:10CA08003A6802FB03F3124AA2FB03239A09114B6B
:10CA18001B6813440F4A13600F4B1B78012B02D17C
:10CA28000C4B00221A600B4B1B680C4AA2FB032319
:10CA3800DB0A0B4A136000BF0837BD4680BD00BF44
:10CA48003C0D0020B003002067666666A809002038
:10CA5800D34D6210AC090020240D0020C5B3A2916B
:10CA6800B009002080B500AFFFF7A6FFFDF75EFB19
:10CA780003461A462E4B1A702E4BDA7A2C4B5A70F4
:10CA88002D4BB3F813309AB2294B5A802B4B1B7895
:10CA9800002B03D0264B4FF4FA725A80264BB3F87A
:10CAA80015309AB2224B9A80254B1B68204AC2F84F
:10CAB8000630244B1B681E4AC2F80A30224B1B78EA
:10CAC800042B04D1214B1A78194BDA7402E0184B65
:10CAD8000022DA741E4B1A88154B9A821C4B5A880E
:10CAE800134BDA821A4B9A88114B1A83184BDA883F
:10CAF8000F4B5A83164B9B680D4AD361154B1A7816
:10CB08000B4B9A740A4A002343F07F4343F47F0394
:10CB180043F43B4343F0A003D381002343F00D03C8
:10CB28001382202202495020FFF7E4FE00BF80BD97
:10CB3800D80C002004090020B0030020CC0C0020F1
:10CB4800A8090020B0090020250D002005000020BC
:10CB58009C090020C60C00204038C0B209289ABFA2
:10CB6800024B33F810004FF6FF707047507D0108F4
:10CB7800F8B504460D4601F003FE0023424A434E31
:10CB88001370434A30601370424A1370A4F1400393
:10CB9800092B71D8DFE803F009145B4E551B2A2EC8
:10CBA8004A0501F0EDFD3060F8BD28783A4B64285D
:10CBB80028BF64201B78394A032B107043D1F8BD75
:10CBC8002B78374A003B18BF01231370F8BD2B8818
:10CBD8009AB2B2F5FA7F43D000202F4A3149A2F821
:10CBE8000F3008706B88A2F81B30F8BD2A782E4BDE
:10CBF8001A70F8BD2D4F2C463E4605F1200C3546DF
:10CC080020686168A268E368103464450FC506F1BE
:10CC18001006F4D16168A268206807C6244A7B8898
:10CC28001D49A2FB0323DB088B70F8BD2A78214B32
:10CC38001A70F8BD2B78204A003B18BF01231370E7
:10CC4800F8BD164B1878BDE8F840FDF747BA2B78C1
:10CC5800002BA9D0BDE8F84005201849FDF780BC95
:10CC6800012200212C240A200E4D0B4B2A701A7425
:10CC7800DC73D8761977F8BD2246BDE8F840052060
:10CC88000F49FDF76DBC00BFCD0C0020C80C00207B
:10CC9800CE0C0020CF0C0020B00300206A0000203A
:10CCA800BD090020CC0C0020C60C0020F80C002088
:10CCB800CDCCCCCC240D0020C50C00203C7901083B
:10CCC800547901082DE9F04102290C46054684B043
:10CCD80030D9431813F8012C13F8027CCE1E023900
:10CCE80089B247EA022790F80080FFF77FFD874264
:10CCF800B6B212D14046FFF72FFF4FF6FF729042AF
:10CD08003AD086422AD13246FEB931464046FFF72C
:10CD18002FFF012004B0BDE8F0810290234642466F
:10CD28000420CDE900671849FDF71AFC002004B07B
:10CD3800BDE8F081D9B1012902784FF0050009D08A
:10CD48006B781249FDF70CFCF0E74046691CFFF7C9
:10CD58000FFFDEE70E49FDF703FCE7E7034642460F
:10CD6800CDE900640B490420FDF7FAFBDEE70A4928
:10CD78000520FDF7F5FBD9E723464246074900960B
:10CD88000520FDF7EDFBD1E7447A0108107A010888
:10CD9800E4790108EC7A0108B4790108A87A010855
:10CDA80080B582B000AF01F0EBFC0246144B1B6863
:10CDB800D31A7B6001F0E4FC0246124B1B68D31ABD
:10CDC8003B607B6840F2DB52934215DD3B6840F2E2
:10CDD800DB52934210DD0C4B93F84230DBB2202B30
:10CDE8000AD10A48FFF71AF9094800F013F801F0C8
:10CDF800C7FC0346034A136000BF0837BD4680BD21
:10CE0800D00C0020D40C002044130020447B0108DF
:10CE1800507B010880B586B004AF78600D4806F0F5
:10CE28008AFF03460B4A92F84120D2B21146094ABA
:10CE380092F84220D2B21046074A12780292019024
:10CE480000917A6805490420FDF78AFB00BF08377E
:10CE5800BD4680BD44130020C20C0020687B010839
:10CE680080B400AF0E4B1B681B689AB20D4B1A803A
:10CE78000B4B1B685A790B4B9A70094B1B681A7934
:10CE8800084BDA70074B01229A80064B0022DA80A1
:10CE9800044B13221A8100BFBD4680BC704700BFF7
:10CEA80000000020C411002080B500AF4FF40472C8
:10CEB80000210D4808F01EF94FF4047200210B48B8
:10CEC80008F018F90A4B00221A7001F059FC0346C1
:10CED800084A1360074B1B68074A136000F014FAEE
:10CEE80000F036FA00BF80BD400D0020500F002032
:10CEF80061110020641100206811002080B500AF86
:10CF080001F03EFC0246214B1B68D31A002B3BDD87
:10CF180001F036FC03461D4A136000F0ADF900F03D
:10CF2800F3F900F015FA1A4B93F84130DBB2212BD4
:10CF380014D1184BD3F80C32002B0FD001F020FC81
:10CF48000246144BD3F80C32D31A642B06DD104872
:10CF580006F038FB0F4B0022C3F80C220D4B93F858
:10CF68000832DBB2002B10D0094B93F84130DBB20A
:10CF7800212B0AD0084800F087FA064B002283F8D4
:10CF8800082200F0C1F900E000BF80BDD0110020E8
:10CF9800FC120020400D0020400F00202E4B70B5E1
:10CFA8001A6803680C46934219D02C4A12689342B7
:10CFB80004D02B4A126893424AD070BD99B32949CC
:10CFC8002246A1F5807000F049F910BB22460520E1
:10CFD8002549FDF7C5FABDE8704000F0B9B991B32D
:10CFE80001F0CEFB0022214B21491A700346214D46
:10CFF800214E2246A1F580702B60336000F02EF997
:10D008000546A8B100221D4B1A70BDE8704000F01B
:10D018007BB90122194B1A481A7000F035FABDE89D
:10D02800704000F095B917490520FDF799FAC6E751
:10D03800224615490520FDF793FA14222946284669
:10D0480000F0B6F8DEE711490520FDF789FAC7E7D1
:10D05800BDE87040FFF712B8FC1200206C120020E7
:10D068004413002050100020FC7B010861110020AF
:10D07800400E00206811002064110020601100207B
:10D0880050110020D87B0108B87B0108947B010867
:10D09800084B1A680368934204D0074A12689342FF
:10D0A80005D070470022054BC3F80C227047FFF7E4
:10D0B8008FB800BFFC12002044130020400D002050
:10D0C800C9B34FF0FF3300B51C4A014410F801EB17
:10D0D8008EEA030E4EF300034EF3400C134083EA2E
:10D0E8005E030CEA020C8CEA530C43F340034CF346
:10D0F800400E134083EA5C030EEA020E8EEA530EDA
:10D1080043F340034EF3400C134083EA5E030CEAFA
:10D11800020C8CEA530C43F3400313404CF3400ECB
:10D1280083EA5C0381420EEA020C8CEA5303CDD1F8
:10D13800D8435DF804FB0846704700BF2083B8ED6C
:10D1480070B51546137060B359B39446022302783C
:10D158004C1EA4B21C440CF8012F05E010F8011F66
:10D16800FB2B0CF8011F20D0A34203F10103F5D1DA
:10D17800A1B24E1CB6B22846FFF7A2FF0346711CA7
:10D18800B21C2B55C3F3072CC3F3074489B292B2E0
:10D19800C3F3076305F806C0F01C6C54AB5480B2A7
:10D1A80070BD012402262146E5E7002070BD00BFBE
:10D1B80038B51346114AFFF7C3FF80B1044610483B
:10D1C80090F84130202B0BD10C4D224629460C48B3
:10D1D80006F0D2F858B901F0D3FAC5F80C0238BDF8
:10D1E80006F0F0F907490520FDF7BAF9ECE704491C
:10D1F8000548BDE8384000F005B900BF400D0020E3
:10D20800FC1200201C7C01084C7C01082DE97841A7
:10D218004B1FFB2B13D804398CB203199D78904609
:10D228005A782D0445EA0225025DDB78154321462C
:10D2380045EA03650646FFF743FF854202D0002012
:10D24800BDE87881731CC8F804303378013C88F84D
:10D25800003088F801400120BDE8788110B5044607
:10D268000846114604F50072FFF7D0FF18B10123F4
:10D27800184684F8083210BD80B582B000AF01F0BE
:10D288007FFA78601A4B1B687A68D31A3B603B6850
:10D2980041F28732934212DD164B1B78DBB2002B2A
:10D2A80009D1154B002283F8082241F2883213492C
:10D2B8000520FDF755F90F4B01221A7002E00D4BBE
:10D2C80000221A700E4B93F84230DBB2202B0AD1A1
:10D2D8000C4B1B687A68D31AC72B04DD00F014F8CE
:10D2E800084A7B68136000BF0837BD4680BD00BF91
:10D2F8006411002061110020400D0020687C0108A5
:10D30800FC1200206811002080B500AF0C4B93F888
:10D318004230DBB2202B11D10A4B93F80832DBB232
:10D32800002B0BD1FF220849054806F0F2F8034606
:10D33800002B03D00249054800F064F800BF80BD07
:10D34800FC120020400D0020400E00208C7C0108BB
:10D3580080B500AF0A4B93F84230DBB2202B0DD1D9
:10D36800FF220849064806F077F80346002B04D048
:10D378000349054800F046F800E000BF80BD00BF43
:10D388006C12002050100020A47C010880B582B0E7
:10D3980000AF78607B68154A934215D11349144849
:10D3A80000F030F8114806F075F9104806F00AF94F
:10D3B800104B0022C3F80C22FFF7A6FF01F0E0F99A
:10D3C80003460D4A13600CE07B680C4A934208D16F
:10D3D8000A490B4800F016F8084806F05BF9FFF711
:10D3E800B7FF00BF0837BD4680BD00BFFC12002054
:10D3F800BC7C0108400D0020681100206C12002040
:10D40800D07C010890B587B004AF786039607B683C
:10D41800002B1CD03B68002B19D03B681B681C46AE
:10D42800386806F088FC02463B6893F84130DBB266
:10D4380019463B6893F84230DBB20293019100929F
:10D4480023467A6804490420FDF78AF800E000BF03
:10D458000C37BD4690BD00BFE47C010880B400AF26
:10D46800BFF34F8F00BF064BDB6803F4E06204494B
:10D47800044B1343CB60BFF34F8F00BF00BFFDE7E2
:10D4880000ED00E00400FA0580B584B000AF7860D4
:10D498001323FB737B681B78C22B00F3D180B02B5E
:10D4A8000FDA602B42D0602B00F3CA80502B43D098
:10D4B800502B00F3C580012B00F0AB80402B2DD002
:10D4C800BEE0B03B122B00F2BB8001A252F823F061
:10D4D80047D5000849D6000849D6000849D60008AB
:10D4E80049D60008F9D5000849D60008EFD5000844
:10D4F80049D6000849D6000849D6000849D6000888
:10D5080049D6000849D6000849D6000849D6000877
:10D5180085D50008E9D50008BDD5000800F0B6F8A3
:10D52800402258214D48FFF743FE94E060220A212B
:10D538004B48FFF73DFE8EE0FCF7B0FF8BE07B68C1
:10D548005B780B2B17D17B685A68464B106851687B
:10D5580003C31189927A19809A70434B01221A7079
:10D56800404BD3F803303F4A40490720FCF7F8FF07
:10D578001223FB7367E01323FB7364E07B685B781B
:10D58800012B14D17B685B681B781A464FF47A73B9
:10D5980002FB03F31A46364B5A61354B5B691A4650
:10D5A80034490720FCF7DCFF1223FB734BE01323FD
:10D5B800FB7348E07B685B78012B0ED17B685B6866
:10D5C8001A782D4B1A702C4B1B781A462B490720BA
:10D5D800FCF7C6FF1223FB7335E01323FB7332E01D
:10D5E8001323FB732FE0FDF739F81223FB732AE0AE
:10D5F800122200210020FFF7DBFD00BF204B93F82B
:10D608004130DBB2212BF9D00A2001F0C3F8FFF733
:10D6180025FF7B685B78092B0FD17B685A68194B0B
:10D628001068516803C3127A1A70174B1B78DBB263
:10D63800012B0FD01223FB7305E01323FB7302E0C9
:10D648001323FB7300BFFB7B1A4600210020FFF762
:10D65800AFFD00E000BF1037BD4680BD6C11002053
:10D66800C411002078000020D4110020147D010886
:10D6780004090020287D0108B00300203C7D010832
:10D68800FC1200206C0000206011002080B500AF63
:10D698008F4B9A788F4B9A708D4BD3F807308D4A01
:10D6A800C2F803308A4BB3F80F309AB2894BA3F80B
:10D6B8000720874BB3F81B309AB2864BA3F8092092
:10D6C800834BB3F813309AB2824BA3F80B20804BEC
:10D6D800B3F815309AB27F4BA3F80D207C4B1A7E15
:10D6E8007C4BDA737A4B5A7F7A4B5A70784B5A785C
:10D6F800784B1A70774B00221A7400225A74754BB3
:10D7080000229A74734B0022DA7400221A750420DE
:10D71800FCF7BEF8034603F00103D9B26D4A537D06
:10D7280061F3000353750320FCF7B2F8034603F0D6
:10D738000103D9B2674A537D61F341035375002051
:10D74800FCF7A6F8034603F00103D9B2614A537DFA
:10D7580061F3820353755F4A537D23F008035375C1
:10D768000320FCF7A5F80346002B0CBF0123002378
:10D77800D9B2584A537D61F304135375FCF77AFE06
:10D788000346002B14BF01230023D9B2514A537D0D
:10D7980061F3451353754F4A537D23F04003537586
:10D7A8004D4B1B7A03F00103D9B24A4A537D61F30A
:10D7B800C71353750020FCF7A1F903465AB2454B2D
:10D7C8005A760120FCF79AF903465AB2414B9A76E9
:10D7D800414B1B6A5AB23F4BDA763E4B00221A770E
:10D7E8003C4B00225A773B4B00229A770022DA778B
:10D7F800384B002283F82020384B9B689AB2354B6F
:10D80800A3F82120354BDB689AB2324BA3F82320CA
:10D81800324B1B699AB22F4BA3F825201122002105
:10D828002F4807F067FC2B4B002283F83820294B40
:10D83800002283F83920002283F83A20254B002261
:10D8480083F83B20002283F83C200422002125484D
:10D8580007F050FC1F4B002283F84120002283F878
:10D868004220002283F84320002283F84420194BE9
:10D87800002283F84720174B002283F84620154BD7
:10D88800002283F84520134B002283F84820002209
:10D8980083F849200F4B002283F84A2008220021F0
:10D8A800114807F027FC0B4B002283F85320094B43
:10D8B800002283F85420002283F85520054B0022CB
:10D8C80083F85620002283F8572000BF80BD00BF90
:10D8D800B00300206C11002004090020D8080020A3
:10D8E80093110020A9110020B711002080B485B041
:10D8F80000AF78607B68002B18D07B6800221A6024
:10D908007B6800229A807B680022DA800023FB81F2
:10D9180008E0FA897B680232002143F82210FB896B
:10D928000133FB81FB89072BF3D900E000BF1437D3
:10D93800BD4680BC704780B485B000AF7860396060
:10D948007B68002B01D13B6856E07B68DB88072B9E
:10D9580027D87B689B881A467B680232396843F867
:10D9680022107B681A683B681A447B681A607B68D7
:10D978009B8801339AB27B689A807B689B88072BC7
:10D9880002D97B6800229A807B68DB8801339AB2CF
:10D998007B68DA807B681B687A68D28893FBF2F32D
:10D9A8002AE07B689B881A467B68023253F822304B
:10D9B800FB607B689B881A467B680232396843F8AB
:10D9C80022107B681A683968FB68CB1A1A447B688E
:10D9D8001A607B689B8801339AB27B689A807B685F
:10D9E8009B88072B02D97B6800229A807B681B687A
:10D9F800002B00DA0733DB1018461437BD4680BC0D
:10DA08007047000080B485B000AF154B9B69144A7D
:10DA180043F001039361124B9B6903F00103BB6060
:10DA2800BB680F4BDB690E4A43F08053D3610C4B44
:10DA3800DB6903F080537B607B680A4B5B68FB60A3
:10DA4800FB6823F0E063FB60FB6843F00073FB6056
:10DA5800044AFB68536000BF1437BD4680BC70475A
:10DA68000010024000000140FEE700BFFEE700BFD3
:10DA7800FEE700BFFEE700BFFEE700BF704700BF3C
:10DA8800704700BF704700BF00F068BE10B5094C72
:10DA980001224FF40061204603F009FA064802F01B
:10DAA800F7FD2046BDE8104000224FF4006103F066
:10DAB800FEB900BF000C0140C0020020014802F07E
:10DAC800E7BD00BF58140020014802F0E1BD00BFC7
:10DAD80014140020014802F0DBBD00BF8C130020A5
:10DAE800014802F0D5BD00BFD013002010B5094C85
:10DAF80001224FF40061204603F0D9F9064801F0ED
:10DB080023F82046BDE8104000224FF4006103F0DE
:10DB1800CEB900BF000C01409002002010B5094C9E
:10DB280001224FF48061204603F0C1F9064802F053
:10DB380047F82046BDE8104000224FF4806103F00A
:10DB4800B6B900BF000C01405C03002010B5094CB9
:10DB580001224FF40061204603F0A9F9064804F0B9
:10DB680087FD2046BDE8104000224FF4006103F015
:10DB78009EB900BF000C0140DC110020014805F0EF
:10DB88002DBE00BFB412002010B5084C0122202180
:10DB9800204603F08CF9064805F020FE2046BDE833
:10DBA80010400022202103F082B900BF0008014084
:10DBB800FC12002010B5084C01224021204603F039
:10DBC80076F9064805F00AFE2046BDE81040002216
:10DBD800402103F06CB900BF000801404413002045
:10DBE80010B5084C01220421204603F060F90648CC
:10DBF80005F0F4FD2046BDE810400022042103F0A2
:10DC080056B900BF001001406C12002010B5094C35
:10DC180001224FF48061204603F049F9064801F0DB
:10DC2800CFFF2046BDE8104000224FF4806103F08A
:10DC38003EB900BF000C01408403002010B5094C18
:10DC480001224FF48061204603F031F9064801F0C3
:10DC5800B7FF2046BDE8104000224FF4806103F072
:10DC680026B900BF000C01408403002080B400AF37
:10DC780001231846BD4680BC704780B582B000AF0E
:10DC88007860396007F03EFA034616221A604FF0B2
:10DC9800FF3318460837BD4680BD80B582B000AF57
:10DCA80078604FF0FF317868FFF7E7FF00BFFDE7C6
:10DCB80080B586B000AFF860B9607A6000237B61F8
:10DCC8000AE0AFF300800146BB685A1CBA60CAB2CA
:10DCD8001A707B6901337B617A697B689A42F0DB51
:10DCE8007B6818461837BD4680BD80B483B000AF46
:10DCF80078604FF0FF3318460C37BD4680BC70473C
:10DD080080B483B000AF786039603B684FF400524C
:10DD18005A60002318460C37BD4680BC704780B453
:10DD280083B000AF7860012318460C37BD4680BC2D
:10DD3800704780B485B000AFF860B9607A6000239E
:10DD480018461437BD4680BC7047000080B586B0C1
:10DD580000AF7860144A154BD31A7B617B693B612D
:10DD6800134B1B68002B02D1114B124A1A60104B3F
:10DD78001A687B6813443A699A4207D207F0C2F9D5
:10DD880003460C221A604FF0FF3309E0084B1B686A
:10DD9800FB60074B1A687B681344054A1360FB68ED
:10DDA80018461837BD4680BD000001200004000059
:10DDB800D8110020F015002080B400AF00BFBD4688
:10DDC80080BC704780B58EB000AF07F128030022F1
:10DDD8001A605A609A60DA6007F1200300221A601C
:10DDE8005A603B1D00221A605A609A60DA601A6114
:10DDF8005A619A61384B394A1A60374B00225A6087
:10DE0800354B00229A60344B4FF6FF72DA60324B82
:10DE180000221A61304B00229A612F4804F0D5F98C
:10DE28000346002B01D0FCF751FF4FF48053BB622F
:10DE380007F128031946284804F028FE0346002B5A
:10DE480001D0FCF743FF244804F00EFA0346002BE8
:10DE580001D0FCF73BFF204804F008FB0346002BE9
:10DE680001D0FCF733FF30233B6200237B6207F1CC
:10DE780020031946184805F0B7F90346002B01D0CE
:10DE8800FCF724FF00237B600123BB600023FB60B9
:10DE980000237B613B1D002219460F4804F0D8FC83
:10DEA8000346002B01D0FCF711FF60237B600023A1
:10DEB800BB603B1D04221946074804F025FD0346B4
:10DEC800002B01D0FCF702FF034800F0CFF800BF99
:10DED8003837BD4680BD00BFDC110020000400407B
:10DEE80080B58EB000AF07F1280300221A605A608F
:10DEF8009A60DA6007F1200300221A605A603B1D1D
:10DF080000221A605A609A60DA601A615A619A614E
:10DF1800374B384A1A60364B4FF434725A60344BD8
:10DF280000229A60324B6422DA60314B00221A6177
:10DF38002F4B00229A612E4804F047F90346002B24
:10DF480001D0FCF7C3FE4FF48053BB6207F12803EE
:10DF58001946274804F09AFD0346002B01D0FCF728
:10DF6800B5FE234804F082FA0346002B01D0FCF7E3
:10DF7800ADFE00233B6200237B6207F120031946B4
:10DF88001B4805F031F90346002B01D0FCF79EFE33
:10DF980060237B600023BB600023FB6000237B6160
:10DFA8003B1D04221946124804F0AEFC0346002B20
:10DFB80001D0FCF78BFE3B1D082219460C4804F0E3
:10DFC800A3FC0346002B01D0FCF780FE3B1D0C226E
:10DFD8001946074804F098FC0346002B01D0FCF7CB
:10DFE80075FE034800F042F800BF3837BD4680BDD3
:10DFF800241200200008004080B584B000AF78608B
:10E008007B681B68164A934214D1164BDB69154A84
:10E0180043F00203D361134BDB6903F00203FB6097
:10E02800FB68002206211D2002F0C5F81D2002F021
:10E03800DEF810E07B681B680B4A93420BD1094B52
:10E04800DB69084A43F00403D361064BDB6903F03C
:10E058000403BB60BB6800BF1037BD4680BD00BF6E
:10E0680000040040001002400008004080B58AB05B
:10E0780000AF786007F1140300221A605A609A60B2
:10E08800DA607B681B68264A934218D1254B9B6946
:10E09800244A43F004039361224B9B6903F0040371
:10E0A8003B613B6980237B610223BB6102233B62A6
:10E0B80007F1140319461C4802F05EFD2BE07B684B
:10E0C8001B681A4A934226D1164B9B69154A43F09E
:10E0D80020039361134B9B6903F02003FB60FB68EB
:10E0E8004FF460437B610223BB6102233B6207F16B
:10E0F800140319460E4802F03FFD0E4B5B687B6225
:10E108007B6A43F0E0637B627B6A43F480537B6203
:10E11800084A7B6A536000BF2837BD4680BD00BFF0
:10E1280000040040001002400008014000080040C0
:10E13800001401400000014080B500AF114B124AA5
:10E148001A60104B4FF416525A600E4B00229A6018
:10E158000C4B0022DA600B4B00221A61094B0C228F
:10E168005A61084B00229A61064B0022DA61054881
:10E1780005F0B2F80346002B01D0FCF7A7FD00BF5D
:10E1880080BD00BF6C1200200050004080B500AF79
:10E19800114B124A1A60104B4FF4E1325A600E4B81
:10E1A80000229A600C4B0022DA600B4B00221A61A5
:10E1B800094B0C225A61084B00229A61064B002237
:10E1C800DA61054805F088F80346002B01D0FCF712
:10E1D8007DFD00BF80BD00BFB412002000380140A3
:10E1E80080B500AF114B124A1A60104B4FF4E13260
:10E1F8005A600E4B00229A600C4B0022DA600B4BDF
:10E2080000221A61094B0C225A61084B00229A61BC
:10E21800064B0022DA61054805F05EF80346002B3C
:10E2280001D0FCF753FD00BF80BD00BFFC120020E9
:10E238000044004080B500AF114B124A1A60104BE1
:10E248004FF4E1325A600E4B00229A600C4B0022C8
:10E25800DA600B4B00221A61094B0C225A61084BF9
:10E2680000229A61064B0022DA61054805F034F86D
:10E278000346002B01D0FCF729FD00BF80BD00BF7D
:10E28800441300200048004080B592B000AF786089
:10E2980007F1300300221A605A609A60DA607B68DE
:10E2A8001B68924A934245D1914BDB69904A43F4EB
:10E2B8008013D3618E4BDB6903F48013FB62FB6A26
:10E2C8008B4B9B698A4A43F010039361884B9B6987
:10E2D80003F01003BB62BB6A854B9B69844A43F019
:10E2E80020039361824B9B6903F020037B627B6A66
:10E2F8004FF480533B6302237B630323FB6307F1E3
:10E30800300319467B4802F037FC04233B630023A3
:10E318007B630023BB6307F130031946764802F09C
:10E328002BFC00220521352001F045FF352001F0A6
:10E338005EFF93E17B681B68704A93423AD16C4B4D
:10E348009B696B4A43F480439361694B9B6903F46F
:10E3580080433B623B6A664B9B69654A43F0040312
:10E368009361634B9B6903F00403FB61FB694FF402
:10E3780000733B6302237B630323FB6307F13003D2
:10E3880019465F4802F0F8FB4FF480633B630023B3
:10E398007B630023BB6307F130031946584802F03A
:10E3A800EBFB00220521252001F005FF252001F0C7
:10E3B8001EFF53E17B681B68524A934240F0AE80CF
:10E3C8004B4BDB694A4A43F40033D361484BDB6962
:10E3D80003F40033BB61BB69454B9B69444A43F076
:10E3E80020039361424B9B6903F020037B617B69A7
:10E3F80020233B6302237B630323FB6307F1300382
:10E4080019463D4802F0B8FB40233B6300237B6379
:10E418000023BB6307F130031946374802F0ACFB11
:10E42800394B5B683B643B6C43F0E0633B643B6C9B
:10E4380043F008033B64344A3B6C5360334B344A23
:10E448001A60324B00225A60304B00229A602F4BE0
:10E458008022DA602D4B00221A612C4B00225A616F
:10E468002A4B00229A61294B4FF44052DA6127481F
:10E4780001F0F4FE0346002B01D0FCF727FC7B6873
:10E48800224ADA63214A7B685362224B224A1A6085
:10E49800204B10225A601F4B00229A601D4B80228D
:10E4A800DA601C4B00221A611A4B00225A61194B80
:10E4B80000229A61174B4FF40052DA61154801F0B7
:10E4C800CDFE0346002B01D0FCF700FC7B68114A07
:10E4D8009A63104A7B68536200220221262001F0C9
:10E4E8006AFE262001F083FEB8E000BF005000401D
:10E4F80000100240001001400014014000380140A3
:10E508000008014000440040000001408C13002036
:10E518006C000240D0130020800002407B681B681A
:10E52800504A934240F09A804F4BDB694E4A43F47D
:10E538008023D3614C4BDB6903F480233B613B6947
:10E54800494B9B69484A43F010039361464B9B69CA
:10E5580003F01003FB60FB684FF480633B63022306
:10E568007B630323FB6307F1300319463F4802F03E
:10E5780003FB4FF400633B6300237B630023BB630F
:10E5880007F130031946394802F0F6FA384B5B6850
:10E598007B647B6C23F030037B647B6C43F0E0632B
:10E5A8007B647B6C43F010037B64314A7B6C536063
:10E5B800304B314A1A602F4B00225A602D4B0022F3
:10E5C8009A602C4B8022DA602A4B00221A61294B70
:10E5D80000225A61274B00229A61264B4FF4405281
:10E5E800DA61244801F03AFE0346002B01D0FCF71B
:10E5F8006DFB7B681F4ADA631E4A7B6853621F4BB8
:10E608001F4A1A601D4B10225A601C4B00229A6048
:10E618001A4B8022DA60194B00221A61174B00222C
:10E628005A61164B00229A61144B4FF40052DA617A
:10E63800124801F013FE0346002B01D0FCF746FBFD
:10E648007B680E4A9A630D4A7B6853620022022156
:10E65800272001F0B0FD272001F0C9FD00BF483791
:10E66800BD4680BD00480040001002400010014037
:10E67800000001401414002030000240581400200B
:10E688001C000240FFF798FB0B480C490C4A00237A
:10E6980002E0D458C4500433C4188C42F9D3094A50
:10E6A800094C002301E013600432A242FBD306F0B8
:10E6B8002FFDFCF721FA70470000002058020020C7
:10E6C8004481010858020020EC150020FEE70000F4
:10E6D80080B500AF084B1B68074A43F0100313606E
:10E6E800032001F05DFD0F2000F008F8FFF78AF91C
:10E6F8000023184680BD00BF0020024080B582B0CC
:10E7080000AF7860124B1A68124B1B7819464FF409
:10E718007A73B3FBF1F3B2FBF3F3184601F075FD1E
:10E728000346002B01D001230EE07B680F2B0AD88B
:10E73800002279684FF0FF3001F03DFD064A7B6802
:10E748001360002300E0012318460837BD4680BD4A
:10E75800840000208C0000208800002080B400AFD6
:10E76800054B1B781A46054B1B681344034A136074
:10E7780000BFBD4680BC70478C0000209C14002060
:10E7880080B400AF024B1B681846BD4680BC70477A
:10E798009C14002080B584B000AF7860FFF7F0FFCC
:10E7A800B8607B68FB60FB68B3F1FF3F05D00A4B9C
:10E7B8001B781A46FB681344FB6000BFFFF7E0FFB5
:10E7C8000246BB68D31AFA689A42F7D800BF00BF5E
:10E7D8001037BD4680BD00BF8C00002080B586B0D4
:10E7E80000AF78600023FB7500233B610023BB600A
:10E7F8000023FB607B68002B01D10123BEE07B680E
:10E808009B68002B7B689B6A002B09D17B680022E0
:10E81800DA627B68002283F824207868FAF73EFFE2
:10E82800786800F0BDFB0346FB757B689B6A03F0C4
:10E838001003002B40F09980FB7D002B40F0958061
:10E848007B689B6A23F4885323F0020343F0020297
:10E858007B689A627B685A687B68DB691A437B68C5
:10E868001B7B5B001343BA681343BB607B689B68E0
:10E87800B3F5807F03D07B689B68012B02D14FF4EE
:10E88800807300E000233A6913433B617B681B7D7A
:10E89800012B19D17B681B7B002B09D17B689B69F5
:10E8A800013B5A033B69134343F400633B610BE0AC
:10E8B8007B689B6A43F020027B689A627B68DB6A0C
:10E8C80043F001027B68DA627B681B685B6823F4AB
:10E8D80069417B681B683A690A435A607B681B6810
:10E8E8009A68284B13407A681268B9680B4393609A
:10E8F8007B689B68B3F5807F03D07B689B68012B9E
:10E9080004D17B681B69013B1B05FB607B681B68A6
:10E91800DB6A23F470017B681B68FA680A43DA62D1
:10E928007B681B689A68184B1340BA689A420BD1E7
:10E938007B680022DA627B689B6A23F0030343F05A
:10E9480001027B689A6218E07B689B6A23F01203D5
:10E9580043F010027B689A627B68DB6A43F001022D
:10E968007B68DA620123FB7507E07B689B6A43F0EA
:10E9780010027B689A620123FB75FB7D18461837E5
:10E98800BD4680BDFDF7E1FFFE0E1FFF80B586B0D6
:10E9980000AFF860B9607A600023FB75FB681B68FC
:10E9A800644A934204D0FB681B68634A934206D1C9
:10E9B800604B5B6803F47023002B40F0B380FB6866
:10E9C80093F82430012B01D10223AEE0FB68012229
:10E9D80083F82420F86800F089FA0346FB75FB7D6C
:10E9E800002B40F09A80FB689B6A23F4706323F045
:10E9F800010343F48072FB689A62FB681B684E4A05
:10EA0800934205D14B4B5B6803F47023002B15D15F
:10EA1800FB689B6A23F48012FB689A62FB681B6898
:10EA28005B6803F48063002B26D0FB689B6A23F4A1
:10EA3800405343F48052FB689A621DE0FB689B6A6E
:10EA480043F48012FB689A62FB681B68394A934258
:10EA580004D0FB681B68384A93420DD1354B5B687C
:10EA680003F48063002B07D0FB689B6A23F44053B0
:10EA780043F48052FB689A62FB689B6A03F48053F4
:10EA8800002B06D0FB68DB6A23F00602FB68DA621B
:10EA980002E0FB680022DA62FB68002283F8242087
:10EAA800FB681B6A254A9A62FB681B6A244ADA6279
:10EAB800FB681B6A234A1A63FB681B686FF0020233
:10EAC8001A60FB681B689A68FB681B6842F48072CE
:10EAD8009A60FB68186AFB681B684C331946BA6869
:10EAE8007B6801F031FCFB681B689B6803F46023BA
:10EAF800B3F5602F08D1FB681B689A68FB681B6830
:10EB080042F4A0029A600FE0FB681B689A68FB68F1
:10EB18001B6842F480129A6006E0FB68002283F8C2
:10EB2800242001E00123FB75FB7D18461837BD46FC
:10EB380080BD00BF00240140002801402BF00008E0
:10EB4800A7F00008C3F0000880B584B000AF786073
:10EB58007B681B681B68FB607B681B685B68BB6025
:10EB6800BB6803F02003002B3ED0FB6803F00203D0
:10EB7800002B39D07B689B6A03F01003002B05D16A
:10EB88007B689B6A43F400727B689A627B681B68A7
:10EB98009B6803F46023B3F5602F1DD17B681B7B52
:10EBA800002B19D17B681B685A687B681B6822F0A8
:10EBB80020025A607B689B6A23F480727B689A62A1
:10EBC8007B689B6A03F48053002B05D17B689B6AA2
:10EBD80043F001027B689A627868FAF7B3FC7B68B5
:10EBE8001B686FF012021A60BB6803F08003002BE9
:10EBF8004DD0FB6803F00403002B48D07B689B6A68
:10EC080003F01003002B05D17B689B6A43F4005284
:10EC18007B689A627B681B689B6803F4E043B3F5E2
:10EC2800E04F12D07B681B685B6803F48063002B9D
:10EC380025D17B681B689B6803F46023B3F5602FBC
:10EC48001DD17B681B7B002B19D17B681B685A6818
:10EC58007B681B6822F080025A607B689B6A23F4F9
:10EC680080527B689A627B689B6A03F48073002BEE
:10EC780005D17B689B6A43F001027B689A627868D9
:10EC880000F0E4FA7B681B686FF00C021A60BB683E
:10EC980003F04003002B12D0FB6803F00103002BA4
:10ECA8000DD07B689B6A43F480327B689A627868EF
:10ECB80000F012F87B681B686FF001021A6000BF51
:10ECC8001037BD4680BD80B483B000AF786000BF08
:10ECD8000C37BD4680BC704780B483B000AF786005
:10ECE80000BF0C37BD4680BC704780B483B000AF0E
:10ECF800786000BF0C37BD4680BC704780B485B0D3
:10ED080000AF786039600023FB730023BB607B6829
:10ED180093F82430012B01D10223DCE07B68012227
:10ED280083F824203B685B68062B1CD87B681B682B
:10ED3800596B3B685A6813469B001344053B1F22D6
:10ED480002FA03F3DB4319403B6818683B685A68CA
:10ED580013469B001344053B00FA03F27B681B68CB
:10ED68000A435A633CE03B685B680C2B1CD87B6801
:10ED78001B68196B3B685A6813469B001344233B76
:10ED88001F2202FA03F3DB4319403B6818683B680B
:10ED98005A6813469B001344233B00FA03F27B682E
:10EDA8001B680A431A631BE07B681B68D96A3B68C7
:10EDB8005A6813469B001344413B1F2202FA03F38F
:10EDC800DB4319403B6818683B685A6813469B0048
:10EDD8001344413B00FA03F27B681B680A43DA627A
:10EDE8003B681B68092B1CD97B681B68D9683B6882
:10EDF8001A6813465B0013441E3B072202FA03F30A
:10EE0800DB4319403B6898683B681A6813465B0007
:10EE180013441E3B00FA03F27B681B680A43DA605E
:10EE280019E07B681B6819693B681A6813465B0020
:10EE38001344072202FA03F3DB4319403B6898683E
:10EE48003B681A6813465B00134400FA03F27B68B8
:10EE58001B680A431A613B681B68102B03D03B6888
:10EE68001B68112B32D17B681B681D4A934225D140
:10EE78007B681B689B6803F40003002B26D17B6822
:10EE88001B689A687B681B6842F400029A603B68BA
:10EE98001B68102B1AD1134B1B68134AA2FB0323C0
:10EEA8009A0C13469B0013445B00BB6002E0BB68EE
:10EEB800013BBB60BB68002BF9D107E07B689B6A0C
:10EEC80043F020027B689A620123FB737B6800226F
:10EED80083F82420FB7B18461437BD4680BC704756
:10EEE800002401408400002083DE1B4380B584B0E9
:10EEF80000AF78600023FB600023BB607B681B6861
:10EF08009B6803F00103012B40D07B681B689A685B
:10EF18007B681B6842F001029A601F4B1B681F4AFE
:10EF2800A2FB03239B0CBB6002E0BB68013BBB60F8
:10EF3800BB68002BF9D1FFF723FCF8601FE0FFF74F
:10EF48001FFC0246FB68D31A022B18D97B681B6882
:10EF58009B6803F00103012B11D07B689B6A43F087
:10EF680010027B689A627B68DB6A43F001027B6867
:10EF7800DA627B68002283F82420012307E07B689B
:10EF88001B689B6803F00103012BD8D100231846A6
:10EF98001037BD4680BD00BF8400002083DE1B43C0
:10EFA80080B584B000AF78600023FB607B681B6885
:10EFB8009B6803F00103012B2ED17B681B689A68BC
:10EFC8007B681B6822F001029A60FFF7D9FBF860A2
:10EFD8001BE0FFF7D5FB0246FB68D31A022B14D9B6
:10EFE8007B681B689B6803F00103012B0DD17B68CC
:10EFF8009B6A43F010027B689A627B68DB6A43F085
:10F0080001027B68DA62012307E07B681B689B6862
:10F0180003F00103012BDCD0002318461037BD464E
:10F0280080BD80B584B000AF78607B685B6AFB60A8
:10F03800FB689B6A03F05003002B27D1FB689B6A8F
:10F0480043F40072FB689A62FB681B689B6803F4D0
:10F058006023B3F5602F15D1FB681B7B002B11D102
:10F06800FB689B6A23F48072FB689A62FB689B6A60
:10F0780003F48053002B05D1FB689B6A43F001021F
:10F08800FB689A62F868FAF75DFA04E0FB681B6AA5
:10F098001B6B7868984700BF1037BD4680BD80B5A8
:10F0A80084B000AF78607B685B6AFB60F868FFF744
:10F0B8000AFE00BF1037BD4680BD80B584B000AFE2
:10F0C80078607B685B6AFB60FB689B6A43F0400280
:10F0D800FB689A62FB68DB6A43F00402FB68DA6249
:10F0E800F868FFF702FE00BF1037BD4680BD00007C
:10F0F80090B587B000AF78600023FB750023FB60F4
:10F108007B6893F82430012B01D1022397E07B68B8
:10F11800012283F824207868FFF742FF0346FB7535
:10F128007868FFF7E3FE0346FB75FB7D002B40F094
:10F1380081807B689B6A23F4885323F0020343F0A1
:10F1480002027B689A62404B1C68022002F0E2FDD2
:10F158000346B4FBF3F35B00FB6002E0FB68013B92
:10F16800FB60FB68002BF9D17B681B689A687B6899
:10F178001B6842F008029A60FFF702FB38611BE047
:10F18800FFF7FEFA02463B69D31A0A2B14D97B68AB
:10F198001B689B6803F00803002B0DD07B689B6AF3
:10F1A80023F0120343F010027B689A627B68002206
:10F1B80083F82420012342E07B681B689B6803F0E6
:10F1C8000803002BDCD17B681B689A687B681B6886
:10F1D80042F004029A60FFF7D3FA38611BE0FFF7A8
:10F1E800CFFA02463B69D31A0A2B14D97B681B68ED
:10F1F8009B6803F00403002B0DD07B689B6A23F007
:10F20800120343F010027B689A627B68002283F83D
:10F218002420012313E07B681B689B6803F0040328
:10F22800002BDCD17B689B6A23F0030343F00102C7
:10F238007B689A627B68002283F82420FB7D18464D
:10F248001C37BD4690BD00BF8400002080B483B049
:10F2580000AF786000BF0C37BD4680BC704780B5F2
:10F2680084B000AF78607B68002B01D10123EDE00A
:10F278007B6893F82030DBB2002B02D17868FAF76C
:10F28800F7FC7B681B681A687B681B6842F0010200
:10F298001A60FFF775FAF86012E0FFF771FA024694
:10F2A800FB68D31A0A2B0BD97B685B6A43F40032DC
:10F2B8007B685A627B68052283F820200123C5E019
:10F2C8007B681B685B6803F00103002BE5D07B6853
:10F2D8001B681A687B681B6822F002021A60FFF735
:10F2E8004FFAF86012E0FFF74BFA0246FB68D31AB0
:10F2F8000A2B0BD97B685B6A43F400327B685A623D
:10F308007B68052283F8202001239FE07B681B6827
:10F318005B6803F00203002BE5D17B681B7E012BA1
:10F3280008D17B681B681A687B681B6842F08002FA
:10F338001A6007E07B681B681A687B681B6822F004
:10F3480080021A607B685B7E012B08D17B681B6892
:10F358001A687B681B6842F040021A6007E07B6805
:10F368001B681A687B681B6822F040021A607B6879
:10F378009B7E012B08D17B681B681A687B681B6819
:10F3880042F020021A6007E07B681B681A687B68F5
:10F398001B6822F020021A607B68DB7E012B08D1F3
:10F3A8007B681B681A687B681B6822F010021A6069
:10F3B80007E07B681B681A687B681B6842F01002CC
:10F3C8001A607B681B7F012B08D17B681B681A6851
:10F3D8007B681B6842F008021A6007E07B681B68BC
:10F3E8001A687B681B6822F008021A607B685B7FDA
:10F3F800012B08D17B681B681A687B681B6842F080
:10F4080004021A6007E07B681B681A687B681B683F
:10F4180022F004021A607B689A687B68DB681A43EA
:10F428007B681B691A437B685B6942EA03017B6856
:10F438005B685A1E7B681B680A43DA617B68002296
:10F448005A627B68012283F820200023184610376F
:10F45800BD4680BD80B487B000AF786039607B68F6
:10F468001B687B617B6893F82030FB74FB7C012B65
:10F4780003D0FB7C022B40F0BE80654B7B617B692F
:10F48800D3F8003243F001027B69C3F800227B699C
:10F49800D3F8003223F47C527B69C3F800227B69DD
:10F4A800D3F800223B685B6A1B021A437B69C3F8E6
:10F4B80000223B685B6903F01F03012202FA03F391
:10F4C800FB607B69D3F81C22FB68DB431A407B692D
:10F4D800C3F81C223B68DB69002B23D17B69D3F876
:10F4E8000C22FB68DB431A407B69C3F80C223B689B
:10F4F800DB6819043B685B689BB23A685269194338
:10F508007B69483243F832103B689B6819043B68B2
:10F518001B689AB23B685B690A4379694833DB0028
:10F528000B445A603B68DB69012B22D17B69D3F815
:10F538000C22FB681A437B69C3F80C223B681B68E2
:10F5480019043B685B689BB23A68526919437B6946
:10F55800483243F832103B689B6819043B68DB6803
:10F568009AB23B685B690A4379694833DB000B440C
:10F578005A603B689B69002B09D17B69D3F8042248
:10F58800FB68DB431A407B69C3F8042207E07B6908
:10F59800D3F80422FB681A437B69C3F804223B684A
:10F5A8001B69002B09D17B69D3F81422FB68DB4364
:10F5B8001A407B69C3F8142207E07B69D3F8142248
:10F5C800FB681A437B69C3F814223B681B6A012B4A
:10F5D80007D17B69D3F81C22FB681A437B69C3F8FF
:10F5E8001C227B69D3F8003223F001027B69C3F83F
:10F5F8000022002306E07B685B6A43F480227B6874
:10F608005A62012318461C37BD4680BC704700BFAC
:10F618000064004080B584B000AF78607B6893F8E0
:10F628002030DBB2012B2ED17B68022283F8202008
:10F638007B681B681A687B681B6822F001021A60E5
:10F64800FFF79EF8F86012E0FFF79AF80246FB68A9
:10F65800D31A0A2B0BD97B685B6A43F400327B68A8
:10F668005A627B68052283F82020012312E07B6818
:10F678001B685B6803F00103002BE5D17B6800225F
:10F688005A62002306E07B685B6A43F400227B68C9
:10F698005A62012318461037BD4680BD80B584B034
:10F6A80000AF78607B6893F82030DBB2022B33D14F
:10F6B8007B681B681A687B681B6842F001021A6045
:10F6C800FFF75EF8F86012E0FFF75AF80246FB68A9
:10F6D800D31A0A2B0BD97B685B6A43F400327B6828
:10F6E8005A627B68052283F8202001231BE07B688F
:10F6F8001B685B6803F00103002BE5D07B681B687F
:10F708001A687B681B6822F002021A607B68012273
:10F7180083F82020002306E07B685B6A43F48012AC
:10F728007B685A62012318461037BD4680BD80B4F5
:10F7380089B000AFF860B9607A603B60FB6893F805
:10F748002030FB77FB681B689B68BB61FB7F012B44
:10F7580003D0FB7F022B40F0AD80BB6903F08063D0
:10F76800002B0AD1BB6903F00063002B05D1BB69EC
:10F7780003F08053002B00F09580BB691B0E03F04B
:10F7880003037B6101227B699A403B681A60BB686E
:10F798009B68002B0DD1BB681B685A05BB68DB68EA
:10F7A800F96809681A437B6918331B010B441A600E
:10F7B8000FE0BB685B68DA00BB689B681A43BB68EC
:10F7C800DB68F96809681A437B6918331B010B4425
:10F7D8001A60FB681968BB681A697B6918331B01D2
:10F7E8000B4404331A60BB681B7D012B11D1FB68E5
:10F7F8001A687B6918331B01134404331B68FA68C1
:10F80800116843F480727B6918331B010B4404337D
:10F818001A607B6807331B781A067B6806331B78E7
:10F828001B041A437B6805331B781B0213437A6851
:10F83800043212781046FA68116843EA00027B69BC
:10F848001B010B4403F5C6731A607B6803331B78EE
:10F858001A067B6802331B781B041A437B68013342
:10F868001B781B0213437A6812781046FA681168ED
:10F8780043EA00027B691B010B4403F5C4731A6059
:10F88800FB681A687B6918331B0113441B68FA6804
:10F89800116843F001027B6918331B010B441A609D
:10F8A80000230EE0FB685B6A43F40012FB685A62AF
:10F8B800012306E0FB685B6A43F48022FB685A6216
:10F8C800012318462437BD4680BC704780B485B0F4
:10F8D80000AF78600023FB607B6893F82030FB72F0
:10F8E800FB7A012B02D0FB7A022B1DD17B681B68A7
:10F8F8009B6803F08063002B02D0FB680133FB6038
:10F908007B681B689B6803F00063002B02D0FB68D0
:10F918000133FB607B681B689B6803F08053002BF6
:10F9280002D0FB680133FB60FB6818461437BD46FC
:10F9380080BC704780B487B000AFF860B9607A6067
:10F948003B60FB6893F82030FB75FB7D012B03D0EF
:10F95800FB7D022B40F00381BB68002B0ED1FB68B6
:10F968001B68DB6803F00303002B16D1FB685B6A96
:10F9780043F40012FB685A620123F7E0FB681B6836
:10F988001B6903F00303002B07D1FB685B6A43F490
:10F998000012FB685A620123E8E0FB681A68BB683A
:10F9A8001B331B0113441B6803F004027B689A6035
:10F9B8007B689B68002B0CD1FB681A68BB681B33FB
:10F9C8001B0113441B685B0DC3F30A027B681A60B2
:10F9D8000BE0FB681A68BB681B331B0113441B68E8
:10F9E800DB0823F060427B685A60FB681A68BB68D2
:10F9F8001B331B0113441B6803F002027B68DA60A7
:10FA0800FB681A68BB681B331B01134404331B686B
:10FA180003F00803002B03D07B6808221A610BE06F
:10FA2800FB681A68BB681B331B01134404331B684B
:10FA380003F00F027B681A61FB681A68BB681B3306
:10FA48001B01134404331B681B0ADAB27B689A61F2
:10FA5800FB681A68BB681B331B01134404331B681B
:10FA68001B0C9AB27B685A61FB681A68BB681B0159
:10FA7800134403F5DC731B68DAB23B681A70FB6841
:10FA88001A68BB681B01134403F5DC731B681A0A68
:10FA98003B680133D2B21A70FB681A68BB681B0155
:10FAA800134403F5DC731B681A0C3B680233D2B2AB
:10FAB8001A70FB681A68BB681B01134403F5DC73F2
:10FAC8001B681A0E3B680333D2B21A70FB681A68B7
:10FAD800BB681B01134403F5DE731A683B680433E3
:10FAE800D2B21A70FB681A68BB681B01134403F58D
:10FAF800DE731B681A0A3B680533D2B21A70FB68BA
:10FB08001A68BB681B01134403F5DE731B681A0CE3
:10FB18003B680633D2B21A70FB681A68BB681B01CF
:10FB2800134403F5DE731B681A0E3B680733D2B221
:10FB38001A70BB68002B08D1FB681B68DA68FB6881
:10FB48001B6842F02002DA6007E0FB681B681A694C
:10FB5800FB681B6842F020021A61002306E0FB687C
:10FB68005B6A43F48022FB685A62012318461C37FB
:10FB7800BD4680BC704780B485B000AF78603960FE
:10FB88007B6893F82030FB73FB7B012B02D0FB7B57
:10FB9800022B09D17B681B6859697B681B683A6826
:10FBA8000A435A61002306E07B685B6A43F48022BB
:10FBB8007B685A62012318461437BD4680BC7047DB
:10FBC80080B58AB000AF786000237B627B681B68D1
:10FBD8005B693B627B681B685B68FB617B681B68D1
:10FBE8009B68BB617B681B68DB687B617B681B6803
:10FBF8001B693B617B681B689B69FB603B6A03F080
:10FC08000103002B7CD0BB6903F00103002B23D038
:10FC18007B681B6801229A60BB6903F00203002B12
:10FC280003D0786800F083F916E0BB6903F0040399
:10FC3800002B04D07B6A43F400637B620CE0BB6951
:10FC480003F00803002B04D07B6A43F480537B62E3
:10FC580002E0786800F086F9BB6903F48073002B32
:10FC680024D07B681B684FF480729A60BB6903F4E8
:10FC78000073002B03D0786800F062F916E0BB69C6
:10FC880003F48063002B04D07B6A43F400537B6247
:10FC98000CE0BB6903F40063002B04D07B6A43F4D7
:10FCA80080437B6202E0786800F065F9BB6903F481
:10FCB8008033002B24D07B681B684FF480329A6015
:10FCC800BB6903F40033002B03D0786800F041F9D6
:10FCD80016E0BB6903F48023002B04D07B6A43F44D
:10FCE80000437B620CE0BB6903F40023002B04D0C3
:10FCF8007B6A43F480337B6202E0786800F044F961
:10FD08003B6A03F00803002B0CD07B6903F0100357
:10FD1800002B07D07B6A43F400737B627B681B6807
:10FD28001022DA603B6A03F00403002B0BD07B69D6
:10FD380003F00803002B06D07B681B680822DA60F2
:10FD4800786800F033F93B6A03F00203002B09D00E
:10FD58007B681B68DB6803F00303002B02D078681C
:10FD680000F01BF93B6A03F04003002B0CD03B6901
:10FD780003F01003002B07D07B6A43F480637B6297
:10FD88007B681B6810221A613B6A03F02003002B72
:10FD98000BD03B6903F00803002B06D07B681B6877
:10FDA80008221A61786800F00AF93B6A03F0100328
:10FDB800002B09D07B681B681B6903F00303002B29
:10FDC80002D07868FBF70EF83B6A03F40033002B87
:10FDD8000BD0FB6903F01003002B06D07B681B686F
:10FDE80010225A60786800F0F3F83B6A03F4803315
:10FDF800002B0BD0FB6903F00803002B06D07B68AF
:10FE08001B6808225A60786800F0EBF83B6A03F434
:10FE18000043002B7BD0FB6903F00403002B72D056
:10FE28003B6A03F48073002B08D0FB6803F00103DE
:10FE3800002B03D07B6A43F001037B623B6A03F427
:10FE48000073002B08D0FB6803F00203002B03D0DB
:10FE58007B6A43F002037B623B6A03F48063002BF6
:10FE680008D0FB6803F00403002B03D07B6A43F03F
:10FE780004037B623B6A03F40063002B43D0FB68F6
:10FE880003F07003002B3ED0FB6803F07003602B77
:10FE98002BD0602B2ED8502B22D0502B2AD8402B79
:10FEA80019D0402B26D8302B10D0302B22D8102B2D
:10FEB80002D0202B05D01DE07B6A43F008037B624B
:10FEC80019E07B6A43F010037B6214E07B6A43F01D
:10FED80020037B620FE07B6A43F040037B620AE009
:10FEE8007B6A43F080037B6205E07B6A43F480739E
:10FEF8007B6200E000BF7B681B689A697B681B68AF
:10FF080022F070029A617B681B6804225A607B6A3F
:10FF1800002B08D07B685A6A7B6A1A437B685A624E
:10FF2800786800F067F800BF2837BD4680BD80B408
:10FF380083B000AF786000BF0C37BD4680BC704707
:10FF480080B483B000AF786000BF0C37BD4680BC7A
:10FF5800704780B483B000AF786000BF0C37BD46EF
:10FF680080BC704780B483B000AF786000BF0C37A6
:10FF7800BD4680BC704780B483B000AF786000BFD6
:10FF88000C37BD4680BC704780B483B000AF786042
:10FF980000BF0C37BD4680BC704780B483B000AF4B
:10FFA800786000BF0C37BD4680BC704780B483B012
:10FFB80000AF786000BF0C37BD4680BC704780B486
:10FFC80083B000AF786000BF0C37BD4680BC704777
:10FFD80080B483B000AF786000BF0C37BD4680BCEA
:10FFE800704780B483B000AF786000BF0C37BD465F
:08FFF80080BC704780B483B0A7
:020000040801F1
:1000000000AF786000BF0C37BD4680BC7047000071
:1000100080B485B000AF78607B6803F00703FB60B5
:100020000C4BDB68BB60BA684FF6FF031340BB6044
:10003000FB681A02BB68134343F0BF6343F4003309
:10004000BB60044ABB68D36000BF1437BD4680BCA8
:10005000704700BF00ED00E080B400AF044BDB68E8
:100060001B0A03F007031846BD4680BC704700BF5B
:1000700000ED00E080B483B000AF0346FB7197F958
:100080000730002B0BDBFB7903F01F02064997F9C1
:1000900007305B09012000FA02F241F8232000BF7B
:1000A0000C37BD4680BC704700E100E080B483B0EF
:1000B00000AF03463960FB7197F90730002B0ADB6C
:1000C0003B68DAB20C4997F907301201D2B20B44FF
:1000D00083F800230AE03B68DAB20849FB7903F0B1
:1000E0000F03043B1201D2B20B441A7600BF0C3747
:1000F000BD4680BC704700BF00E100E000ED00E0BD
:1001000080B489B000AFF860B9607A60FB6803F032
:100110000703FB61FB69C3F10703042B28BF04231A
:10012000BB61FB690433062B02D9FB69033B00E08A
:1001300000237B614FF0FF32BB6902FA03F3DA431D
:10014000BB681A407B699A404FF0FF317B6901FA26
:1001500003F3D9437B680B40134318462437BD464D
:1001600080BC704780B582B000AF78607B68013B8F
:10017000B3F1807F01D301230FE00A4A7B68013B82
:1001800053600F214FF0FF30FFF790FF054B002227
:100190009A60044B07221A60002318460837BD46B0
:1001A00080BD00BF10E000E080B582B000AF786095
:1001B0007868FFF72DFF00BF0837BD4680BD80B5CA
:1001C00086B000AF0346B9607A60FB7300237B61A1
:1001D000FFF742FF78617A68B9687869FFF790FFA6
:1001E000024697F90F3011461846FFF75FFF00BF30
:1001F0001837BD4680BD80B582B000AF0346FB71A5
:1002000097F907301846FFF735FF00BF0837BD469E
:1002100080BD80B582B000AF78607868FFF7A2FF3C
:10022000034618460837BD4680BD80B582B000AF92
:1002300078607B68002B01D101230EE07B685B793D
:10024000DBB2002B05D17B6800221A717868FAF7BF
:1002500087F87B6801225A71002318460837BD468B
:1002600080BD000080B485B000AF78600023FB60E3
:100270007B68002B01D1012359E07B681B681A467B
:100280002D4B9A420FD87B681B681A462B4B1344A0
:100290002B4AA2FB03231B099A007B681A647B6824
:1002A000284ADA630EE07B681B681A46264B134423
:1002B000234AA2FB03231B099A007B681A647B680C
:1002C000224ADA637B68022283F821207B681B685C
:1002D0001B68FB60FB6823F47F5323F03003FB6053
:1002E0007B685A687B689B681A437B68DB681A43A3
:1002F0007B681B691A437B685B691A437B689B694F
:100300001A437B68DB691343FA681343FB607B681D
:100310001B68FA681A607B6800229A637B68012276
:1003200083F821207B68002283F8202000231846D0
:100330001437BD4680BC704707040240F8FFFDBF7C
:10034000CDCCCCCC00000240F8FBFDBF0004024045
:1003500080B586B000AFF860B9607A603B6000237A
:10036000FB75FB6893F82030012B01D102234BE091
:10037000FB68012283F82020FB6893F82130DBB270
:10038000012B3AD1FB68022283F82120FB6800226E
:100390009A63FB681B681A68FB681B6822F00102FD
:1003A0001A603B687A68B968F86800F0BCFBFB68C3
:1003B000DB6A002B08D0FB681B681A68FB681B68A7
:1003C00042F00E021A600FE0FB681B681A68FB68B7
:1003D0001B6822F004021A60FB681B681A68FB683D
:1003E0001B6842F00A021A60FB681B681A68FB6807
:1003F0001B6842F001021A6005E0FB68002283F8E6
:1004000020200223FB75FB7D18461837BD4680BDB2
:1004100080B485B000AF78600023FB737B6893F8ED
:100420002130DBB2022B08D07B6804229A637B6800
:10043000002283F82020012320E07B681B681A68D3
:100440007B681B6822F00E021A607B681B681A68C2
:100450007B681B6822F001021A607B681A6C7B685B
:10046000DB6B012101FA02F25A607B68012283F8FA
:1004700021207B68002283F82020FB7B184614375C
:10048000BD4680BC7047000080B584B000AF786086
:100490000023FB737B6893F82130DBB2022B05D07D
:1004A0007B6804229A630123FB73D6E07B681B6898
:1004B0001A687B681B6822F00E021A607B681B6852
:1004C0001A687B681B6822F001021A607B681B684F
:1004D0001A46644B9A4258D97B681B68624A934219
:1004E0004FD07B681B68614A934248D07B681B6889
:1004F0005F4A934240D07B681B685E4A934238D083
:100500007B681B685C4A934230D07B681B685B4AFF
:10051000934228D07B681B68524A934220D07B6864
:100520001B68574A934219D07B681B68554A93420F
:1005300012D07B681B68544A93420AD07B681B68C0
:10054000524A934202D14FF480531BE04FF4803360
:1005500018E04FF4807315E0102313E0012311E03D
:100560004FF080730EE04FF480130BE04FF48033B4
:1005700008E04FF4805305E04FF4807302E010234D
:1005800000E00123424A536057E07B681B68364A0B
:1005900093424FD07B681B68344A934248D07B68B3
:1005A0001B68334A934240D07B681B68314A9342B0
:1005B00038D07B681B68304A934230D07B681B6818
:1005C0002E4A934228D07B681B68264A934220D04B
:1005D0007B681B682A4A934219D07B681B68294AAA
:1005E000934212D07B681B68274A93420AD07B68EB
:1005F0001B68264A934202D14FF480531BE04FF40C
:10060000803318E04FF4807315E0102313E00123CA
:1006100011E04FF080730EE04FF480130BE04FF4C5
:10062000803308E04FF4805305E04FF4807302E01C
:10063000102300E00123174A53607B68012283F8EE
:1006400021207B68002283F820207B685B6B002BD5
:1006500003D07B685B6B78689847FB7B1846103744
:10066000BD4680BD80000240080002401C000240E0
:100670003000024044000240580002406C0002403A
:10068000080402401C0402403004024044040240BA
:10069000000402400000024080B584B000AF7860E2
:1006A0007B68DB6B1B68FB607B681B681B68BB603F
:1006B0007B681B6C04229A40FB681340002B00F0FF
:1006C000F180BB6803F00403002B00F0EB807B6833
:1006D0001B681B6803F02003002B07D17B681B6895
:1006E0001A687B681B6822F004021A607B681B682A
:1006F0001A465F4B9A4258D97B681B685D4A934201
:100700004FD07B681B685C4A934248D07B681B686B
:100710005A4A934240D07B681B68594A934238D06A
:100720007B681B68574A934230D07B681B68564AE7
:10073000934228D07B681B684D4A934220D07B6847
:100740001B68524A934219D07B681B68504A9342F7
:1007500012D07B681B684F4A93420AD07B681B68A3
:100760004D4A934202D14FF480431BE04FF4802363
:1007700018E04FF4806315E0402313E0042311E0F8
:100780004FF080630EE04FF480030BE04FF48023C2
:1007900008E04FF4804305E04FF4806302E040231B
:1007A00000E004233D4A536057E07B681B68314AF0
:1007B00093424FD07B681B682F4A934248D07B6896
:1007C0001B682E4A934240D07B681B682C4A934298
:1007D00038D07B681B682B4A934230D07B681B68FB
:1007E000294A934228D07B681B68214A934220D033
:1007F0007B681B68254A934219D07B681B68244A92
:10080000934212D07B681B68224A93420AD07B68CD
:100810001B68214A934202D14FF480431BE04FF4FE
:10082000802318E04FF4806315E0402313E0042395
:1008300011E04FF080630EE04FF480030BE04FF4C3
:10084000802308E04FF4804305E04FF4806302E02A
:10085000402300E00423124A53607B68DB6A002BCC
:1008600000F036817B68DB6A7868984730E100BF2A
:1008700080000240080002401C000240300002409C
:1008800044000240580002406C000240080402404C
:100890001C040240300402404404024000040240B0
:1008A000000002407B681B6C02229A40FB681340E8
:1008B000002B00F0DD80BB6803F00203002B00F08A
:1008C000D7807B681B681B6803F02003002B0BD1CB
:1008D0007B681B681A687B681B6822F00A021A6032
:1008E0007B68012283F821207B681B681A467B4BBA
:1008F0009A4258D97B681B68794A93424FD07B68EB
:100900001B68784A934248D07B681B68764A9342BA
:1009100040D07B681B68754A934238D07B681B685F
:10092000734A934230D07B681B68724A934228D046
:100930007B681B68694A934220D07B681B686E4ABB
:10094000934219D07B681B686C4A934212D07B6833
:100950001B686B4A93420AD07B681B68694A9342C2
:1009600002D14FF400531BE04FF4003318E04FF472
:10097000007315E0202313E0022311E04FF0007311
:100980000EE04FF400130BE04FF4003308E04FF497
:10099000005305E04FF4007302E0202300E002233F
:1009A000594A536057E07B681B684D4A93424FD0C9
:1009B0007B681B684B4A934248D07B681B684A4A55
:1009C000934240D07B681B68484A934238D07B688A
:1009D0001B68474A934230D07B681B68454A934264
:1009E00028D07B681B683D4A934220D07B681B68F7
:1009F000414A934219D07B681B68404A934212D007
:100A00007B681B683E4A93420AD07B681B683D4A5C
:100A1000934202D14FF400531BE04FF4003318E02F
:100A20004FF4007315E0202313E0022311E04FF090
:100A300000730EE04FF400130BE04FF4003308E0B6
:100A40004FF4005305E04FF4007302E0202300E070
:100A500002232E4A53607B68002283F820207B68A3
:100A60009B6A002B34D07B689B6A786898472FE09C
:100A70007B681B6C08229A40FB681340002B28D02F
:100A8000BB6803F00803002B23D07B681B681A683F
:100A90007B681B6822F00E021A607B681A6C7B6808
:100AA000DB6B012101FA02F25A607B6801229A6332
:100AB0007B68012283F821207B68002283F82020B4
:100AC0007B681B6B002B04D07B681B6B7868984796
:100AD00000BF00BF1037BD4680BD00BF8000024090
:100AE000080002401C000240300002404400024066
:100AF000580002406C000240080402401C040240FE
:100B0000300402404404024000040240000002405D
:100B100080B483B000AF78607B689B6B18460C375D
:100B2000BD4680BC704780B485B000AFF860B96046
:100B30007A603B60FB681A6CFB68DB6B012101FA91
:100B400002F25A60FB681B683A685A60FB685B688F
:100B5000102B08D1FB681B687A689A60FB681B68D9
:100B6000BA68DA6007E0FB681B68BA689A60FB68DD
:100B70001B687A68DA6000BF1437BD4680BC7047D6
:100B800080B48BB000AF7860396000237B620023B3
:100B90003B6269E101227B6A02FA03F3FB613B6875
:100BA0001B68FA691340BB61BA69FB699A4240F05D
:100BB00058813B685B689A4A93425ED0984A934258
:100BC00075D8984A934258D0964A93426FD8964A1D
:100BD000934252D0944A934269D8944A93424CD05B
:100BE000924A934263D8924A934246D0904A9342A3
:100BF0005DD8122B2AD8122B59D801A252F823F013
:100C00007B0C0108550C0108670C0108A90C0108B0
:100C1000AF0C0108AF0C0108AF0C0108AF0C0108C4
:100C2000AF0C0108AF0C0108AF0C0108AF0C0108B4
:100C3000AF0C0108AF0C0108AF0C0108AF0C0108A4
:100C4000AF0C01085D0C0108710C0108794A934250
:100C500013D02CE03B68DB683B6229E03B68DB6833
:100C600004333B6224E03B68DB6808333B621FE0EF
:100C70003B68DB680C333B621AE03B689B68002BE7
:100C800002D104233B6213E03B689B68012B05D132
:100C900008233B627B68FA691A6109E008233B621A
:100CA0007B68FA695A6103E000233B6200E000BF01
:100CB000BB69FF2B01D87B6801E07B6804337B6153
:100CC000BB69FF2B02D87B6A9B0002E07B6A083B72
:100CD0009B003B617B691A680F213B6901FA03F3B2
:100CE000DB431A40396A3B6901FA03F31A437B6913
:100CF0001A603B685B6803F08053002B00F0B18002
:100D00004D4B9B694C4A43F0010393614A4B9B69ED
:100D100003F00103BB60BB68484A7B6A9B0802334F
:100D200052F82330FB607B6A03F003039B000F2221
:100D300002FA03F3DB43FA681340FB607B68404A26
:100D4000934213D07B683F4A93420DD07B683E4A62
:100D5000934207D07B683D4A934201D1032306E0CA
:100D6000042304E0022302E0012300E000237A6A66
:100D700002F0030292009340FA681343FB602F498C
:100D80007B6A9B080233FA6841F823203B685B6862
:100D900003F48013002B06D02D4B9A682C49BB69B5
:100DA00013438B6006E02A4B9A68BB69DB432849F2
:100DB00013408B603B685B6803F40013002B06D084
:100DC000234BDA682249BB691343CB6006E0204B12
:100DD000DA68BB69DB431E491340CB603B685B6844
:100DE00003F40033002B06D0194B5A681849BB692D
:100DF00013434B6006E0164B5A68BB69DB4314494A
:100E000013404B603B685B6803F48033002B21D0B8
:100E10000F4B1A680E49BB6913430B6021E000BFFA
:100E200000003210000031100000221000002110DC
:100E300000001210000011100010024000000140DC
:100E400000080140000C0140001001400014014066
:100E5000000401400B4B1A68BB69DB43094913408E
:100E60000B607B6A01337B623B681A687B6A22FAFB
:100E700003F3002B7FF48EAE00BF00BF2C37BD46BE
:100E800080BC70470004014080B485B000AF78603A
:100E90000B467B807B689A687B881340002B02D0CE
:100EA0000123FB7301E00023FB73FB7B184614371F
:100EB000BD4680BC704780B483B000AF78600B46FD
:100EC0007B8013467B707B78002B03D07A887B680D
:100ED0001A6103E07B881A047B681A6100BF0C3733
:100EE000BD4680BC7047000080B400AF034B0122B8
:100EF0001A6000BFBD4680BC704700BF20000E4294
:100F000080B582B000AFFDF73FFC7860604B1B6896
:100F10005F4A43F00103136008E0FDF735FC024629
:100F20007B68D31A022B01D90323ACE0584B1B6812
:100F300003F00203002BF0D0554B1B6823F0F8039D
:100F4000534A43F080031360FDF71EFC7860504B5A
:100F500000225A600AE0FDF717FC02467B68D31AAC
:100F600041F28832934201D903238CE0484B5B68FD
:100F700003F00C03002BEED1464B474A1A60474B57
:100F80001B681846FDF7BEFB0346002B01D001236A
:100F900079E0FDF7F9FB78603D4B1B683C4A23F094
:100FA0008073136008E0FDF7EFFB02467B68D31AFD
:100FB000022B01D9032366E0354B1B6803F0007355
:100FC000002BF0D1324B00225A60FDF7DDFB786038
:100FD0002F4B1B682E4A23F41023136008E0FDF703
:100FE000D3FB02467B68D31A642B01D903234AE062
:100FF000274B1B6803F40033002BF0D1244B1B68F4
:10100000234A23F480231360FDF7BEFB7860204B56
:101010001B681F4A23F08063136008E0FDF7B4FBF0
:1010200002467B68D31A642B01D903232BE0184BAB
:101030001B6803F00063002BF0D1FDF7A5FB78607F
:10104000134B1B68124A23F08053136008E0FDF72E
:101050009BFB02467B68D31A642B01D9032312E061
:101060000B4B1B6803F00053002BF0D1084B002200
:10107000DA62074B5B6A064A43F080735362044BA3
:1010800000229A60002318460837BD4680BD00BF85
:10109000001002408400002000127A008800002026
:1010A00080B586B000AF78607B68002B01D101234A
:1010B00004E37B681B6803F00103002B00F08780CA
:1010C000924B5B6803F00C03042B0CD08F4B5B68D6
:1010D00003F00C03082B12D18C4B5B6803F48033B4
:1010E000B3F5803F0BD1894B1B6803F40033002B11
:1010F0006CD07B689B68002B68D10123DEE27B68A3
:101100009B68B3F5803F06D1804B1B687F4A43F450
:10111000803313602EE07B689B68002B0CD17B4BE7
:101120001B687A4A23F480331360784B1B68774A34
:1011300023F4802313601DE07B689B68B3F5A02F28
:101140000CD1724B1B68714A43F4802313606F4BC0
:101150001B686E4A43F4803313600BE06B4B1B68D3
:101160006A4A23F480331360684B1B68674A23F490
:10117000802313607B689B68002B13D0FDF704FB72
:10118000386108E0FDF700FB02463B69D31A642B87
:1011900001D9032392E25D4B1B6803F40033002B5B
:1011A000F0D014E0FDF7F0FA386108E0FDF7ECFA52
:1011B00002463B69D31A642B01D903237EE2534BC9
:1011C0001B6803F40033002BF0D100E000BF7B6804
:1011D0001B6803F00203002B63D04C4B5B6803F0E9
:1011E0000C03002B0BD0494B5B6803F00C03082B5E
:1011F0001CD1464B5B6803F48033002B16D1434B64
:101200001B6803F00203002B05D07B685B69012B90
:1012100001D0012352E23D4B1B6823F0F8027B68AA
:101220009B69DB00394913430B603AE07B685B69DB
:10123000002B20D0364B01221A60FDF7A5FA386149
:1012400008E0FDF7A1FA02463B69D31A022B01D947
:10125000032333E22D4B1B6803F00203002BF0D075
:101260002A4B1B6823F0F8027B689B69DB00274947
:1012700013430B6015E0264B00221A60FDF784FA39
:10128000386108E0FDF780FA02463B69D31A022B69
:1012900001D9032312E21D4B1B6803F00203002B4C
:1012A000F0D17B681B6803F00803002B3AD07B6801
:1012B000DB69002B19D0174B01221A60FDF764FA85
:1012C000386108E0FDF760FA02463B69D31A022B49
:1012D00001D90323F2E10D4B5B6A03F00203002BFB
:1012E000F0D0012000F0CAFB1CE00A4B00221A607B
:1012F000FDF74AFA38610FE0FDF746FA02463B690E
:10130000D31A022B08D90323D8E100BF00100240F2
:1013100000004242800442429B4B5B6A03F002039E
:10132000002BE9D17B681B6803F00403002B00F05D
:10133000A6800023FB75944BDB6903F08053002BE0
:101340000DD1914BDB69904A43F08053D3618E4BB2
:10135000DB6903F08053BB60BB680123FB758B4BDB
:101360001B6803F48073002B18D1884B1B68874AD5
:1013700043F480731360FDF707FA386108E0FDF766
:1013800003FA02463B69D31A642B01D9032395E182
:101390007E4B1B6803F48073002BF0D07B681B69C5
:1013A000012B06D1784B1B6A774A43F00103136285
:1013B0002DE07B681B69002B0CD1734B1B6A724AB2
:1013C00023F001031362704B1B6A6F4A23F004037E
:1013D00013621CE07B681B69052B0CD16A4B1B6AEE
:1013E000694A43F004031362674B1B6A664A43F081
:1013F000010313620BE0644B1B6A634A23F0010391
:101400001362614B1B6A604A23F0040313627B681A
:101410001B69002B15D0FDF7B7F938610AE0FDF71D
:10142000B3F902463B69D31A41F28832934201D99B
:10143000032343E1544B1B6A03F00203002BEED05D
:1014400014E0FDF7A1F938610AE0FDF79DF90246C5
:101450003B69D31A41F28832934201D903232DE12B
:10146000494B1B6A03F00203002BEED1FB7D012BDD
:1014700005D1454BDB69444A23F08053D3617B6837
:10148000DB6A002B00F08C803F4B5B6803F48033F9
:10149000B3F5803F0ED13C4B5B6803F00C03082B87
:1014A00008D1394BDB6A03F48033B3F5803F01D1B7
:1014B000012303E17B68DB6A022B4ED1324B1B68B0
:1014C00003F08053002B09D02F4BDB6A03F0F002AE
:1014D0007B685B6B9A4201D00123EFE02C4B00222A
:1014E0001A60FDF751F9386108E0FDF74DF9024641
:1014F0003B69D31A642B01D90323DFE0224B1B681D
:1015000003F00063002BF0D11F4BDB6A23F0F002E5
:101510007B685B6B1C491343CB621B4BDB6A23F478
:1015200070627B681B6B18491343CB62184B012216
:101530001A60FDF729F9386108E0FDF725F9024640
:101540003B69D31A642B01D90323B7E00E4B1B6808
:1015500003F00063002BF0D022E00B4BDB6A0A4A59
:1015600023F48033D3620A4B00221A60FDF70CF992
:1015700038610FE0FDF708F902463B69D31A642B86
:1015800008D903239AE000BF001002400070004019
:10159000680042424B4B1B6803F00063002BE9D10B
:1015A0007B681B6A002B00F08880464B5B6803F069
:1015B0000C03082B68D07B681B6A022B4DD1424B71
:1015C00000221A60FDF7E0F8386108E0FDF7DCF86A
:1015D00002463B69D31A022B01D903236EE0394B33
:1015E0001B6803F00073002BF0D17B685B6AB3F5D6
:1015F000803F0FD1334BDA6A7B685B683149134314
:10160000CB62304BDB6A23F00F027B68DB682D492D
:101610001343CB622B4B5B6823F474127B68596ACB
:101620007B689B6A0B43274913434B60264B01227F
:101630001A60FDF7A9F8386108E0FDF7A5F8024641
:101640003B69D31A022B01D9032337E01D4B1B68DA
:1016500003F00073002BF0D02FE01B4B00221A6028
:10166000FDF792F8386108E0FDF78EF802463B6915
:10167000D31A022B01D9032320E0124B1B6803F07D
:101680000073002BF0D118E07B681B6A012B01D19D
:10169000012313E00B4B5B68FB60FB6803F48032B3
:1016A0007B685B6A9A4206D1FB6803F470127B6820
:1016B0009B6A9A4201D0012300E0002318461837A4
:1016C000BD4680BD001002406000424280B584B03B
:1016D00000AF786039607B68002B01D10123D0E036
:1016E0006A4B1B6803F007033A689A4210D9674BAC
:1016F0001B6823F0070265493B6813430B60634B8B
:101700001B6803F007033A689A4201D00123B8E04E
:101710007B681B6803F00203002B20D07B681B68EA
:1017200003F00403002B05D0594B5B68584A43F47F
:10173000E06353607B681B6803F00803002B05D04F
:10174000534B5B68524A43F460535360504B5B68A1
:1017500023F0F0027B689B684D4913434B607B6824
:101760001B6803F00103002B40D07B685B68012BF2
:1017700007D1474B1B6803F40033002B15D101231D
:101780007FE07B685B68022B07D1414B1B6803F04D
:101790000073002B09D1012373E03D4B1B6803F05C
:1017A0000203002B01D101236BE0394B5B6823F06E
:1017B00003027B685B68364913434B60FCF7E4FF28
:1017C000F8600AE0FCF7E0FF0246FB68D31A41F23A
:1017D0008832934201D9032353E02D4B5B6803F019
:1017E0000C027B685B689B009A42EBD1274B1B681D
:1017F00003F007033A689A4210D2244B1B6823F087
:10180000070222493B6813430B60204B1B6803F01F
:1018100007033A689A4201D0012332E07B681B68D3
:1018200003F00403002B08D0194B5B6823F4E0623B
:101830007B68DB68164913434B607B681B6803F0C9
:101840000803002B09D0124B5B6823F460527B68BD
:101850001B69DB000E4913434B6000F021F8024680
:101860000B4B5B681B0903F00F030A49CB5C22FAA0
:1018700003F3094A1360094B1B681846FCF742FF43
:10188000002318461037BD4680BD00BF002002402F
:1018900000100240647D01088400002088000020C0
:1018A0002DE9B04F8EB000AF0023FB620023BB6276
:1018B00000237B6300237B6200233B6300233B62A6
:1018C0000023FB614E4B5B68FB62FB6A03F00C0379
:1018D000042B02D0082B03D089E04A4B3B6389E0FC
:1018E000FB6A9B0C03F00F02474B9B5C7B62FB6A1D
:1018F00003F48033002B72D0414BDB6A03F00F02FC
:10190000424B9B5CBB623E4BDB6A03F48033002B93
:1019100053D03B4BDB6A1B0903F00F0301333B62DF
:10192000374BDB6A1B0A03F00F030233FB61FB69D1
:1019300000229A4693467B6A00223B617A613B69AA
:1019400003FB0BF27B690AFB03F313443A69AAFB1E
:1019500002010B4419462B4B03FB01F2002300FB51
:1019600003F31344274AA0FB02452B441D463B6A60
:101970000022BB60FA60BB6A00223B607A60D7E954
:1019800002010B46D7E900AB524602FB03F25B466D
:1019900084460CFB03F3134402465146A2FB018923
:1019A0004B44994642464B4620462946F7F722FCCF
:1019B00002460B4613467B6307E07B6A114A03FB32
:1019C00002F2BB6AB2FBF3F37B630F4B5B7B1A46FD
:1019D0007B6A934208D17B6B5B087B6304E07B6A84
:1019E0000B4A02FB03F37B637B6B3B6302E0094B17
:1019F0003B6300BF3B6B18463837BD46BDE8B08F30
:101A00000010024040787D017C7D01088C7D01083A
:101A100000093D0000127A0080B400AF024B1B6841
:101A20001846BD4680BC70478400002080B500AFDA
:101A3000FFF7F2FF0246054B5B681B0A03F0070342
:101A40000349CB5C22FA03F3184680BD0010024024
:101A5000747D010880B500AFFFF7DEFF0246054B3D
:101A60005B68DB0A03F007030349CB5C22FA03F34C
:101A7000184680BD00100240747D010880B485B016
:101A800000AF78600A4B1B680A4AA2FB03235B0A7B
:101A90007A6802FB03F3FB6000BFFB685A1EFA6022
:101AA000002BF9D100BF00BF1437BD4680BC704782
:101AB00084000020D34D621080B588B000AF7860FC
:101AC00000237B6100233B610023FB617B681B6873
:101AD00003F00103002B7DD00023FB768B4BDB69E9
:101AE00003F08053002B0DD1884BDB69874A43F00C
:101AF0008053D361854BDB6903F08053FB60FB6847
:101B00000123FB76824B1B6803F48073002B18D1F2
:101B10007F4B1B687E4A43F480731360FCF734FEEE
:101B2000786108E0FCF730FE02467B69D31A642B2B
:101B300001D90323E5E0764B1B6803F48073002B87
:101B4000F0D0724B1B6A03F440733B613B69002B7E
:101B50002ED07B685B6803F440733A699A4227D0C1
:101B60006A4B1B6A23F440733B616A4B01221A6083
:101B7000684B00221A60654A3B6913623B6903F0B7
:101B80000103002B14D0FCF7FFFD78610AE0FCF79D
:101B9000FBFD02467B69D31A41F28832934201D998
:101BA0000323AEE0594B1B6A03F00203002BEED077
:101BB000564B1B6A23F440727B685B68534913439E
:101BC0000B62FB7E012B05D1504BDB694F4A23F0A2
:101BD0008053D3617B681B6803F00203002B08D09D
:101BE0004A4B5B6823F440427B689B684749134338
:101BF0004B607B681B6803F00403002B08D0434B49
:101C0000DB6A23F400327B68DB6840491343CB6214
:101C10007B681B6803F00803002B08D03B4BDB6A92
:101C200023F480227B681B6938491343CB62374B0E
:101C3000DB6A03F40033002B05D1344BDB6A03F479
:101C40008023002B01D00123FB61FB69012B48D1CC
:101C50002E4B1B6803F08053002B38D12B4B1B6895
:101C600003F08063002B09D0284BDB6A03F0F002FD
:101C70007B689B699A4201D0012342E0234BDB6AD7
:101C800023F0F0027B689B6920491343CB621F4B12
:101C9000DB6A23F470427B685B691C491343CB62A7
:101CA0001D4B01221A60FCF76FFD786108E0FCF71C
:101CB0006BFD02467B69D31A642B01D9032320E014
:101CC000124B1B6803F00053002BF0D009E00F4BC0
:101CD000DB6A03F470427B685B699A4201D001239E
:101CE0000FE07B681B6803F01003002B08D0074B44
:101CF0005B6823F480027B68DB69044913434B6013
:101D0000002318462037BD4680BD00BF00100240AA
:101D100000700040400442427000424280B58AB0E8
:101D200000AF78600023FB6100237B620023BB616E
:101D300000237B6100233B610023FB600023BB6029
:101D400000233B627B68013B0F2B00F21D8101A247
:101D500052F823F0091F01086D1F0108891F0108AF
:101D6000671E0108891F0108891F0108891F0108D2
:101D7000B91E0108891F0108891F0108891F010870
:101D8000891F0108891F0108891F0108891F01088F
:101D9000951D0108834B5B68BB60824B1B6803F099
:101DA0008073002B00F0F280BB689B0C03F00F03E4
:101DB0007D4AD35CBB61BB6803F48033002B3BD00E
:101DC000784BDB6A03F00F03784AD35CFB61754BF9
:101DD000DB6A03F48033002B1CD0724BDB6A1B09D7
:101DE00003F00F030133FB606E4BDB6A1B0A03F049
:101DF0000F0302337B616E4AFB68B2FBF3F37A692F
:101E000003FB02F2FB69B2FBF3F2BB6902FB03F3D3
:101E10007B6207E0664AFB69B2FBF3F2BB6902FB37
:101E200003F37B62604B5B7B1A46BB69934208D12C
:101E30007B6A5B087B6204E0BB695E4A02FB03F3DA
:101E40007B62584B5B6803F48003B3F5800F02D1CB
:101E50007B6A3B629AE07B6A5B00574AA2FB0323E2
:101E60005B083B6292E04F4BDB6A03F40033002BCC
:101E700003D1FFF715FD38628AE04A4B1B6803F077
:101E80008053002B00F08480464BDB6A1B0903F073
:101E90000F030133FB60434BDB6A1B0B03F00F03A3
:101EA00002333B61424AFB68B2FBF3F33A6902FB3F
:101EB00003F35B003B626BE03A4BDB6A03F4802385
:101EC000002B03D1FFF7ECFC386263E0354B1B6855
:101ED00003F08053002B5DD0324BDB6A1B0903F00B
:101EE0000F030133FB602F4BDB6A1B0B03F00F0367
:101EF00002333B612E4AFB68B2FBF3F33A6902FB03
:101F000003F35B003B6245E0264B1B6ABB60BB688A
:101F100003F44073B3F5807F08D1BB6803F002037C
:101F2000002B03D04FF400433B621EE0BB6803F478
:101F30004073B3F5007F09D11A4B5B6A03F00203CB
:101F4000002B03D049F640433B620EE0BB6803F42C
:101F50004073B3F5407F1FD1124B1B6803F400336D
:101F6000002B19D0154B3B6216E015E0FFF772FD10
:101F700002460C4B5B689B0B03F0030301335B00D1
:101F8000B2FBF3F33B6208E000BF06E000BF04E0F1
:101F900000BF02E000BF00E000BF3B6A18462837E0
:101FA000BD4680BD001002409C7D0108AC7D01084B
:101FB00040787D0100093D00ABAAAAAAF0FA020010
:101FC00080B584B000AF78600023FB607B68002B95
:101FD00001D101237AE07B685B7CDBB2002B05D169
:101FE0007B6800221A747868F9F7B6FF7B680222D2
:101FF0005A74786800F070F80346002B04D07B68B0
:1020000004225A74012361E0786800F092F80346D4
:10201000002B04D07B6804225A74012356E07B68AD
:102020001B685A687B681B6822F007025A607B684D
:102030009B68002B05D0274B1B6B264A23F001031E
:102040001363244BDB6A23F460727B689B6821492D
:102050001343CB627B685B68B3F1FF3F03D07B68BF
:102060005B68FB600EE00120FFF758FEF860FB683C
:10207000002B04D17B6804225A74012326E0FB68FC
:10208000013BFB60FB681A0C7B681B6802F00F02C7
:102090009A607B681B68FA6892B2DA60786800F030
:1020A00070F80346002B04D07B6804225A74012385
:1020B0000CE07B680022DA737B6801225A737B682C
:1020C00001229A737B6801225A7400231846103744
:1020D000BD4680BD006C004080B584B000AF786024
:1020E0000023FB607B68002B01D101231DE07B688E
:1020F0001B685A687B681B6822F008025A60FCF76C
:1021000043FBF86009E0FCF73FFB0246FB68D31A8B
:10211000B3F57A7F01D9032307E07B681B685B680E
:1021200003F00803002BEED0002318461037BD46FD
:1021300080BD80B584B000AF78600023FB60FCF701
:1021400023FBF86009E0FCF71FFB0246FB68D31A8B
:10215000B3F57A7F01D903230FE07B681B685B68C6
:1021600003F02003002BEED07B681B685A687B6865
:102170001B6842F010025A60002318461037BD4613
:1021800080BD80B584B000AF78600023FB607B68C1
:102190001B685A687B681B6822F010025A60FCF7C3
:1021A000F3FAF86009E0FCF7EFFA0246FB68D31A8D
:1021B000B3F57A7F01D9032307E07B681B685B686E
:1021C00003F02003002BEED0002318461037BD4645
:1021D00080BD80B582B000AF78607B68002B01D1F4
:1021E000012341E07B6893F83D30DBB2002B06D140
:1021F0007B68002283F83C207868FBF701FF7B684E
:10220000022283F83D207B681A687B6804331946F4
:10221000104600F033FD7B68012283F846207B687E
:10222000012283F83E207B68012283F83F207B68EF
:10223000012283F840207B68012283F841207B68DB
:10224000012283F842207B68012283F843207B68C7
:10225000012283F844207B68012283F845207B68B3
:10226000012283F83D20002318460837BD4680BD73
:1022700080B582B000AF78607B68002B01D101236C
:1022800041E07B6893F83D30DBB2002B06D17B68E0
:10229000002283F83C20786800F039F87B6802223D
:1022A00083F83D207B681A687B6804331946104622
:1022B00000F0E4FC7B68012283F846207B68012261
:1022C00083F83E207B68012283F83F207B6801224F
:1022D00083F840207B68012283F841207B6801223B
:1022E00083F842207B68012283F843207B68012227
:1022F00083F844207B68012283F845207B68012213
:1023000083F83D20002318460837BD4680BD80B4C1
:1023100083B000AF786000BF0C37BD4680BC70470B
:1023200080B584B000AF786039603B68002B09D17C
:102330007B6893F83E30DBB2012B14BF01230023EE
:10234000DBB222E03B68042B09D17B6893F83F3075
:10235000DBB2012B14BF01230023DBB215E03B6885
:10236000082B09D17B6893F84030DBB2012B14BFF6
:1023700001230023DBB208E07B6893F84130DBB235
:10238000012B14BF01230023DBB2002B01D001235A
:1023900063E03B68002B04D17B68022283F83E2077
:1023A00013E03B68042B04D17B68022283F83F20B2
:1023B0000BE03B68082B04D17B68022283F84020A5
:1023C00003E07B68022283F841207B681B680122BE
:1023D0003968184600F0E8FE7B681B68214A934282
:1023E00007D17B681B685A6C7B681B6842F400420B
:1023F0005A647B681B681B4A934213D07B681B6836
:10240000B3F1804F0ED07B681B68174A934209D006
:102410007B681B68154A934204D07B681B68144A8A
:10242000934211D17B681B689B6803F00703FB6034
:10243000FB68062B10D07B681B681A687B681B68DA
:1024400042F001021A6007E07B681B681A687B682B
:102450001B6842F001021A60002318461037BD467F
:1024600080BD00BF002C0140000400400008004077
:10247000000C004080B582B000AF78607B68002B14
:1024800001D1012341E07B6893F83D30DBB2002BA2
:1024900006D17B68002283F83C20786800F039F888
:1024A0007B68022283F83D207B681A687B680433CE
:1024B0001946104600F0E2FB7B68012283F84620B3
:1024C0007B68012283F83E207B68012283F83F204D
:1024D0007B68012283F840207B68012283F8412039
:1024E0007B68012283F842207B68012283F8432025
:1024F0007B68012283F844207B68012283F8452011
:102500007B68012283F83D20002318460837BD462A
:1025100080BD80B483B000AF786000BF0C37BD468B
:1025200080BC704780B584B000AF786039603B688C
:10253000002B09D17B6893F83E30DBB2012B14BF2E
:1025400001230023DBB222E03B68042B09D17B6826
:1025500093F83F30DBB2012B14BF01230023DBB221
:1025600015E03B68082B09D17B6893F84030DBB25B
:10257000012B14BF01230023DBB208E07B6893F832
:102580004130DBB2012B14BF01230023DBB2002B4F
:1025900001D0012363E03B68002B04D17B68022259
:1025A00083F83E2013E03B68042B04D17B680222B1
:1025B00083F83F200BE03B68082B04D17B680222A4
:1025C00083F8402003E07B68022283F841207B6887
:1025D0001B6801223968184600F0E6FD7B681B681D
:1025E000214A934207D17B681B685A6C7B681B6841
:1025F00042F400425A647B681B681B4A934213D022
:102600007B681B68B3F1804F0ED07B681B68174A4C
:10261000934209D07B681B68154A934204D07B68BB
:102620001B68144A934211D17B681B689B6803F0B6
:102630000703FB60FB68062B10D07B681B681A68D9
:102640007B681B6842F001021A6007E07B681B6828
:102650001A687B681B6842F001021A600023184662
:102660001037BD4680BD00BF002C01400004004073
:1026700000080040000C004080B584B000AF7860D6
:102680007B681B68DB68FB607B681B681B69BB6041
:10269000BB6803F00203002B20D0FB6803F00203A9
:1026A000002B1BD07B681B686FF002021A617B68ED
:1026B00001221A777B681B689B6903F00303002BD8
:1026C00003D0786800F0BFFA05E0786800F0B2FA4D
:1026D000786800F0C1FA7B6800221A77BB6803F0C3
:1026E0000403002B20D0FB6803F00403002B1BD055
:1026F0007B681B686FF004021A617B6802221A77FC
:102700007B681B689B6903F44073002B03D07868D7
:1027100000F099FA05E0786800F08CFA786800F02B
:102720009BFA7B6800221A77BB6803F00803002B32
:1027300020D0FB6803F00803002B1BD07B681B68CC
:102740006FF008021A617B6804221A777B681B68A5
:10275000DB6903F00303002B03D0786800F073FA01
:1027600005E0786800F066FA786800F075FA7B6832
:1027700000221A77BB6803F01003002B20D0FB68FF
:1027800003F01003002B1BD07B681B686FF0100256
:102790001A617B6808221A777B681B68DB6903F47F
:1027A0004073002B03D0786800F04DFA05E078689C
:1027B00000F040FA786800F04FFA7B6800221A7740
:1027C000BB6803F00103002B0CD0FB6803F001038E
:1027D000002B07D07B681B686FF001021A617868D4
:1027E00000F01FFABB6803F08003002B0CD0FB68DD
:1027F00003F08003002B07D07B681B686FF080021A
:102800001A61786800F063FDBB6803F04003002B99
:102810000CD0FB6803F04003002B07D07B681B68DB
:102820006FF040021A61786800F01FFABB6803F08D
:102830002003002B0CD0FB6803F02003002B07D0F3
:102840007B681B686FF020021A61786800F036FD23
:1028500000BF1037BD4680BD80B586B000AFF860C0
:10286000B9607A600023FB75FB6893F83C30012B5C
:1028700001D1022348E0FB68012283F83C207B68F9
:102880000C2B39D801A252F823F000BFC12801084F
:10289000F9280108F9280108F9280108CF280108BA
:1028A000F9280108F9280108F9280108DD2801089C
:1028B000F9280108F9280108F9280108EB2801087E
:1028C000FB681B68B968184600F050FA17E0FB680F
:1028D0001B68B968184600F0AFFA10E0FB681B6887
:1028E000B968184600F012FB09E0FB681B68B9687C
:1028F000184600F075FB02E00123FB7500BFFB6882
:10290000002283F83C20FB7D18461837BD4680BD69
:1029100080B586B000AFF860B9607A600023FB75BF
:10292000FB6893F83C30012B01D10223AEE0FB6839
:10293000012283F83C207B680C2B00F29F8001A2CF
:1029400052F823F0792901087D2A01087D2A01081F
:102950007D2A0108B92901087D2A01087D2A01087C
:102960007D2A0108FB2901087D2A01087D2A01082A
:102970007D2A01083B2A0108FB681B68B9681846D4
:1029800000F0F4F9FB681B689A69FB681B6842F069
:1029900008029A61FB681B689A69FB681B6822F051
:1029A00004029A61FB681B689969BB681A69FB6835
:1029B0001B680A439A6164E0FB681B68B9681846A3
:1029C00000F03AFAFB681B689A69FB681B6842F4DE
:1029D00000629A61FB681B689A69FB681B6822F4B5
:1029E00080629A61FB681B689969BB681B691A025F
:1029F000FB681B680A439A6143E0FB681B68B9687F
:102A0000184600F083FAFB681B68DA69FB681B68EC
:102A100042F00802DA61FB681B68DA69FB681B6830
:102A200022F00402DA61FB681B68D969BB681A6985
:102A3000FB681B680A43DA6123E0FB681B68B9681E
:102A4000184600F0CDFAFB681B68DA69FB681B6862
:102A500042F40062DA61FB681B68DA69FB681B6894
:102A600022F48062DA61FB681B68D969BB681B6964
:102A70001A02FB681B680A43DA6102E00123FB7556
:102A800000BFFB68002283F83C20FB7D1846183706
:102A9000BD4680BD80B584B000AF7860396000234A
:102AA000FB737B6893F83C30012B01D10223B4E027
:102AB0007B68012283F83C207B68022283F83D205A
:102AC0007B681B689B68BB60BB6823F07703BB60B7
:102AD000BB6823F47F43BB607B681B68BA689A605D
:102AE0003B681B68B3F5005F3ED0B3F5005F00F2B2
:102AF0008780B3F5805F00F08680B3F5805F7FD874
:102B0000702B1AD0702B7BD8602B50D0602B77D8CD
:102B1000502B3CD0502B73D8402B58D0402B6FD823
:102B2000302B64D0302B6BD8202B60D0202B67D873
:102B3000002B5CD0102B5AD062E07B6818683B6891
:102B400099683B685A683B68DB6800F00EFB7B685D
:102B50001B689B68BB60BB6843F07703BB607B6806
:102B60001B68BA689A604FE07B6818683B68996890
:102B70003B685A683B68DB6800F0F7FA7B681B68C3
:102B80009A687B681B6842F480429A603CE07B68EC
:102B900018683B6859683B68DB681A4600F06EFAB3
:102BA0007B681B685021184600F0C5FA2CE07B6852
:102BB00018683B6859683B68DB681A4600F08CFA75
:102BC0007B681B686021184600F0B5FA1CE07B6842
:102BD00018683B6859683B68DB681A4600F04EFA93
:102BE0007B681B684021184600F0A5FA0CE07B6862
:102BF0001A683B681B681946104600F09CFA03E00F
:102C00000123FB7300E000BF7B68012283F83D20B5
:102C10007B68002283F83C20FB7B18461037BD46BA
:102C200080BD80B483B000AF786000BF0C37BD4674
:102C300080BC704780B483B000AF786000BF0C37B1
:102C4000BD4680BC704780B483B000AF786000BFE1
:102C50000C37BD4680BC704780B483B000AF78604D
:102C600000BF0C37BD4680BC704780B483B000AF56
:102C7000786000BF0C37BD4680BC704780B485B01B
:102C800000AF786039607B681B68FB607B68334A03
:102C900093420FD07B68B3F1804F0BD07B68304AF2
:102CA000934207D07B682F4A934203D07B682E4A19
:102CB000934208D1FB6823F07003FB603B685B68BC
:102CC000FA681343FB607B68244A93420FD07B6809
:102CD000B3F1804F0BD07B68214A934207D07B68C9
:102CE000204A934203D07B681F4A934208D1FB6875
:102CF00023F44073FB603B68DB68FA681343FB60B6
:102D0000FB6823F080023B685B691343FB607B68D0
:102D1000FA681A603B689A687B68DA623B681A68EE
:102D20007B689A627B680D4A934203D13B681A69BB
:102D30007B681A637B6801225A617B681B6903F018
:102D40000103002B05D07B681B6923F001027B681F
:102D50001A6100BF1437BD4680BC7047002C01408B
:102D60000004004000080040000C004080B487B020
:102D700000AF786039607B681B6A7B617B681B6A87
:102D800023F001027B681A627B685B683B617B68A9
:102D90009B69FB60FB6823F07003FB60FB6823F01A
:102DA0000303FB603B681B68FA681343FB607B69A5
:102DB00023F002037B613B689B687A6913437B6164
:102DC0007B681C4A93420CD17B6923F008037B612A
:102DD0003B68DB687A6913437B617B6923F00403FA
:102DE0007B617B68134A934211D13B6923F4807362
:102DF0003B613B6923F400733B613B685B693A6963
:102E000013433B613B689B693A6913433B617B68B1
:102E10003A695A607B68FA689A613B685A687B68CD
:102E20005A637B687A691A6200BF1C37BD4680BC52
:102E3000704700BF002C014080B487B000AF7860BD
:102E400039607B681B6A7B617B681B6A23F0100218
:102E50007B681A627B685B683B617B689B69FB608F
:102E6000FB6823F4E043FB60FB6823F44073FB60E2
:102E70003B681B681B02FA681343FB607B6923F005
:102E800020037B613B689B681B017A6913437B616C
:102E90007B681D4A93420DD17B6923F080037B61DF
:102EA0003B68DB681B017A6913437B617B6923F014
:102EB00040037B617B68144A934213D13B6923F43E
:102EC00080633B613B6923F400633B613B685B6962
:102ED0009B003A6913433B613B689B699B003A69DD
:102EE00013433B617B683A695A607B68FA689A6170
:102EF0003B685A687B689A637B687A691A6200BF8C
:102F00001C37BD4680BC7047002C014080B487B0A0
:102F100000AF786039607B681B6A7B617B681B6AE5
:102F200023F480727B681A627B685B683B617B6814
:102F3000DB69FB60FB6823F07003FB60FB6823F038
:102F40000303FB603B681B68FA681343FB607B6903
:102F500023F400737B613B689B681B027A6913430F
:102F60007B617B681D4A93420DD17B6923F400632A
:102F70007B613B68DB681B027A6913437B617B6979
:102F800023F480637B617B68144A934213D13B69CD
:102F900023F480533B613B6923F400533B613B685E
:102FA0005B691B013A6913433B613B689B691B01E9
:102FB0003A6913433B617B683A695A607B68FA68F7
:102FC000DA613B685A687B68DA637B687A691A62FF
:102FD00000BF1C37BD4680BC704700BF002C0140BD
:102FE00080B487B000AF786039607B681B6A3B6152
:102FF0007B681B6A23F480527B681A627B685B687B
:103000007B617B68DB69FB60FB6823F4E043FB606A
:10301000FB6823F44073FB603B681B681B02FA6883
:103020001343FB603B6923F400533B613B689B689F
:103030001B033A6913433B617B680F4A934209D1F2
:103040007B6923F480437B613B685B699B017A6900
:1030500013437B617B687A695A607B68FA68DA613E
:103060003B685A687B681A647B683A691A6200BFD9
:103070001C37BD4680BC7047002C014080B487B02F
:1030800000AFF860B9607A60FB681B6A7B61FB681F
:103090001B6A23F00102FB681A62FB689B693B61B3
:1030A0003B6923F0F0033B617B681B013A691343E2
:1030B0003B617B6923F00A037B617A69BB68134338
:1030C0007B61FB683A699A61FB687A691A6200BFA2
:1030D0001C37BD4680BC704780B487B000AFF86035
:1030E000B9607A60FB681B6A7B61FB681B6A23F02E
:1030F0001002FB681A62FB689B693B613B6923F421
:1031000070433B617B681B033A6913433B617B69F6
:1031100023F0A0037B61BB681B017A6913437B61C9
:10312000FB683A699A61FB687A691A6200BF1C37CA
:10313000BD4680BC704780B485B000AF7860396010
:103140007B689B68FB60FB6823F07003FB603A6858
:10315000FB68134343F00703FB607B68FA689A60DF
:1031600000BF1437BD4680BC704780B487B000AF45
:10317000F860B9607A603B60FB689B687B617B6943
:1031800023F47F437B613B681A027B681A43BB6868
:1031900013437A6913437B61FB687A699A6000BFC5
:1031A0001C37BD4680BC704780B487B000AFF86064
:1031B000B9607A60BB6803F01F03012202FA03F3CF
:1031C0007B61FB681A6A7B69DB431A40FB681A6201
:1031D000FB681A6ABB6803F01F03796801FA03F3FE
:1031E0001A43FB681A6200BF1C37BD4680BC70479B
:1031F00080B485B000AF786039607B6893F83C306C
:10320000012B01D102234BE07B68012283F83C2093
:103210007B68022283F83D207B681B685B68FB604B
:103220007B681B689B68BB60FB6823F07003FB60D6
:103230003B681B68FA681343FB607B681B68FA688D
:103240005A607B681B68194A934213D07B681B68DD
:10325000B3F1804F0ED07B681B68154A934209D0AA
:103260007B681B68134A934204D07B681B68124A30
:1032700093420CD1BB6823F08003BB603B685B6862
:10328000BA681343BB607B681B68BA689A607B6846
:10329000012283F83D207B68002283F83C20002334
:1032A00018461437BD4680BC704700BF002C014053
:1032B0000004004000080040000C004080B483B0CF
:1032C00000AF786000BF0C37BD4680BC704780B44B
:1032D00083B000AF786000BF0C37BD4680BC70473C
:1032E00080B582B000AF78607B68002B01D10123EC
:1032F00042E07B6893F84130DBB2002B06D17B685B
:10330000002283F840207868FAF7C2FF7B68242205
:1033100083F841207B681B68DA687B681B6822F4AD
:103320000052DA60786801F003F97B681B681A695B
:103330007B681B6822F490421A617B681B685A699B
:103340007B681B6822F02A025A617B681B68DA6876
:103350007B681B6842F40052DA607B6800225A6482
:103360007B68202283F841207B68202283F842205A
:103370007B6800225A63002318460837BD4680BD8B
:1033800080B58CB000AFF860B9601346FB80FB6875
:1033900093F84130DBB2202B56D1BB68002B02D012
:1033A000FB88002B01D101234FE0BA68FB681A6249
:1033B000FB68FA889A84FB68FA88DA84FB68002242
:1033C0005A64FB68212283F84120FB689B6B214AE9
:1033D0009A62FB689B6B204ADA62FB689B6B1F4A10
:1033E0001A63FB689B6B00225A6307F10803FB62B8
:1033F000FB68986BFB6A1968FB681B6804331A4604
:10340000FB88FCF7A5FFFB681B686FF040021A60A1
:10341000FB681B681433BB61BB6953E8003F7B61E9
:103420007B6943F08003BB62FB681B681433BA6A94
:103430007A623B62396A7A6A41E80023FB61FB6980
:10344000002BE5D1002300E0022318463037BD46AB
:1034500080BD00BF553D0108EF3D0108733F0108E5
:1034600080B58CB000AFF860B9601346FB80FB6894
:1034700093F84230DBB2202B4AD1BB68002B02D03C
:10348000FB88002B01D1012343E0FB6801221A6372
:10349000FB6800225A63FB881A46B968F86800F096
:1034A000B2FD034687F82F3097F82F30002B2CD130
:1034B000FB681B6B012B25D100233B61FB681B685C
:1034C0001B683B61FB681B685B683B613B69FB6891
:1034D0001B680C33BB61BB6953E8003F7B617B69B0
:1034E00043F01003BB62FB681B680C33BA6A7A6254
:1034F0003B62396A7A6A41E80023FB61FB69002B71
:10350000E5D102E0012387F82F3097F82F3000E053
:10351000022318463037BD4680BD80B58CB000AF61
:10352000F860B9601346FB80FB6893F84230DBB269
:10353000202B46D1BB68002B02D0FB88002B01D189
:1035400001233FE0FB6801221A63FB6800225A63F3
:10355000FB881A46B968F86800F08EFD034687F8C4
:103560002F30FB681B6B012B25D100233B61FB68CF
:103570001B681B683B61FB681B685B683B613B69C0
:10358000FB681B680C33BB61BB6953E8003F7B6180
:103590007B6943F01003BB62FB681B680C33BA6A9B
:1035A0007A623B62396A7A6A41E80023FB61FB690F
:1035B000002BE5D102E0012387F82F3097F82F3058
:1035C00000E0022318463037BD4680BD80B58EB07E
:1035D00000AF78607B681B680C333B623B6A53E842
:1035E000003FFB61FB6923F0C0037B637B681B68C2
:1035F0000C337A6BFA62BB62B96AFA6A41E800235B
:103600007B627B6A002BE5D17B681B685B6903F0FA
:103610008003002B36D07B681B681433FB60FB688B
:1036200053E8003FBB60BB6823F080033B637B68CB
:103630001B6814333A6BBA617B617969BA6941E8F6
:1036400000233B613B69002BE5D17B689B6B002B22
:1036500018D07B689B6B00225A637B689B6B184673
:10366000FCF7D6FE0346002B0CD07B689B6B1846FC
:10367000FDF74EFA0346202B04D17B6810225A64D2
:10368000032307E07B680022DA847B68202283F82A
:103690004120002318463837BD4680BD80B59AB01A
:1036A00000AF78607B681B680C33BB64BB6C53E86D
:1036B000003F7B647B6C23F490737B667B681B68A4
:1036C0000C337A6E7A653B65396D7A6D41E800237B
:1036D000FB64FB6C002BE5D17B681B6814337B63B8
:1036E0007B6B53E8003F3B633B6B23F001033B667E
:1036F0007B681B6814333A6E3A64FB63F96B3A6C6F
:1037000041E80023BB63BB6B002BE5D17B681B6BDF
:10371000012B19D17B681B680C333B623B6A53E871
:10372000003FFB61FB6923F01003FB657B681B68AE
:103730000C33FA6DFA62BB62B96AFA6A41E8002397
:103740007B627B6A002BE5D17B681B685B6903F0B9
:103750004003002B36D07B681B681433FB60FB688A
:1037600053E8003FBB60BB6823F04003BB657B6848
:103770001B681433BA6DBA617B617969BA6941E833
:1037800000233B613B69002BE5D17B68DB6B002BA1
:1037900018D07B68DB6B00225A637B68DB6B1846B2
:1037A000FCF736FE0346002B0CD07B68DB6B18461B
:1037B000FDF7AEF90346202B04D17B6810225A6432
:1037C00003230AE07B680022DA857B68202283F8E5
:1037D00042207B6800221A63002318466837BD46E2
:1037E00080BD000080B5BAB000AF78607B681B6810
:1037F0001B68C7F8E4307B681B68DB68C7F8E030FB
:103800007B681B685B69C7F8DC300023C7F8D830D9
:103810000023C7F8D430D7F8E43003F00F03C7F81B
:10382000D830D7F8D830002B0FD1D7F8E43003F0D8
:103830002003002B09D0D7F8E03003F02003002B41
:1038400003D0786800F0B6FD5BE2D7F8D830002BE3
:1038500000F0DE80D7F8DC3003F00103002B06D146
:10386000D7F8E03003F49073002B00F0D180D7F844
:10387000E43003F00103002B0BD0D7F8E03003F461
:103880008073002B05D07B685B6C43F001027B6882
:103890005A64D7F8E43003F00403002B0BD0D7F8B8
:1038A000DC3003F00103002B05D07B685B6C43F038
:1038B00002027B685A64D7F8E43003F00203002B5D
:1038C0000BD0D7F8DC3003F00103002B05D07B6868
:1038D0005B6C43F004027B685A64D7F8E43003F071
:1038E0000803002B11D0D7F8E03003F02003002BA1
:1038F00005D1D7F8DC3003F00103002B05D07B683D
:103900005B6C43F008027B685A647B685B6C002B3D
:1039100000F0F281D7F8E43003F02003002B08D048
:10392000D7F8E03003F02003002B02D0786800F0D5
:1039300041FD7B681B685B6903F04003002B14BFEB
:1039400001230023DBB2C7F8D4307B685B6C03F043
:103950000803002B03D1D7F8D430002B4FD0786860
:1039600000F04BFC7B681B685B6903F04003002B95
:1039700041D07B681B681433C7F89C30D7F89C3063
:1039800053E8003FC7F89830D7F8983023F0400349
:10399000C7F8D0307B681B681433D7F8D020C7F83D
:1039A000A820C7F8A430D7F8A410D7F8A82041E879
:1039B0000023C7F8A030D7F8A030002BD9D17B68FE
:1039C000DB6B002B13D07B68DB6B7E4A5A637B6812
:1039D000DB6B1846FCF758FD0346002B16D07B68BE
:1039E000DB6B5B6B7A68D26B104698470EE07868A9
:1039F000F8F78EFB0AE07868F8F78AFB06E078684B
:103A0000F8F786FB7B6800225A6475E100BF73E11A
:103A10007B681B6B012B40F04F81D7F8E43003F03B
:103A20001003002B00F04881D7F8E03003F01003BA
:103A3000002B00F041810023BB607B681B681B6882
:103A4000BB607B681B685B68BB60BB687B681B688E
:103A50005B6903F04003002B00F0B6807B68DB6BF2
:103A60001B685B68A7F8BE30B7F8BE30002B00F0CB
:103A700045817B689B8DB7F8BE209A4280F03E81DD
:103A80007B68B7F8BE20DA857B68DB6B9B69202BEF
:103A900000F088807B681B680C33C7F88830D7F843
:103AA000883053E8003FC7F88430D7F8843023F4D7
:103AB0008073C7F8B8307B681B680C33D7F8B82020
:103AC000C7F89420C7F89030D7F89010D7F8942012
:103AD00041E80023C7F88C30D7F88C30002BD9D1BF
:103AE0007B681B6814337B677B6F53E8003F3B6741
:103AF0003B6F23F00103C7F8B4307B681B681433B5
:103B0000D7F8B420C7F88020FB67F96FD7F880207A
:103B100041E80023BB67BB6F002BE1D17B681B68CA
:103B200014333B663B6E53E8003FFB65FB6D23F0AF
:103B30004003C7F8B0307B681B681433D7F8B02057
:103B4000FA66BB66B96EFA6E41E800237B667B6E4F
:103B5000002BE3D17B68202283F842207B6800227F
:103B60001A637B681B680C33FB64FB6C53E8003FF3
:103B7000BB64BB6C23F01003C7F8AC307B681B68D8
:103B80000C33D7F8AC20BA657B65796DBA6D41E826
:103B900000233B653B6D002BE3D17B68DB6B184654
:103BA000FCF736FC7B6802225A637B689A8D7B683F
:103BB000DB8D9BB2D31A9BB219467868F9F7F2F9FC
:103BC0009CE000BFBF4201087B689A8D7B68DB8D5B
:103BD0009BB2D31AA7F8CE307B68DB8D9BB2002B4B
:103BE00000F08E80B7F8CE30002B00F089807B6823
:103BF0001B680C33BB63BB6B53E8003F7B637B6B81
:103C000023F49073C7F8C8307B681B680C33D7F86F
:103C1000C8207A643B64396C7A6C41E80023FB630A
:103C2000FB6B002BE3D17B681B6814337B627B6AE0
:103C300053E8003F3B623B6A23F00103C7F8C430FE
:103C40007B681B681433D7F8C4203A63FB62F96AB7
:103C50003A6B41E80023BB62BB6A002BE3D17B686F
:103C6000202283F842207B6800221A637B681B684D
:103C70000C333B613B6953E8003FFB60FB6823F07A
:103C80001003C7F8C0307B681B680C33D7F8C0201E
:103C9000FA61BB61B969FA6941E800237B617B691C
:103CA000002BE3D17B6802225A63B7F8CE30194665
:103CB0007868F9F777F923E0D7F8E43003F0800368
:103CC000002B09D0D7F8E03003F08003002B03D09D
:103CD000786800F008FB14E0D7F8E43003F0400304
:103CE000002B0ED0D7F8E03003F04003002B08D0B3
:103CF000786800F047FB04E000BF02E000BF00E08E
:103D000000BFE837BD4680BD80B483B000AF7860A7
:103D100000BF0C37BD4680BC704780B483B000AF95
:103D2000786000BF0C37BD4680BC704780B483B05C
:103D300000AF786000BF0C37BD4680BC704780B4D0
:103D400083B000AF78607B685B6C18460C37BD466B
:103D500080BC704780B590B000AF78607B685B6ACC
:103D6000FB637B681B681B6803F02003002B37D1C3
:103D7000FB6B0022DA84FB6B1B6814337B627B6A6B
:103D800053E8003F3B623B6A23F08003BB63FB6B5D
:103D90001B681433BA6B3A63FB62F96A3A6B41E809
:103DA0000023BB62BB6A002BE5D1FB6B1B680C33A5
:103DB0003B613B6953E8003FFB60FB6843F0400315
:103DC0007B63FB6B1B680C337A6BFA61BB61B9696F
:103DD000FA6941E800237B617B69002BE5D102E0B1
:103DE000F86BF9F759F900BF4037BD4680BD80B583
:103DF00084B000AF78607B685B6AFB60F868FFF7AF
:103E000083FF00BF1037BD4680BD80B59CB000AFBA
:103E100078607B685B6AFB667B681B681B6803F0E5
:103E20002003002B72D1FB6E0022DA85FB6E1B682B
:103E30000C33FB64FB6C53E8003FBB64BB6C23F4A6
:103E40008073BB66FB6E1B680C33BA6EBA657B650C
:103E5000796DBA6D41E800233B653B6D002BE5D1E0
:103E6000FB6E1B681433BB63BB6B53E8003F7B6383
:103E70007B6B23F001037B66FB6E1B6814337A6E49
:103E80007A643B64396C7A6C41E80023FB63FB6B1A
:103E9000002BE5D1FB6E1B6814337B627B6A53E811
:103EA000003F3B623B6A23F040033B66FB6E1B68AE
:103EB00014333A6E3A63FB62F96A3A6B41E80023C5
:103EC000BB62BB6A002BE5D1FB6E202283F8422047
:103ED000FB6E1B6B012B19D1FB6E1B680C333B6116
:103EE0003B6953E8003FFB60FB6823F01003FB6570
:103EF000FB6E1B680C33FA6DFA61BB61B969FA6934
:103F000041E800237B617B69002BE5D1FB6E002239
:103F10005A63FB6E1B6B012B06D1FB6E9B8D194602
:103F2000F86EF9F73FF802E0F86EFFF7F6FE00BF13
:103F30007037BD4680BD80B584B000AF78607B68C7
:103F40005B6AFB60FB6801225A63FB681B6B012BF9
:103F500008D1FB689B8D5B089BB21946F868F9F79E
:103F600021F802E0F868FFF7E1FE00BF1037BD4618
:103F700080BD80B584B000AF78600023FB607B68B3
:103F80005B6ABB60BB681B685B6903F08003002B46
:103F900014BF01230023DBB2FB60BB6893F8413000
:103FA000DBB2212B08D1FB68002B05D0BB680022B7
:103FB000DA84B86800F0FAF8BB681B685B6903F044
:103FC0004003002B14BF01230023DBB2FB60BB685E
:103FD00093F84230DBB2222B08D1FB68002B05D0CE
:103FE000BB680022DA85B86800F007F9BB685B6C33
:103FF00043F01002BB685A64B868F8F789F800BF4C
:104000001037BD4680BD80B485B000AFF860B960A0
:104010001346FB80FB68BA689A62FB68FA889A8547
:10402000FB68FA88DA85FB6800225A64FB68222262
:1040300083F84220FB681B69002B07D0FB681B68D4
:10404000DA68FB681B6842F48072DA60FB681B6800
:104050005A69FB681B6842F001025A61FB681B68E1
:10406000DA68FB681B6842F02002DA600023184619
:104070001437BD4680BC704780B598B000AFF8607B
:10408000B9601346FB80BA68FB689A62FB68FA88DD
:104090009A85FB6800225A64FB68222283F842203A
:1040A000FB68DB6B3E4A9A62FB68DB6B3D4ADA6277
:1040B000FB68DB6B3C4A1A63FB68DB6B00225A63CC
:1040C00007F10803FB65FB68D86BFB681B680433CA
:1040D0001946FB6D1A68FB88FCF73AF900233B612F
:1040E000FB681B681B683B61FB681B685B683B6186
:1040F0003B69FB681B69002B19D0FB681B680C33FC
:104100003B643B6C53E8003FFB63FB6B43F4807301
:10411000BB65FB681B680C33BA6DFA64BB64B96C91
:10412000FA6C41E800237B647B6C002BE5D1FB68D3
:104130001B681433FB62FB6A53E8003FBB62BB6A37
:1041400043F001037B65FB681B6814337A6DBA6327
:104150007B63796BBA6B41E800233B633B6B002BBD
:10416000E5D1FB681B681433BB61BB6953E8003FB2
:104170007B617B6943F040033B65FB681B6814333C
:104180003A6D7A623B62396A7A6A41E80023FB61E0
:10419000FB69002BE5D1002318466037BD4680BD82
:1041A0000B3E0108373F0108733F010880B489B016
:1041B00000AF78607B681B680C33FB60FB6853E8DA
:1041C000003FBB60BB6823F0C003FB617B681B68DA
:1041D0000C33FA69BA617B617969BA6941E80023F5
:1041E0003B613B69002BE5D17B68202283F84120AD
:1041F00000BF2437BD4680BC704780B495B000AF87
:1042000078607B681B680C337B637B6B53E8003FF3
:104210003B633B6B23F49073FB647B681B680C333C
:10422000FA6C3A64FB63F96B3A6C41E80023BB63B8
:10423000BB6B002BE5D17B681B6814333B623B6A88
:1042400053E8003FFB61FB6923F00103BB647B681B
:104250001B681433BA6CFA62BB62B96AFA6A41E845
:1042600000237B627B6A002BE5D17B681B6B012BF3
:1042700019D17B681B680C33FB60FB6853E8003F77
:10428000BB60BB6823F010037B647B681B680C3346
:104290007A6CBA617B617969BA6941E800233B6154
:1042A0003B69002BE5D17B68202283F842207B68A4
:1042B00000221A6300BF5437BD4680BC704780B5EA
:1042C00084B000AF78607B685B6AFB60FB680022AB
:1042D000DA85FB680022DA84F868F7F719FF00BF77
:1042E0001037BD4680BD80B485B000AF78607B6874
:1042F00093F84130DBB2212B3ED17B689B68B3F54C
:10430000805F14D17B681B69002B10D17B681B6A0E
:10431000FB60FB681B881A467B681B68C2F30802B7
:104320005A607B681B6A9A1C7B681A6208E07B688B
:104330001B6A591C7A6811621A787B681B685A607C
:104340007B68DB8C9BB2013B9BB27A681946D184B7
:10435000002B0FD17B681B68DA687B681B6822F032
:104360008002DA607B681B68DA687B681B6842F051
:104370004002DA60002300E0022318461437BD46ED
:1043800080BC704780B582B000AF78607B681B68E6
:10439000DA687B681B6822F04002DA607B682022C2
:1043A00083F841207868F8F777FE0023184608372D
:1043B000BD4680BD80B58CB000AF78607B6893F857
:1043C0004230DBB2222B40F0AE807B689B68B3F5B5
:1043D000805F17D17B681B69002B13D10023FB6220
:1043E0007B689B6ABB627B681B685B689BB2C3F39C
:1043F00008039AB2BB6A1A807B689B6A9A1C7B6826
:104400009A6226E07B689B6AFB620023BB627B6842
:104410009B68B3F5805F07D07B689B68002B0AD14F
:104420007B681B69002B06D17B681B685B68DAB26E
:10443000FB6A1A7008E07B681B685B68DBB203F0FC
:104440007F03DAB2FB6A1A707B689B6A5A1C7B682E
:104450009A627B68DB8D9BB2013B9BB27A681946FE
:10446000D185002B5DD17B681B68DA687B681B688F
:1044700022F02002DA607B681B68DA687B681B68C0
:1044800022F48072DA607B681B685A697B681B685B
:1044900022F001025A617B68202283F842207B6867
:1044A00000225A637B681B6B012B35D17B6800228D
:1044B0001A637B681B680C337B617B6953E8003FA0
:1044C0003B613B6923F010037B627B681B680C3304
:1044D0007A6A3A62FB61F9693A6A41E80023BB6192
:1044E000BB69002BE5D17B681B681B6803F01003D8
:1044F000102B0AD10023FB607B681B681B68FB60E4
:104500007B681B685B68FB60FB687B689B8D19465A
:104510007868F8F747FD02E07868FFF7FEFB0023B4
:1045200002E0002300E0022318463037BD4680BD7C
:1045300080B584B000AF78607B681B681B6923F48A
:1045400040517B68DA687B681B680A431A617B68A4
:104550009A687B681B691A437B685B691343BB607D
:104560007B681B68DB6823F4B05323F00C037A6884
:104570001268B9680B43D3607B681B685B6923F4DE
:1045800040717B689A697B681B680A435A617B6843
:104590001B682C4A934203D1FDF75CFAF86002E0F5
:1045A000FDF744FAF860FA6813469B0013449A003A
:1045B0001A447B685B689B00B2FBF3F3224AA2FBC0
:1045C00003235B091901FA6813469B0013449A0000
:1045D0001A447B685B689B00B2FBF3F21A4BA3FBA7
:1045E00002035B09642000FB03F3D31A1B0132337F
:1045F000154AA2FB03235B0903F0F0031944FA6890
:1046000013469B0013449A001A447B685B689B0026
:10461000B2FBF3F20C4BA3FB02035B09642000FB2B
:1046200003F3D31A1B013233074AA2FB03235B09AE
:1046300003F00F027B681B680A449A6000BF1037C2
:10464000BD4680BD003801401F85EB51002B2DE990
:10465000F0471D46BBBF03F100431D4600232D2339
:1046600088B01446B8BF1446129A109E1370149B5B
:10467000DDF84CA023F02008B8F1460F05D0B8F1C2
:10468000450F00D10136022300E0032307AA04925C
:1046900006AACDE902A2CDE9003622462B4600F05B
:1046A0002BFEB8F1470F074619D1119BDB070ED53A
:1046B00000EB06090022002320462946F4F7E0F922
:1046C00008B1CDF81C903022079B4B451ED33846CD
:1046D000079B159ADB1B136008B0BDE8F087B8F1A3
:1046E000460F00EB0609E5D10378302B0AD10022F2
:1046F000002320462946F4F7C3F918B9C6F101068C
:10470000CAF80060DAF800309944D3E7591C0791E1
:104710001A70D9E7F7B50029B6BF2D232B234942DC
:1047200009290270437029DD0DF107031D460A2790
:10473000B1FBF7F61A4607FB1614303402F8014CA9
:104740000C46632C314603F1FF33F1DC3031941E0B
:1047500003F8011C2346411CAB420AD30DF10903A7
:104760009B1AAC4288BF002302330344181A03B0DB
:10477000F0BD13F8016B01F8016FEDE73023303124
:104780008370C170031DF1E72DE9F04F91B00C4625
:10479000DDF8688016461F46054600F0E5FC036814
:1047A00018460893F3F740FD00230E93D8F8003025
:1047B0000990073323F0070303F1080294F818A0C7
:1047C000D4F800B0C8F80020D3E9008929F00043EC
:1047D0000B93CDF828804FF0FF32DDE90A01C4E9E0
:1047E00012899C4BF4F77EF970BBDDE90A014FF0AA
:1047F000FF32984BF4F758F930BB002200234046B3
:104800004946F4F747F910B12D2384F84330924A12
:10481000924BBAF1470F8CBF9046984603234FF056
:10482000000923612BF00403236033462146284608
:1048300000970FAA00F0D4F9013040F090804FF0BB
:10484000FF3011B0BDE8F08F42464B464046494626
:10485000F4F748F948B14B46002BB8BF2D23804AE6
:10486000B8BF84F843307F4BD3E763680AF0DF01B9
:104870005A1C3FD10623636000224BF480632360FF
:1048800006920EAACDE904A20DAA03920DF13302FD
:10489000CDE9013263684246009328464B460A91AF
:1048A000FFF7D4FE0A99804647290D9928D1C81CE4
:1048B00002DB6368994240DDAAF1020A5FFA8AFAD4
:1048C0005246013904F150000D91FFF723FF0E9A73
:1048D00081461318012A236102DC2268D20701D520
:1048E000013323619DF83330002B9ED02D2384F8B3
:1048F00043309AE74729BFD1002BBDD10123BAE746
:10490000BAF1650FDCD9BAF1660F18D100296368D6
:104910000BDD216113B92268D00702D501330B44A6
:1049200023614FF00009A165DCE713B92268D207C3
:1049300001D50233F4E70123F2E74FF0670A0E9B3B
:10494000994205DB23682161D807EAD54B1CE7E7CC
:104950000029CCBF0122C1F102021344E0E7236821
:104960005A0507D42369424631462846B8470130E4
:104970002BD164E7BAF1650F40F2DC80D4E9120173
:1049800000220023F4F77CF8002833D001233146BD
:104990002846354AB84701303FF451AFDDE90D38BC
:1049A000434502DB2368D8070FD5DDE908233146EC
:1049B0002846B84701303FF442AF4FF0000908F1F4
:1049C000FF3804F11A0AC84509DC23689B0700F187
:1049D0000281E0680F9B9842B8BF184631E7012377
:1049E000524631462846B84701303FF428AF09F116
:1049F0000109E8E70D9B002B38DC012331462846EE
:104A0000194AB84701303FF41AAFDDE90D3959EAC8
:104A1000030302D12368D907D7D5DDE9082331463E
:104A20002846B84701303FF40AAF4FF0000A04F1BE
:104A30001A0B0D9B5B42534501DC4B4693E7012368
:104A40005A4631462846B84701303FF4F8AE0AF1DD
:104A5000010AEEE7FFFFEF7FC07D0108BC7D010882
:104A6000C87D0108C47D0108CC7D0108A36DDDF877
:104A700038A05345A8BF5346002B994636DC4FF06B
:104A8000000B29EAE97904F11A02A36D0A93A3EB5A
:104A900009035B4531DC0D9B9A453ADC2368DA0754
:104AA00037D40D9BAAEB03090A9BAAEB0303994594
:104AB000A8BF9946B9F1000F33DC4FF0000829EA8E
:104AC000E97904F11A0B0D9BAAEB0303A3EB09038D
:104AD00043457FF77AAF01235A4631462846B84707
:104AE00001303FF4ACAE08F10108ECE74246314634
:104AF0002846B8470130C2D1A1E6012331462846F5
:104B00000A92B84701303FF49AAE0A9A0BF1010BB2
:104B1000BBE73146DDE908232846B8470130C0D15C
:104B20008DE60A9A4B46314628464244B847013042
:104B3000C3D184E6DDF838A0BAF1010F01DCDB0750
:104B400036D50123424631462846B84701303FF466
:104B500076AEDDE9082331462846B84701303FF4F8
:104B60006EAED4E91201002200230AF1FF3AF3F7F6
:104B700087FFC0B9534608F1010231462846B847BD
:104B800001300CD15BE601235A4631462846B8472E
:104B900001303FF454AE08F10108D045F3DB4B4639
:104BA00004F15002E0E64FF0000804F11A0BF4E7BC
:104BB00001234246E1E701234A4631462846B847E9
:104BC00001303FF43CAE08F10108E3680F995B1A2D
:104BD0004345F0DCFDE64FF0000804F11909F4E765
:104BE0002DE9F047164698468A680B6907469342B6
:104BF000B8BF1346336091F843200C46DDF820908F
:104C00000AB1013333602368990642BF3368023327
:104C10003360256815F0060506D104F1190AE3682A
:104C200032689B1AAB422BDC94F843302268003B7D
:104C300018BF0123920630D44146384604F143029E
:104C4000C847013023D02368226903F00603042BF0
:104C500014BF002533684FF0000608BFE56804F173
:104C60001A0408BFED1A54F8123C08BF25EAE5758E
:104C70009342C4BF9B1AED18B5421AD1002008E038
:104C80000123524641463846C847013003D14FF010
:104C9000FF30BDE8F0870135C1E73020E11881F829
:104CA00043005A1C94F845102244023382F8431002
:104CB000C2E70123224641463846C8470130E6D0C4
:104CC0000136D9E72DE9FF470F7E9146782F8046C0
:104CD0000C469A460C9E01F1430207D8622F0AD86F
:104CE000002F00F0D180582F00F0B88004F1420668
:104CF00084F842703AE0A7F16303152BF6D801A1BE
:104D000051F823F05D4D0108714D0108ED4C01088B
:104D1000ED4C0108ED4C0108ED4C0108714D010806
:104D2000ED4C0108ED4C0108ED4C0108ED4C01087B
:104D30006F4E01089B4D0108294E0108ED4C0108FA
:104D4000ED4C0108914E0108ED4C01089B4D010806
:104D5000ED4C0108ED4C0108314E010833681A1D75
:104D60001B68326004F1420684F8423001239CE063
:104D700033682068191D3160060601D51D6803E0FF
:104D80004506FBD5B3F90050002D03DA2D236D4203
:104D900084F843300A23584811E021683368080634
:104DA00053F8045B02D4490648BFADB26F2F33609D
:104DB00014BF0A2308235048002184F84310666872
:104DC000002EA66005DB21682E4321F0040121603E
:104DD0004BD01646B5FBF3F103FB1157C75D06F840
:104DE000017D2F46BB420D46F4D9082B0BD1236819
:104DF000DF0708D5236961689942DEBF302306F8D2
:104E0000013C06F1FF36921B22614B46214640468B
:104E1000CDF800A003AAFFF7E3FE01304AD14FF01E
:104E2000FF3004B0BDE8F087236843F0200323601F
:104E30007827324884F84570236831681F0651F896
:104E4000045B02D45F0648BFADB23160D90744BFEE
:104E500043F0200323601DB11023ADE72648E9E7A6
:104E6000236823F020032360F6E71646BDE7336886
:104E70002568181D616930602E061B6801D5196010
:104E800002E06806FBD51980002316462361BCE7C3
:104E9000336800211A1D32601E686268304600F0D7
:104EA00067F908B1801B606063682361002384F8A0
:104EB0004330AAE73246494640462369D04701308D
:104EC000ADD023689B0713D4E068039B9842B8BF1A
:104ED0001846A6E70123324649464046D0470130EE
:104EE0009DD00135E36803995B1AAB42F2DCEBE736
:104EF000002504F11906F5E7CE7D0108DF7D0108E4
:104F0000002310B50446C0E90033C0E904338360D0
:104F100081814366C2818361194608225C3000F0BA
:104F2000EDF80D4B246263620C4BA3620C4BE36201
:104F30000C4B23630C4B9C4206D003F16802944255
:104F400002D0D0339C4205D104F15800BDE8104096
:104F500000F006B910BD00BF016B0108236B01080A
:104F60005B6B01087F6B0108A0140020024A034913
:104F7000034800F0A5B800BF90000020A563010819
:104F8000A000002041680C4B10B59942044601D0A6
:104F900001F008FAA168094B994202D0204601F0BD
:104FA00001FAE168064B994204D02046BDE8104062
:104FB00001F0F8B910BD00BFA014002008150020B2
:104FC0007015002010B50B4B0B4C0C4A20461A6094
:104FD00004210022FFF794FF04F168000122092157
:104FE000FFF78EFF04F1D0000222BDE8104012212D
:104FF000FFF786BFD8150020A01400206D4F0108D0
:10500000014800F0AEB800BFDD150020014800F0F7
:10501000A9B800BFDD15002010B50446FFF7F0FF6A
:10502000236A1BB1BDE81040FFF7F0BF044B2362B9
:10503000044B1B68002BF5D1FFF7C4FFF2E700BF5C
:10504000854F0108D815002030B51446002C0546C0
:105050001A469BB005DA8B2303604FF0FF301BB07C
:1050600030BD4FF40273ADF80C304FF000031993CC
:105070000CBF234604F1FF33029305934FF6FF73F1
:1050800000910491ADF80E3069461E9B00F064FF5C
:10509000431CBCBF8B232B60002CE0D00022009B64
:1050A0001A70DCE707B5009313460A460146034829
:1050B0000068FFF7C9FF03B05DF804FB9C00002007
:1050C0002DE9F8430746884614460026D4E90195A1
:1050D000B9F1010905D52468002CF7D13046BDE8A7
:1050E000F883AB89012B07D9B5F90E30013303D012
:1050F00029463846C04706436835E9E70346024477
:10510000934200D1704703F8011BF9E7014B18687F
:10511000704700BF9C00002070B500260C4D0D4C60
:10512000641BA410A64209D102F004F900260A4D1E
:105130000A4C641BA410A64205D170BD55F8043B6F
:1051400098470136EEE755F8043B98470136F2E7F9
:105150003C8101083C8101083C8101084081010833
:10516000704770477047000000487047DC0100201E
:10517000034610B5C9B202449342184601D100203B
:1051800003E0047801338C42F6D110BD0A44914209
:1051900000F1FF3300D1704710B511F8014B914277
:1051A00003F8014FF9D110BD1FB514461A46094B3B
:1051B00005461B68D8684CB1074BCDE90134009116
:1051C0002B46064901F0E0FC01F08EFD044B1C4625
:1051D000F3E700BF9C000020F07D0108FD7D010881
:1051E0002B7E01082DE9F74F03690C690746A3429E
:1051F0007EDB013CA30000F1140501F114080093CB
:1052000005EB8403019358F8243055F8242001332A
:105210009A42B2FBF3F608EB84092ED34FF0000A52
:10522000C446AE46D3465CF8043B98B206FB00A0E9
:105230001B0C020C06FB0323DEF8002080B292B2A6
:10524000121A5A44DEF800004FEA134A9BB2C3EB2D
:10525000224303EB104392B242EA0342E1454FEA94
:10526000234B4EF8042BDED2009BEB582BB9019B4D
:10527000043B9D421A462FD33C61384601F038FB6F
:10528000002825DB2946002058F8042BD1F800C05F
:105290001FFA82FE1FFA8CF3A3EB0E030344120CD9
:1052A000C2EB234202EB1C429BB243EA0243C145DC
:1052B0004FEA224041F8043BE6D255F8242005EBA2
:1052C000840322B9043B9D421A460BD33C6101364C
:1052D000304603B0BDE8F08F1268043B002ACBD102
:1052E000013CC6E71268043B002AEFD1013CEAE723
:1052F0000020EEE7000000002DE9F04F14461D46A7
:10530000C76997B08146CDE90645239E7FB9102035
:1053100000F01EFF0246C9F81C0020B9EF21AC4B7B
:10532000AC48FFF741FFC0E901770760C760D9F8D3
:105330001C30196859B15A68012393404A608B6048
:10534000484601F0A3F80022D9F81C301A602B1E41
:10535000AFBF0023012223F000430793A8BF3360AF
:10536000DDF81C809C4BB8BF326033EA080312D1D1
:1053700042F20F73229A1360C8F31303234300F021
:105380005E85249BDFF854A2002B00F060850AF1B3
:10539000030300F05ABDDDE90623CDE90C23DDE966
:1053A0000C0100220023F3F76BFB074658B10123E1
:1053B000229A1360249B13B1894B249A1360DFF85F
:1053C00024A200F044BD14AB019315AB00934846F2
:1053D000DDE90C2301F03CFBC8F30A560390002ED4
:1053E00078D0DDE90C010D9BA6F2FF36C3F3130361
:1053F00043F07F5343F440131297194600227A4B2F
:10540000F2F71EFF6CA3D3E90023F3F7D1F86CA3E6
:10541000D3E90023F2F716FF044630460D46F3F7B2
:105420005DF869A3D3E90023F3F7C2F802460B46FF
:1054300020462946F2F706FF04460D46F3F768FBBF
:1054400000220746002320462946F3F723FB40B1FC
:105450003846F3F743F822462B46F3F711FB00B921
:10546000013F162F54D8DDE90C01604B03EBC70355
:10547000D3E90023F3F70EFB00284BD00023013FB4
:105480000F93149B9B1B5A1E49BFC3F101030023BA
:1054900004930023099254BF04930993002F3BDB2C
:1054A000099B0E973B44099300230A93209B092BE9
:1054B00065D8052BC4BF043B2093209BC8BF0024A4
:1054C000A3F10203D8BF0124032B64D8DFE803F063
:1054D0005355382CDDE914631E4406F23243202B69
:1054E000C1BFC3F1400308FA03F806F2124324FADD
:1054F00003F3D6BFC3F1200348EA030004FA03F024
:10550000F2F7DCFF0122A1F1F873013E129274E779
:105510000123B5E70F90B4E7049BDB1B04937B42A8
:105520000A9300230E93C1E701230B93219B07EB02
:10553000030B0BF10103012B0893B8BF012306E015
:1055400001230B93219B002B28DD9B460893002110
:105550000422D9F81C0002F114059D4226D94160AD
:10556000484600F053FF8246002843D1024640F2ED
:10557000AF111F4BD4E60023E3E70023D5E7012456
:1055800000230B9420934FF0FF3B00221223CDF811
:1055900020B02192DBE701230B93F4E74FF0010BDE
:1055A0005B46CDF820B0CDF884B0D0E70131520091
:1055B000D1E700BFAFF3008061436F63A787D23F9D
:1055C000B3C8608B288AC63FFB799F501344D33FF2
:1055D000397E0108507E01080000F07F357E010809
:1055E000CD7D0108CC7D01080000F83F687F0108EF
:1055F000A87E0108D9F81C301860089B0E2B00F219
:10560000A180002C00F09E80002F33DD9C4B07F022
:105610000F0203EBC203F805D3E90034CDE91034DF
:105620004FEA271416D5DDE90C01964B0326D3E982
:105630000823F3F7E7F8CDE9060104F00F04914DD4
:1056400054B9DDE91023DDE90601F3F7DBF8CDE914
:10565000060128E00226F2E7E10708D5DDE910019E
:10566000D5E90023F2F7A4FFCDE91001013664105B
:105670000835E5E700F0AF80DDE90C017C42804BA6
:1056800004F00F0203EBC203D3E90023F2F790FF0B
:1056900002260023CDE906017A4D2411002C40F0AA
:1056A0008F80002BD3D1DDE906450F9B002B00F046
:1056B0009480002220462946734BF3F7EBF900282B
:1056C00000F08B80089B002B00F08780BBF1000F5F
:1056D00034DD2046002229466C4BF2F769FF5C4618
:1056E000CDE9060107F1FF3801363046F2F7F6FE44
:1056F000DDE90623F2F75CFF0022654BF2F7A2FD1D
:105700000546A1F15076002C6AD1DDE906010022A0
:10571000604BF2F795FD02460B46CDE906232A467B
:105720003346F3F7D5F9002840F09882DDE9060109
:105730002A4606F10043F3F7ADF938BBDDE90C3436
:10574000CDE90634159B002BC0F257810E2F00F3D4
:1057500054814B4B03EBC703D3E90034CDE9043448
:10576000219B002B80F2E580089B002B00F3E18059
:105770000CD1DDE904010022464BF2F719FFDDE907
:105780000623F3F79BF9002800F0668200242546E3
:10579000219B56466FEA030800272146484600F041
:1057A00075FE002D00F0BD802FB1AF4203D0394609
:1057B000484600F06BFE2946484600F067FEB0E020
:1057C000E20705D5D5E90023F2F7F2FE0123013601
:1057D0006410083562E7022665E7B846089C84E74E
:1057E000274B0B9903EBC40353E9022354440029CC
:1057F00054D000202849F3F705F833462A46F2F73B
:105800001FFD5646CDE91001DDE90601F3F780F9E9
:105810000546F2F763FE02460B46DDE90601F2F7A4
:105820000FFD02460B463035CDE90623DDE9102396
:1058300006F8015BF3F72EF9002872D1DDE90623A3
:1058400000201149F2F7FCFCDDE91023F3F722F9FF
:10585000002840F0B480A6423FF470AFDDE91001AB
:1058600000220A4BF2F7A4FE0022CDE91001DDE987
:105870000601064BF2F79CFECDE90601C4E700BF26
:10588000687F0108407F01080000F03F00002440CD
:1058900000001C40000014400000E03F3146284654
:1058A000F2F786FE5646CDE910011394DDE90601B4
:1058B000F3F72EF90546F2F711FE02460B46DDE935
:1058C0000601F2F7BDFC02460B46303506F8015BD7
:1058D000A642CDE906234FF0000224D1DDE91001F4
:1058E000AE4BF2F7AFFC02460B46DDE90601F3F7DB
:1058F000EFF8002863D1DDE910230020A749F2F773
:105900009FFC02460B46DDE90601F3F7C3F80028C9
:105910003FF414AF139E731E139316F8013C302B03
:10592000F8D047463BE09E4BF2F742FECDE9060138
:10593000BCE75646DDE90645DDE904232046294655
:10594000F2F760FFF3F7E4F88046F2F7C7FDDDE910
:105950000423F2F72DFE02460B4620462946F2F7B5
:105960006FFC08F13004089D06F8014BA6EB0A0411
:10597000A54202460B4633D1F2F764FCDDE904236D
:1059800004460D46F3F7A4F8C0B9DDE90423204628
:105990002946F3F775F810B118F0010F0ED14846FB
:1059A000039900F073FD00233370229B01371F60C1
:1059B000249B002B00F04B821E6048E2B846334621
:1059C0001E4613F8012D392A06D19A45F8D1302206
:1059D00008F101088AF800201A7801321A70A0E74D
:1059E00000226F4BF2F7E4FD0022002304460D462F
:1059F000F3F746F800289FD0D1E70B9A002A00F071
:105A0000EA80209A012A00F3CD80129A002A00F041
:105A1000C18003F233430A9C049E049A01211A4474
:105A20000492099A48461A44099200F0E3FD05469B
:105A300066B1099B002B09DDB342A8BF3346049A27
:105A4000F61AD21A0492099AD31A09930A9B0BB335
:105A50000B9B002B00F0C680002C00F0C080294674
:105A60002246484600F07EFE039A01460546484617
:105A700000F0D6FD03998046484600F007FD0A9BDA
:105A80001B1B0A9300F0B18041460A9A484600F079
:105A900069FE03900121484600F0ACFD0E9B0446D0
:105AA000002B00F0D8811A460146484600F05AFE05
:105AB000209B0446012B00F39F80069B002B40F0A7
:105AC0009780079BC3F31303002B40F09380079B41
:105AD00023F000431B0D1B0533B1049B01330493DA
:105AE000099B0133099301230A930E9B002B00F0BD
:105AF000B881236904EB8303186900F02FFDC0F11E
:105B00002000099B184410F01F0000F08280C0F1B3
:105B10002003042B73DD049BC0F11C000344049399
:105B2000099B064403440993049B002B05DD1A4698
:105B30004846039900F070FE0390099B002B05DD99
:105B400021461A46484600F067FE04460F9B002B8C
:105B500061D02146039800F0CBFE00285BDA0023D9
:105B60000A224846039900F0B3FC0B9B07F1FF386B
:105B70000390002B00F07781294600230A22484633
:105B800000F0A6FCBBF1000F05466FDC209B022B4A
:105B900049DC6BE0149BC3F136033CE70000E03FB7
:105BA00000002440089B5C1E0A9BA34209DB1C1BCF
:105BB000089B002BBFF630AF049B089A9E1A002367
:105BC0002BE70A9B0E9AE31A1A440A94049E0024B7
:105BD000089B0E9221E70A9C049E0B9D28E7DDF8A6
:105BE0000C8051E70A9A039950E7CDF80C8051E7F1
:105BF000002379E7069B77E700230A9379E793D0A0
:105C0000049A1C331A440492099A1E441A440992B5
:105C10008AE70346F4E7089BB846002B20DC9B4646
:105C2000209B022B1EDDBBF1000F7FF4B1AD21469E
:105C30005B460522484600F04BFC014604460398AB
:105C400000F056FE00287FF7A3AD5646312308F139
:105C5000010806F8013B9FE5B846089C2546F4E795
:105C6000DDF820B00B9B002B00F00181002E05DD3C
:105C700029463246484600F0CFFD05460A9B002BD8
:105C80005CD04846696800F0C1FB064628B9024668
:105C900040F2EF21804BFFF743BB2A6905F10C016D
:105CA000023292000C30FFF771FA01223146484669
:105CB00000F0B2FD2F4605460AF1010304930AEBFA
:105CC0000B030A93069B03F001030993049B2146EF
:105CD000039803F1FF3BFFF785FA0346394630335B
:105CE000069003980B9300F003FE2A460890214685
:105CF000484600F019FEC26806460B9B02BB0146EF
:105D0000039800F0F5FD02460B9B31464846CDE96D
:105D10000B3200F0BBFB209B0C9A049E42EA03016D
:105D2000099B19430B9B0DD1392B27D0089A002AC8
:105D300001DD069B31338BF800302EE52846B9E7AC
:105D40000122E2E70899002904DB20980143099821
:105D5000014320D1002AEEDD012203994846049335
:105D600000F05AFD2146039000F0C2FD0028049B7C
:105D700002DCE0D1DA07DED5392BDAD139238BF812
:105D8000003033461E4616F8012C013B392A4ED00E
:105D900001321A7001E5002A03DD392BEED0013300
:105DA000C9E7049A0A9902F8013C8A4228D00023E4
:105DB0000A220399484600F08BFBAF4203904FF054
:105DC00000034FF00A023946484607D100F080FB35
:105DD00007460546049B0133049377E700F078FB00
:105DE0002946074600230A22484600F071FB054673
:105DF000F0E7BBF1000FCCBF5E46012600275644FA
:105E0000012203994846049300F006FD21460390C1
:105E100000F06EFD0028B4DC02D1049BDB07B0D497
:105E200033461E4613F8012D302AFAD0B5E49A45C0
:105E3000A8D1312308F101088AF80030ADE4249B91
:105E4000DFF858A01BB10AF10803249A13605046EA
:105E500017B0BDE8F08F209B012B7FF72EAE0E9B75
:105E60000A9301204DE6BBF1000F7FF7D9AE5646ED
:105E700021460398FFF7B6F900F1300306F8013B1D
:105E8000A6EB0A029345B4DD00230A224846039993
:105E900000F01EFB0390EBE7A87E01082C7E0108B2
:105EA0002DE9F0471F468E688246BE420C4690465A
:105EB0000B682DD8B1F90C2012F4906F26D06569CB
:105EC000096905EB4505A3EB010905EBD5757B1CBD
:105ED0004B446D109D4238BF1D46530527D52946BA
:105EE00000F060F9064660B34A462169FFF74EF9B3
:105EF000A38923F4906343F08003A38126614E4479
:105F000026603E466561A5EB0905A560BE4200D945
:105F10003E4632464146206800F076FE0020A368E7
:105F20009B1BA360236833442360BDE8F0872A46A7
:105F300000F03CFE06460028E0D15046216900F002
:105F4000EFFE0C23CAF80030A3894FF0FF3043F076
:105F50004003A381E9E700002DE9F04F98468B89C3
:105F600007461B060D4614469DB010D50B6973B944
:105F7000402100F017F92860286130B90C233B60FC
:105F80004FF0FF301DB0BDE8F08F40236B61002360
:105F9000099320238DF8293030234FF00109CDF8E3
:105FA0000C80DFF898818DF82A3023469A4613F842
:105FB000012B0AB1252AF9D1BAEB040B0BD05B46B1
:105FC000224629463846FFF76BFF013000F0A780D4
:105FD000099A5A4409929AF80030002B00F09F80E9
:105FE00000234FF0FF32CDE905230AF1010A0493A3
:105FF00007938DF853301A935446052214F8011B69
:106000004E48FFF7B5F8049AD8B9D00644BF20230C
:106010008DF85330110744BF2B238DF853309AF875
:1060200000302A2B15D0544600204FF00A0C079A56
:10603000214611F8013B303B092B4BD9B0B10792F7
:1060400014E0A0EB080309FA03F31343A2460493F8
:10605000D2E7039B191D1B680391002BBBBF5B425A
:1060600042F0020207930793B8BF049223782E2BC5
:106070000AD163782A2B32D1039B02341A1D1B6884
:10608000039243EAE3730593DFF8B4A0032250467A
:106090002178FFF76DF838B14022049BA0EB0A008D
:1060A000824013430134049314F8011B062225484F
:1060B0008DF82810FFF75CF8002836D0224B1BBB68
:1060C000039B073323F0070308330393099B3344EF
:1060D00009936AE70C4601200CFB0232A8E7002373
:1060E0004FF00A0C194601340593204610F8012B95
:1060F000303A092A03D9002BC6D00591C4E70446DB
:1061000001230CFB0121F0E703AB00932A4638463C
:106110000E4B04A9FEF738FB421C0646D6D1AB89CC
:106120005B063FF52DAF09982CE703AB00932A4699
:106130003846064B04A9FEF7C5FDEDE7B97E010818
:10614000BF7E0108C37E010889470108A15E0108DE
:10615000024B0146186800F025B800BF9C000020E3
:1061600070B50F4E0C463168054611B900F08AFD36
:1061700030602146284600F085FD431C03D14FF0D6
:10618000FF34204670BDC41C24F00304A042F8D0A4
:10619000211A284600F076FD0130F2D1EFE700BF6A
:1061A000E01500202DE9F843CD1C25F00305083546
:1061B0000C2D38BF0C25002D064601DBA94204D961
:1061C0000C2333600020BDE8F883DFF8D48000F0B2
:1061D00011F9D8F800301C4644BB29463046FFF779
:1061E000BFFF431C044658D1D8F800402746002F73
:1061F00043D1002C4BD023683946304604EB0309C9
:1062000000F040FD814542D1216830466D1A294693
:10621000FFF7A6FF01303AD023682B442360D8F85B
:1062200000305A6862BBC8F800700FE02268521B49
:1062300020D40B2A17D96119A342256018BF5960D1
:10624000636808BFC8F8001062514B60304600F028
:10625000D7F804F10B00231D20F00700C21A1CBF61
:106260001B1AA350AFE76268A3420CBFC8F8002016
:106270005A60EBE723466468AEE73C467F68B6E7C2
:106280001A465B68A342FBD100235360DEE70C2370
:106290003046336000F0B4F894E70560D6E700BFFD
:1062A000E4150020B1F90C20F8B5160705460C4698
:1062B00054D44B68002B02DC0B6C002B48DDE66AE3
:1062C000002E45D0002312F480522F68216A2B60E3
:1062D00030D0626DA389590705D56368D21A636B04
:1062E0000BB1236CD21A00232846E66A216AB04714
:1062F000431CA38906D129681D292BD8284ACA40E6
:10630000D60727D5002262602269D904226004D50D
:10631000421C01D12B6803B96065616B2F60B9B174
:1063200004F14403994202D0284600F0F9FC00230E
:1063300063630DE001232846B0470246501CC9D1D3
:106340002B68002BC6D01D2B01D0162B1DD12F6022
:10635000002021E043F040031BB21AE00F69002F38
:10636000F6D0930718BF00230E6808BF4B69F61BD1
:106370000F608B60002EEBDD33463A462846216ADB
:10638000D4F828C0E047002807DCB4F90C3043F00B
:1063900040034FF0FF30A381F8BD0744361AE9E708
:1063A0000100402038B50B6905460C4613B900259D
:1063B000284638BD18B1036A0BB9FEF72DFEB4F9B3
:1063C0000C30002BF3D0626ED00704D4990502D4B0
:1063D000A06DFEF7C6FE28462146FFF763FF636EF9
:1063E0000546DA07E4D4A3899B05E1D4A06DFEF746
:1063F000B9FEDDE70148FEF7B4BE00BFDC150020A2
:106400000148FEF7AFBE00BFDC15002070B5C669BD
:1064100004460D4676B91020FFF79AFE0246E06169
:1064200020B96B21174B1848FEF7BEFEC0E9016684
:106430000660C660E669F36883B1E369DB6853F818
:106440002500B8B9012101FA05F6721D2046920017
:1064500000F051FC60B1C0E901560EE02122042198
:10646000204600F048FCE369F060DB68002BE4D1D3
:10647000002070BD026843F825200023C0E90333E3
:10648000F7E700BF397E0108CA7E010870B5C6690A
:1064900005460C4676B91020FFF75AFE0246E86121
:1064A00020B98F21084B0948FEF77EFEC0E901663E
:1064B0000660C6603CB1EB696268DB6853F8221085
:1064C000216043F8224070BD397E0108CA7E010870
:1064D0002DE9F04107460C461E4600200D6901F1EA
:1064E000140CDCF80030013099B202FB01611E0C83
:1064F0000B0C02FB063389B201EB034185424FEAE4
:1065000013464CF8041BECDC0EB3A368AB4219DC59
:10651000616838460131FFF779FF804628B90246A5
:10652000BA210C4B0C48FEF73FFE226904F10C0126
:10653000023292000C30FEF729FE21463846FFF762
:10654000A5FF444604EB850301355E6125612046C5
:10655000BDE8F081A87E0108CA7E01080346B0F5B7
:10656000803F3ABF030410200020B3F1807F3CBF7E
:106570001B020830B3F1805F3CBF1B010430B3F154
:10658000804F3CBF9B000230002B05DB13F0804F97
:1065900000F1010008BF202070470368024613F095
:1065A00007000BD0D90721D4980749BF5B089B0887
:1065B000012013605CBF02201360704799B209B9D3
:1065C00010201B0CD9B209B908301B0A190704BFE7
:1065D0001B090430990704BF9B080230D90703D474
:1065E0005B0800F1010003D0136070470020704782
:1065F0002020704710B50C460121FFF707FF024627
:1066000028B940F24511044B0448FEF7CDFD0123A3
:106610004461036110BD00BFA87E0108CA7E010865
:106620002DE9F04F17460A693B6989469A42A2BF95
:106630003B460F4699463D69D9F810A0BB6879687A
:1066400005EB0A06B34285B0B8BF0131FFF7DEFEA5
:1066500030B902464FF4B171404B4148FEF7A4FDFA
:1066600000F114042346002204EB860E734520D368
:1066700007F1140809F1140108EB850501EB8A0301
:106680000293EB1B153B23F0030304331537BD4284
:1066900038BF04230193029B03918B420CD8002E38
:1066A00003DD5EF8043D002B55D0066105B0BDE862
:1066B000F08F43F8042BD9E7B1F800A0BAF1000F2E
:1066C0001FD0C446A14600275CF8042BD9F800303F
:1066D0001FFA82FB9BB20AFB0B333B44D9F80070D4
:1066E000120C3F0C0AFB027202EB13429BB243EA0C
:1066F000024365454FEA124749F8043BE4D8019B41
:10670000E750039B0431B3F80290B9F1000F20D099
:106710004746A4464FF0000A2368B7F800B0BCF81B
:1067200002209BB209FB0B22524443EA02434CF87D
:10673000043B57F8043B4FEA134ABCF80030BD4213
:1067400009FB0A3303EB12434FEA134AE5D8019AD7
:10675000A35004349FE7013EA1E700BFA87E0108D3
:10676000CA7E01082DE9F843154612F003020746D8
:106770000E4607D0254C013A002354F82220FFF79B
:10678000A7FE0646AD103DD0FC697CB91020FFF78E
:10679000DFFC0246F86128B940F2B3111C4B1D48DA
:1067A000FEF702FDC0E901440460C460D7F81C8014
:1067B000D8F808404CB940F271213846FFF71AFF6B
:1067C00000230446C8F8080003604FF00009EB07F7
:1067D0000AD5314622463846FFF722FF8046314629
:1067E0003846FFF753FE46466D100BD0206838B987
:1067F000224621463846FFF713FF2060C0F800907C
:106800000446E4E73046BDE8F88300BF307F010866
:10681000397E0108CA7E01082DE9F0470C4607467B
:1068200091462369496803EB6218A3684FEA621A2C
:1068300008F10106B3420BDB3846FFF7E7FD0546DA
:1068400048B902464FF4EF71274B2848FEF7ACFCDD
:1068500001315B00EEE7002300F1140100F11002AA
:106860001846534533DB20692AEAEA7A04F1140317
:1068700019F01F0901EB8A0103EB800C2BD08A462B
:106880000022C9F1200E186800FA09F010434AF8F6
:10689000040B53F8042B9C4522FA0EF2F3D8ACEB10
:1068A0000403153B23F00303043304F11500604592
:1068B00088BF0423CA500AB108F10206013E3846D7
:1068C00021462E61FFF7E2FD2846BDE8F08742F839
:1068D000040F0133C5E7043953F8042B9C4541F8F4
:1068E000042FF9D8EAE700BFA87E0108CA7E010894
:1068F00003460A69006930B5801A0ED11433143189
:1069000003EB820401EB820154F8045D51F8042D7D
:10691000954203D005D24FF0FF3030BDA342F3D3F0
:10692000FBE70120F9E700002DE9F74F894606460D
:10693000114648461446FFF7DBFF051E12D12946D3
:106940003046FFF763FD024628B940F237213E4B3F
:106950003E48FEF729FC0123C0E90435104603B088
:10696000BDE8F08FBCBF4B46A1463046D9F80410B5
:10697000BABF1C4601250025FFF748FD024618B99D
:1069800040F24521304BE3E700F1140BD9F81070C9
:1069900009F11003C5604FF0000C09F11405D94648
:1069A000266904F1140E05EB87080EEB86060193A9
:1069B000019B5EF8040B53F804AF81B201931FFAF8
:1069C0008AF35B1A000C6344C0EB1A4000EB2340CF
:1069D0009BB243EA004376454FEA204C49F8043B1A
:1069E000E6D8331B153B23F0030315340433A642CA
:1069F00038BF04231D445B441E462C4644450ED339
:106A000008F10301491B21F00301033DA84538BFEC
:106A100000210B4453F8041D99B117619EE7E64627
:106A200054F8041B1FFA81FCF444080C714400EB79
:106A30002C4089B241EA00414FEA204C46F8041B41
:106A4000DCE7013FE6E700BFA87E0108CA7E010837
:106A50002DE97343012190469946089EFFF7D6FC25
:106A6000044630B9024640F20F31234B2348FEF76B
:106A70009BFBC9F30A55C9F313030DB143F480130B
:106A80000193B8F1000324D068460093FFF785FD19
:106A9000DDE90012D8B1C0F1200302FA03F30B4381
:106AA000C24063610192019B002B0CBF01220222B4
:106AB000A3612261ADB1A5F2334505443560C0F153
:106AC0003500099B1860204602B0BDE87083616103
:106AD000E9E701A8FFF761FD019B01226361203016
:106AE000E7E7A0F2324004EB820330601869FFF759
:106AF00035FDC0EB4210E4E7A87E0108CA7E01081C
:106B000010B50C46B1F90E1000F0AAF80028ABBF82
:106B1000636DA3891B1823F48053ACBF6365A38105
:106B200010BD2DE9F0411F468B890546DB050C465B
:106B3000164605D502230022B1F90E1000F07EF8AA
:106B4000A389324623F48053A38128463B46B4F9F7
:106B50000E10BDE8F04100F0A5B810B50C46B1F933
:106B60000E1000F06BF8431CA38915BF606523F479
:106B7000805343F48053A38118BFA38110BDB1F9A2
:106B80000E1000F0A1B800000EB403B5014603AB2F
:106B9000054853F8042B0068019300F031F902B066
:106BA0005DF804EB03B070479C0000202DE9F04134
:106BB000074614460D4621B91146BDE8F041FFF7DE
:106BC000F1BA2AB900F0ACF825462846BDE8F081B4
:106BD00000F040FA8442064602D8B4EB500FF4D8D5
:106BE00021463846FFF7DEFA804608B94546ECE70D
:106BF000B4422246294628BF3246FEF7C7FA294644
:106C0000384600F08DF8F1E7884210B501EB020438
:106C100002D98442234607D8431EA14208D011F866
:106C2000012B03F8012FF8E7014602448A4200D104
:106C300010BD13F8014D02F8014DF7E738B50446D1
:106C4000084611460022054D2A601A46F7F775F8E6
:106C5000431C02D12B6803B1236038BDE815002026
:106C600038B50446084611460022054D2A601A46EA
:106C7000F7F722F8431C02D12B6803B1236038BD1B
:106C8000E815002038B50023054D044608462B6062
:106C9000F7F760F8431C02D12B6803B1236038BDBD
:106CA000E815002038B50446084611460022054D77
:106CB0002A601A46F3F772FB431C02D12B6803B11A
:106CC000236038BDE815002038B50023054D044683
:106CD00008462B60F7F70DF8431C02D12B6803B16F
:106CE000236038BDE8150020062008B500F0E4FA5E
:106CF0000120F6F7D6FF70B5A1FB025434B929463E
:106D0000FFF750FA064628B9304670BD0C2200261F
:106D10000260F9E72A462146FEF7F0F9F4E70000A1
:106D200038B50546002940D051F8043C0C1F002B13
:106D3000B8BFE418FFF75EFB1C4A136833B9636001
:106D400014602846BDE83840FFF75ABBA34208D973
:106D5000206821188B4201BF19685B6809182160FF
:106D6000EDE71A465B680BB1A342FAD911685018D7
:106D7000A0420BD120680144501883421160E0D139
:106D800018685B68084410605360DAE702D90C2386
:106D90002B60D6E7206821188B4201BF19685B6819
:106DA0000918216063605460CBE738BDE41500200A
:106DB000936810B4013B002B936007DA9469A342F7
:106DC00001DB0A2902D110BC00F04CB91368581C31
:106DD00010601970084610BC7047F8B506460F469B
:106DE0001446D518AC4201D1002007E03A4630469F
:106DF00014F8011BFFF7DCFF431CF3D1F8BD0000C2
:106E00002DE9F04F0D461446984606469DB018B140
:106E1000036A0BB9FEF700F96B6ED90705D4AB898D
:106E20009A0502D4A86DFEF79CF9AB891B0701D522
:106E30002B699BB92946304600F052F970B16B6E50
:106E4000DC0704D54FF0FF301DB0BDE8F08FAB89F3
:106E50009805F7D4A86DFEF785F9F3E700230993A9
:106E600020238DF8293030234FF00109CDF80C8014
:106E7000DFF8A8818DF82A3023469A4613F8012BB3
:106E80000AB1252AF9D1BAEB040B0BD05B46224696
:106E900029463046FFF7A1FF013000F0A780099A8C
:106EA0005A4409929AF80030002B00F09F8000238A
:106EB0004FF0FF32CDE905230AF1010A049307934D
:106EC0008DF853301A935446052214F8011B534889
:106ED000FEF74EF9049AD8B9D10644BF20238DF8A5
:106EE0005330130744BF2B238DF853309AF80030EA
:106EF0002A2B15D0544600204FF00A0C079A214641
:106F000011F8013B303B092B4BD9B0B1079214E08B
:106F1000A0EB080309FA03F31343A2460493D2E754
:106F2000039B191D1B680391002BBBBF5B4242F002
:106F3000020207930793B8BF049223782E2B0AD13D
:106F400063782A2B32D1039B02341A1D1B680392EB
:106F500043EAE3730593DFF8C8A003225046217883
:106F6000FEF706F938B14022049BA0EB0A008240EC
:106F700013430134049314F8011B062229488DF8A9
:106F80002810FEF7F5F800283FD0274B1BBB039BCA
:106F9000073323F0070308330393099B3B4409930A
:106FA0006AE70C4601200CFB0232A8E700234FF0F1
:106FB0000A0C194601340593204610F8012B303A8B
:106FC000092A03D9002BC6D00591C4E70446012342
:106FD0000CFB0121F0E703AB00932A463046134B2C
:106FE00004A9FDF7D1FB0746781CD6D16B6ED907F3
:106FF00005D4AB899A0502D4A86DFEF7B3F8AB8926
:107000005B063FF51FAF09981EE703AB00932A46C6
:107010003046064B04A9FDF755FEE4E7B97E0108AA
:10702000BF7E0108C37E010889470108DB6D0108A6
:1070300082B001B901A942B14BB113780B6012784B
:10704000101E18BF012002B070471046FBE76FF01A
:107050000100F8E751F8043C181F002BBCBF0B5887
:10706000C0187047F8B50E461446054618B1036AB5
:107070000BB9FDF7D1FFA369A360A3891A0701D556
:10708000236943B92146284600F02AF818B14FF089
:10709000FF373846F8BD23682269F6B2981A63694B
:1070A0003746834205DC21462846FFF77BF9002856
:1070B000EDD1A368013BA36023685A1C22601E70B7
:1070C0006269431C9A4204D0A389DB07E1D50A2EEA
:1070D000DFD121462846FFF765F90028D9D0D6E749
:1070E00038B5294B054618680C4618B1036A0BB928
:1070F000FDF792FFB4F90C30190722D4DA0607D451
:1071000009222A6043F040034FF0FF30A38133E0AF
:10711000580712D5616B41B104F14403994202D082
:107120002846FFF7FDFD00236363A38923F02403B2
:10713000A3810023636023692360A38943F00803CC
:10714000A38123694BB9A38903F42073B3F5007FAE
:1071500003D02146284600F04BF8B4F90C3013F068
:1071600001020AD00022A26062695242A261226931
:1071700042B913F08000C5D138BD990758BF626984
:10718000A260F4E70020F7E79C00002003460846D1
:1071900041B1FF2A04D98A224FF0FF301A607047AC
:1071A00001200A70704770B50C46B1F90E101546F3
:1071B00000291E4696B00CDAA389002113F0800F37
:1071C00014BF40234FF48063002031602B6016B061
:1071D00070BD6A4600F09CF80028EDDB019901F4CF
:1071E0007041A1F50053594259414FF48063EBE7D8
:1071F0008B89F7B59D0706460C4607D504F1470372
:10720000236023610123636103B0F0BD6A4601ABD3
:10721000FFF7C9FF009F054639463046FEF7C2FF1B
:1072200048B9B4F90C309A05EED423F0030343F0C7
:107230000203A381E2E7A389C4E9040743F08003C2
:10724000A381019B20605BB13046B4F90E1000F0C1
:107250003BF828B1A38923F0030343F00103A38182
:10726000A3891D43A581CFE71F2938B505460C46E4
:1072700004D9162303604FF0FF3038BDC26B12B142
:1072800052F821304BB9284600F040F8224601461A
:107290002846BDE8384000F027B8012B0AD0591C19
:1072A00003D1162303600120E7E70021204642F8BE
:1072B000241098470020E0E7024B01461868FFF7CA
:1072C000D3BF00BF9C00002038B50023054D044605
:1072D00008462B60F6F727FD431C02D12B6803B14B
:1072E000236038BDE815002038B50023064D04465C
:1072F000084611462B60F6F7C4FC431C02D12B68EC
:1073000003B1236038BD00BFE8150020F6F7B2BC1A
:1073100038B50023064D0446084611462B60F6F7A3
:10732000F3FC431C02D12B6803B1236038BD00BFBE
:10733000E8150020F8B500BFF8BC08BC9E467047B1
:0C734000F8B500BFF8BC08BC9E467047C2
:10735000434F4E4E30204572726F723A2025640AB8
:1073600000000000436F6E6E6563746F723A2055C3
:107370006E6B6E6F776E0A00436F6E6E6563746F2F
:10738000723A20556E706C75676765640A0000007C
:10739000436F6E6E6563746F723A20446973616205
:1073A0006C65640A00000000436F6E6E6563746F65
:1073B000723A20507265706172696E670A0000004F
:1073C000436F6E6E6563746F723A204175746852D4
:1073D000657175697265640A00000000436F6E6E26
:1073E0006563746F723A2057616974696E67466F9E
:1073F00072456E657267790A00000000436F6E6E19
:107400006563746F723A204368617267696E675092
:10741000617573656445560A00000000436F6E6E27
:107420006563746F723A204368617267696E675072
:107430006175736564455653450A0000436F6E6E6F
:107440006563746F723A204368617267696E670A98
:1074500000000000436F6E6E6563746F723A2041E6
:1074600075746854696D656F75740A00436F6E6E4C
:107470006563746F723A2046696E69736865640A61
:1074800000000000436F6E6E6563746F723A2046B1
:10749000696E6973686564455653450A00000000CB
:1074A000436F6E6E6563746F723A2046696E6973DE
:1074B00068656445560A0000436F6E6E6563746FBD
:1074C000723A205265706C756767696E670A0000D2
:1074D0004350207374617465206368616E676564EE
:1074E0003A202564202D3E2025640A004350206464
:1074F000757479206368616E6765643A202575202C
:107500002D3E2025750A00004649524520414C4138
:10751000524D206163746976617465640A000000ED
:10752000434353206D6F64756C652073746172748E
:107530000A00000053657269616C206E756D6265AA
:10754000723A2025640A0000426F617264207265FD
:10755000766973696F6E3A2025640A004657207673
:10756000657273696F6E3A2025642E25642E25643A
:107570000A000000505355206F6E2074696D656FCE
:1075800075740A00436F6E746163746F7220657264
:10759000726F722C2073746F7070696E672E2E2E4E
:1075A0000A000000505355206F66662074696D65AF
:1075B0006F75740A00000000504520004E45200001
:1075C000464520004F52452000000000444D412018
:1075D000000000005541525425752048414C20655B
:1075E00072726F72206465636F64653A204E4F4E0D
:1075F000450A00005541525425752048414C2065EC
:1076000072726F72206465636F64653A202573251A
:10761000732573257325732573207261773D307848
:107620002530386C780A00005541525433205258A6
:107630002061726D206661696C656420282573295C
:107640003A2048414C5F5374617475733D25642042
:107650006572725F61667465723D30782530386C92
:10766000780A000055415254332052582061726DFF
:10767000206661696C65642064657461696C73007F
:1076800055415254332052582064726F703A20771B
:10769000726F6E6720687561727420696E2052780F
:1076A0004576656E7443616C6C6261636B20287310
:1076B000697A653D2575290A00000000554152543C
:1076C000332052582064726F703A205278457665A4
:1076D0006E742073697A653D30202869646C652C6E
:1076E000206E6F207061796C6F6164290A00000060
:1076F00052784576656E7443616C6C6261636B00B1
:1077000055415254332052582064726F703A20739E
:10771000697A653D2575203E2072785F62756666E0
:10772000657220257520286F766572666C6F772CE0
:10773000206E6F7420706172736564290A00000006
:107740005541525425752048414C206572726F7224
:107750002028495352293A207261773D30782530EC
:10776000386C7820E28094205258206D6179206234
:107770006520636F7272757074656420756E7469CC
:107780006C2072652D61726D0A0000004572726F87
:107790007243616C6C6261636B000000554152542E
:1077A0003320545820444D4120726573656E642027
:1077B0006661696C656400004553544F50207472D3
:1077C000696767657265640A0000000053746F7032
:1077D00070696E67206368617267696E672E2E2E0E
:1077E0000A00000046696E697368656445562C207E
:1077F00073746F7070696E672E2E2E0A0000000081
:10780000457665726573742074696D656F75740A69
:1078100000000000457665726573742074696D65BB
:107820006F75742C2073746F7070696E6720636855
:10783000617267696E672E2E2E0A000043686172BE
:1078400067696E67206572726F722025642C2073E1
:1078500074617465202D3E2064697361626C656497
:107860000A0000004368617267696E672070657284
:107870006D69747465642C2073746172742063681C
:10788000617267696E670A0043617220756E706C81
:1078900075676765640A00005265706C7567676993
:1078A0006E672E2E2E0A00005265706C7567676930
:1078B0006E672066696E69736865642C20627574F2
:1078C0002063617220756E706C75676765640A006D
:1078D0005265706C756767696E672066696E69735B
:1078E0006865642C2063617220706C7567676564DD
:1078F0002C207374617465202D3E2061757468209E
:1079000072657175697265640A000000496E697478
:107910000000000043435320696E69740A000000B0
:10792000554152543320545820444D4120737461C2
:107930007274206661696C6564000000457665724A
:1079400065737420726573657420636F6D6D616E0D
:10795000640A000055415254332052582077617216
:107960006E3A20636D64203078253032782043529F
:10797000432F6C656E204F4B20627574206E6F2014
:107980007377697463682063617365202865787014
:1079900065637465645F7061796C6F616420767390
:1079A000206170706C795F636F6D6D616E64290A20
:1079B0000000000055415254332052582064726F29
:1079C000703A20746F6F5F73686F7274206C656EAD
:1079D0003D302028656D707479206368756E6B2961
:1079E0000A00000055415254332052582064726FEF
:1079F000703A20746F6F5F73686F7274206C656E7D
:107A00003D312062303D3078253032780A00000068
:107A100055415254332052582064726F703A20748A
:107A20006F6F5F73686F7274206C656E3D32206299
:107A3000303D3078253032782062313D3078253045
:107A400032780A0055415254332052582064726FE4
:107A5000703A206372635F6D69736D61746368204F
:107A6000636D643D30782530327820746F74616CBA
:107A70005F6C656E3D2575207061796C6F61645F28
:107A80006C656E3D2575206372635F72783D30785A
:107A900025303478206372635F63616C633D3078B6
:107AA000253034780A000000554152543320525892
:107AB0002064726F703A20756E6B6E6F776E5F63C5
:107AC0006D6420636D643D30782530327820746FAA
:107AD00074616C5F6C656E3D2575207061796C6FAB
:107AE00061645F6C656E3D25750A00005541525416
:107AF000332052582064726F703A206C656E5F6D4F
:107B000069736D6174636820636D643D30782530FE
:107B100032782065787065637465645F7061796C34
:107B20006F61643D257520676F745F7061796C6F5C
:107B300061643D257520746F74616C5F6C656E3D8A
:107B400025750A005761746368646F670000000060
:107B50005541525433207761746368646F672072B3
:107B60006561726D0000000025733A206572723DF8
:107B700030782530386C7820673D256C7520727818
:107B80003D256C752074785F627573793D25750AA3
:107B90000000000055415254322052582069646C54
:107BA00065206576656E742077697468207A6572E1
:107BB0006F2073697A650A00554152543220525839
:107BC00020696E76616C6964207061636B657420F6
:107BD0006C656E3D25750A0055415254352052584A
:107BE0002069646C65206576656E742077697468B9
:107BF000207A65726F2073697A650A005541525484
:107C00003520525820696E76616C6964207061631A
:107C10006B6574206C656E3D25750A0055415254A4
:107C20003220545820627573792C2061626F72740F
:107C3000207472616E736D6974206265666F72651F
:107C400020726573656E640A00000000554152544D
:107C50003220545820444D41207374617274206660
:107C600061696C65640000005541525432205258DD
:107C7000207061636B65742074696D656F75742025
:107C8000282575206D73290A0000000055415254C3
:107C90003220525820444D412061726D2066616946
:107CA0006C65640055415254352052582049542087
:107CB00061726D206661696C6564000055415254C3
:107CC00032207265636F766572207374617274001E
:107CD0005541525435207265636F76657220737416
:107CE0006172740025733A20696E7374616E636506
:107CF0003D30782530386C78206572723D307825BB
:107D000030386C7820673D256C752072783D256C85
:107D1000750A000053657420436F6E6669673A20E8
:107D200025732025640A0000506F776572206C6906
:107D30006D69743A2025640A00000000436861728E
:107D40006765207065726D69743A2025640A0000C9
:107D500001000100010001000100040001002C00ED
:107D60000100000000000000000000000102030408
:107D700006070809000000000102030400000405D2
:107D80000607080900000000000D000001020304BE
:107D900005060708090A0B0C0D0E0F10000004055C
:107DA0000607080900000000000D0000010203049E
:107DB00005060708090A0B0C0D0E0F10494E460068
:107DC000696E66004E414E006E616E0030003031CB
:107DD0003233343536373839414243444546003032
:107DE0003132333435363738396162636465660061
:107DF0002C2066756E6374696F6E3A200061737330
:107E0000657274696F6E2022257322206661696C29
:107E100065643A2066696C6520222573222C206CEB
:107E2000696E65202564257325730A00496E6669AD
:107E30006E697479004E614E005245454E54206D76
:107E4000616C6C6F63207375636365656465640062
:107E50002F6275696C642F676E752D746F6F6C730C
:107E60002D666F722D73746D33325F31332E332E66
:107E700072656C312E32303234303932362D313732
:107E800031352F7372632F6E65776C69622F6E6563
:107E9000776C69622F6C6962632F7374646C6962BA
:107EA0002F64746F612E630042616C6C6F6320738A
:107EB000756363656564656400232D302B2000685D
:107EC0006C4C00656667454647002F6275696C64B7
:107ED0002F676E752D746F6F6C732D666F722D73B7
:107EE000746D33325F31332E332E72656C312E3226
:107EF000303234303932362D313731352F737263A9
:107F00002F6E65776C69622F6E65776C69622F6C76
:107F10006962632F7374646C69622F6D707265633C
:107F20002E63004300504F534958002E00000000BC
:107F300005000000190000007D00000000000000A6
:107F40000080E03779C34143176E05B5B5B8934655
:107F5000F5F93FE9034F384D321D30F94877825A21
:107F60003CBF737FDD4F1575000000000000F03F3F
:107F70000000000000002440000000000000594004
:107F80000000000000408F40000000000088C34057
:107F900000000000006AF8400000000080842E41CC
:107FA00000000000D01263410000000084D7974118
:107FB0000000000065CDCD41000000205FA002421E
:107FC000000000E876483742000000A2941A6D4293
:107FD000000040E59C30A2420000901EC4BCD64286
:107FE00000003426F56B0C430080E03779C3414331
:107FF00000A0D8855734764300C84E676DC1AB43A7
:10800000003D9160E458E143408CB5781DAF1544C4
:1080100050EFE2D6E41A4B4492D54D06CFF080449F
:10802000F64AE1C7022DB544B49DD9794378EA44B4
:108030000020202020202020202028282828282038
:108040002020202020202020202020202020202030
:108050002088101010101010101010101010101098
:108060001004040404040404040404101010101088
:108070001010414141414141010101010101010152
:1080800001010101010101010101010110101010A4
:108090001010424242424242020202020202020224
:1080A0000202020202020202020202021010101078
:1080B00020000000000000000000000000000000A0
:1080C00000000000000000000000000000000000B0
:1080D00000000000000000000000000000000000A0
:1080E0000000000000000000000000000000000090
:1080F0000000000000000000000000000000000080
:10810000000000000000000000000000000000006F
:10811000000000000000000000000000000000005F
:10812000000000000000000000000000000000004F
:04813000000000004B
:08813400F400FF7F01000000D0
:04813C000D820008A8
:04814000E9810008C9
:10814400E40100000606060601000000FA00000A29
:10815400050A050000000000FF00000A0A0A0A00E0
:1081640000000000400000320A320040000000001D
:10817400008000320A320000800000000000FF0A84
:108184000A0A0A000000000000FF00320A32000060
:1081940020000000FFFFFF320A3200FFFFFF000053
:1081A400FF0000320A3200200000640000FFFF00DC
:1081B400000000000000000052555301000000FEC2
:1081C400529E66000024F40010000000010000002C
:1081D4000000000003000000A0140020A000002004
:1081E40000000000A01400200815002070150020D5
:1081F400000000000000000000000000000000007B
:10820400000000000000000000000000000000006A
:10821400000000000000000000000000000000005A
:108224000000000000000000000000004300000007
:10823400000000000000000000000000000000003A
:1082440000000000000000000000000043000000E7
:10825400000000000000000000000000000000001A
:1082640000000000000000000000000043000000C7
:1082740000000000000000000000000000000000FA
:1082840000000000000000000000000043000000A7
:1082940000000000000000000000000000000000DA
:1082A4000000000000000000000000004300000087
:1082B40000000000000000000000000000000000BA
:1082C4000000000000000000000000004300000067
:1082D400000000000000000000000000000000009A
:1082E4000000000000000000000000004300000047
:1082F400000000000000000000000000000000007A
:108304000000000000000000000000008D71010862
:108314003170010800000000308001082B7F010843
:108324002B7E01082B7E01082B7E01082B7E010881
:108334002B7E01082B7E01082B7E01082B7E010871
:108344002B7E0108FFFFFFFFFFFFFFFFFFFFFFFF83
:10835400FFFF0000010041534349490000000000B1
:108364000000000000000000000000000000000009
:108374000000000000004153434949000000000090
:1083840000000000000000000000000000000000E9
:088394000000000000000000E1
:040000050800E68D7C
:00000001FF
